:020000040000FA
:107800005469616E59696E673130300000000000C4
:1078100054593230302E3038303030306200000071
:10782000424154333247313339474B3634464200B4
:1078300043414E5F5354440000000000000000002C
:1078400043414E5F43485F300000000000000000ED
:1078500043414E5F3530304B6270730000000000D2
:10786000E8070000E0070000DF070000000000005C
:020000040000FA
:10800000802F0020DD800000E5800000E780000078
:108010000000000000000000000000000000000060
:10802000000000000000000000000000EF800000E1
:108030000000000000000000F380000089A701009C
:10804000BD0A0100010B0100310B0100610B0100B1
:10805000910B0100C10B0100F10B0100210C01008B
:10806000510C0100810C0100B50C0100C90C01008C
:10807000D90C01000D0D01001D0D01002D0D010099
:10808000610D0100A50D0100ED0D0100350E01008F
:108090007D0E0100C50E0100D50E0100090F010083
:1080A0003D0F01006D0F0100A10F0100D50F010070
:1080B000E50F0100F50F0100291001005D1001001E
:1080C000EF3FE8FF0448854600F02CFA00480047DF
:1080D0006DE90100C046C046802F00201648804749
:1080E00016480047FEE7FEE7FEE7FEE7FEE7FEE78D
:1080F000FEE7FEE7FEE7FEE7FEE7FEE7FEE7FEE758
:10810000FEE7FEE7FEE7FEE7FEE7FEE7FEE7FEE747
:10811000FEE7FEE7FEE7FEE7FEE7FEE7FEE7FEE737
:10812000FEE7FEE7FEE7FEE7FEE7FEE7FEE7FEE727
:10813000FEE7FEE7FEE7000091AD0100C58000000C
:1081400030B50B46014600202022012409E00D46EF
:10815000D5409D4205D31D469540491B2546954077
:1081600040191546521E002DF1DC30BD70B50024BB
:108170002546002801DA01244042002901DA0125C0
:108180004942FFF7DDFFAC4200D04042002C00D056
:10819000494270BDF0B51FB40646002082B00546C6
:1081A0004024019100901BE0019922460F46304681
:1081B00000F066F9049A059B801A994110D3104685
:1081C0001946224600F04CF9361A8F410197224693
:1081D00001200021009F00F043F938184D41009024
:1081E0002046641E0028DFDC019B009829463246A9
:1081F00007B0F0BDF0B51FB486B00020009001902C
:1082000002900698069980B204900798090C02041F
:108210000014114307900027089D099806913E46D7
:108220003C4603900398A9B20204000C0390049802
:108230002D0C154348430021224600F011F9C719BF
:10824000714110340E46402CECDB3846029A00F0A7
:1082500007F9009A019B80180090594102980191FA
:10826000103002904028CCDB00980BB0F0BD0346E4
:108270000B439B0703D009E008C9121F08C0042A5A
:10828000FAD203E00B780370401C491C521EF9D24D
:108290007047D2B201E00270401C491EFBD2704709
:1082A0000022F6E710B513460A4604461946FFF7C2
:1082B000F0FF204610BD30B504460020034600E024
:1082C0005B1C934203D2E05CCD5C401BF8D030BD18
:1082D0000321001D401E037812021A43491EF9D5DE
:1082E00010467047034603220870000A491C521EBC
:1082F000FAD518467047024670B54A40D30FDB07DF
:1083000040002DD04A002AD0010E140E00021202A5
:108310000919400A520A8418E50104465443000A28
:10832000120A2E045043A4194219200CC543AA185E
:10833000120C0125AD03521C521912047F3924047A
:1083400000D0521C104301D44000491EC2B20C069A
:10835000C0092018401C4008802A02D003E00020F9
:1083600070BD40084000002900DA0020184370BDAD
:1083700070B502464A40D50F40004A00ED0740085C
:108380005208002814D0002A12D0C40DD30D410287
:108390000120C0055202490A520AE41A09181218AB
:1083A0007D34914201D3641C00E04900002C01DAC5
:1083B000002070BD0023914201D3891A0343400875
:1083C00049000028F7D100290AD0914202D10121A9
:1083D000C90705E0914201D2012101E00121C94311
:1083E000E005C018401900F05CF870BD10B500221F
:1083F0009623114600F05DF810BDC20FD207400071
:1084000040080BD0C10D0723DB01C9184002090544
:10841000400A1143C208400711437047002001463B
:108420007047000010B5002904DB0124E407404236
:108430008C412146002B04DB1C460123DB07524202
:10844000A341994200D1904210BD00000122D20701
:10845000002800DB101A002900DB511A88427047FF
:1084600010B5202A04DB0146203A9140002010BDBF
:10847000914020239C1A0346E3401943904010BDCD
:1084800010B5202A04DB0846203AD040002110BD58
:108490000B46D340D0402024A21A914008431946ED
:1084A00010BD002904DA401C490001D140084000F9
:1084B000704770B40024050C05D11024000402D1CB
:1084C000002921D01124050E01D100020834050F26
:1084D00001D10001241D850F01D18000A41C0028BA
:1084E00001DB4000641C002908D020252E1B0D460E
:1084F000F540A14000D001212943084301061B1B80
:10850000000ADB1D02D5002070BC7047DB0518187F
:1085100080180029F8DA401C4900F5D170BC4008E9
:1085200040007047064C0125064E05E0E36807CC85
:108530002B430C3C98471034B442F7D3FFF7C6FDE9
:108540004CFD01006CFD010070B58C180578401CD5
:108550006B075B0F01D10378401C2A1106D102780A
:10856000401C03E006780E70401C491C5B1EF9D1CC
:108570002B0705D40023521E0DD40B70491CFAE7BB
:108580000378401CCB1A921C03E01D780D70491C27
:108590005B1C521EF9D5A142D8D3002070BD70B526
:1085A00006F076FE0524204616F09AF900252846A6
:1085B00006F062FE204616F093F90126304606F0DA
:1085C00037FE204616F08CF9284606F031FE20468C
:1085D00016F086F9304606F04FFE204616F080F978
:1085E00070BDB0B506F054FE0524204616F078F9AB
:1085F0000125284606F040FE204616F071F928466F
:1086000006F016FE204616F06BF9002006F010FE6C
:10861000204616F065F9B0BDF0B581B006F024FE35
:10862000052016F05DF908270026012006F000FE5F
:108630000524204616F054F9204616F051F906F0AC
:1086400009FE0546204616F04BF9002006F0F0FD25
:10865000204616F045F976002E437F1E3806E4D1F9
:10866000F0B201B0F0BD70B50446002006F0E0FDA8
:1086700006F00EFE052016F033F90826E0B2C00918
:1086800006F0FAFD0525284616F02AF9012006F025
:10869000CFFD284616F024F9002006F0C9FD284633
:1086A00016F01EF9284616F01BF96400761E3006F7
:1086B000E4D1052016F014F9012070BDF0B583B0A7
:1086C000019314460E4607460120384302900325C5
:1086D00004E000F08EF86D1E280631D000F067F837
:1086E0003846FFF7C0FF00F0A7F80028F1D1304668
:1086F000FFF7B9FF00F0A0F80028EAD100F057F822
:108700000298FFF7B0FF00F097F80028E1D1019838
:1087100002280BD3451E0026FFF77EFF2070FFF7CF
:108720003EFF641C761CF0B28542F5DCFFF774FF57
:108730002070FFF756FF00F05CF8202003B0F0BD7A
:10874000102003B0F0BDF0B583B01C46009201913B
:108750000290032504E000F04CF86D1E280623D09B
:1087600000F025F80298FFF77EFF00F065F800287A
:10877000F1D10198FFF777FF00F05EF80028EAD109
:10878000002C0CD00026009F3878FFF76CFF00F01B
:1087900053F80028DFD1761C7F1CA642F4D300F0EA
:1087A00028F8082003B0F0BD102003B0F0BDB0B52C
:1087B00006F06EFD0524204616F092F801252846A5
:1087C00006F036FD204616F08BF8284606F054FDDC
:1087D000204616F085F80025284606F04DFD204677
:1087E00016F07EF8284606F023FD642016F078F88F
:1087F000B0BDB0B506F04CFD0524204616F070F86B
:108800000025284606F014FD204616F069F8284693
:1088100006F032FD204616F063F80125284606F0E2
:1088200007FD204616F05CF8284606F025FD64207A
:1088300016F056F8B0BD0000B0B506F015FD0524E1
:10884000204616F04DF8012006F0F2FC204616F006
:1088500047F80B4D06F0FEFC044606F0E3FC002C46
:1088600002D06D1E2804F5D10525284616F038F8EB
:10887000002006F0DDFC284616F032F82046B0BD98
:1088800033210000034801780B2901D8491C0170ED
:108890007047C0466F2B002070B584B0002503954B
:1088A00002950195009506F0BDFC0F20C6430E4CC5
:1088B0001036F1B2A0206A461023FFF744FF20468D
:1088C00016F00EF8204616F00BF8912EF0D3A020EB
:1088D000B0216A461023FFF736FF204616F000F855
:1088E0000248058004B070BD581B0000622B0020B8
:1088F00070B5022902D2EB24E0B270BD891EEB25CF
:108900000022134605E0401C5B1CDDB2A94225464F
:108910000EDB04786C40154604E034466E1C072DCF
:108920003546F0D26608E407F7D09A246640F4E7AB
:10893000E0B270BDF0B591B00C91417810AA117001
:1089400083781B025918C37804792402E3181B04A6
:1089500059180B0ED3700C0C94700D0A55700B91B6
:1089600008956918099409190A93C9180278D2431D
:108970008918427983791B029A18C379047A2402F0
:10898000E3181B049A188918130A0693C918130CC4
:108990000593C9180792120E04928918827AC37A35
:1089A0001B029A18037B0F90447B2402E3181B04DC
:1089B00098180918020A02928918020C0192891863
:1089C0000D910390000E0E9000200346014606E034
:1089D00032409A40D2B211435B1C082B0ED00126C4
:1089E00035469D400746024602E07F1C042FEFD02B
:1089F00010ACE45D2542F8D0521CF6E70E9C0D98B1
:108A00000019C3B20F98827B934205D0427A9142FB
:108A100002D1002011B0F0BD1021FFF769FF0C99C1
:108A2000CC72019A8A72029A4A72039A0A72049A62
:108A3000CA71059A8A71069A4A71079A0A710A9A46
:108A4000CA70099A8A70089A4A700B9A0A7011B013
:108A5000F0BDF0B58DB055220270002747720B783B
:108A60004370CA79059202728A790492C2714A7976
:108A7000039282710A7902924271CA7A0892427311
:108A80008A7A019202734E7AC6720C7A84720CAAA8
:108A900013704D782D02EB188D78C97809024919A9
:108AA0000904CB18190E01711D0CC57009931B0A1E
:108AB0000B90837038460A91D17007959570069394
:108AC000537031020919089A1202019BD21812043C
:108AD0005118089103990902029A8918059A1202FD
:108AE000049BD2181204511805913D463A4605E000
:108AF0002640AE4032436D1C082D0ED00124214685
:108B0000A9400346064602E05B1C042BF0D00CAFE4
:108B1000FF5C3942F8D0761CF6E70B9B5A72099835
:108B200006994018079940180A994018059A801824
:108B3000110A4018110C4018110E4018089A80189C
:108B4000110A4018110C4018110E4018563898732D
:108B500010211846FFF7CCFE0DB0F0BDF0B58FB078
:108B60000446FF20E070A07060700F20C0430290A8
:108B70000F302070704815F0B3FE70490868632804
:108B800001D8642008606E4F002038806D4E01903F
:108B9000308008E00B99814222D338881030388029
:108BA00080B2A1286DD206F03DFB3978A02003AA3F
:108BB0001023FFF783FD30802028EED103AD0BA9F1
:108BC0002846FFF7B7FEE97B8842E6D1287855288A
:108BD000E3D15D48017800290298DBD10846D9E746
:108BE0003888A0284DD8C0B20021019105E006F0D8
:108BF00019FB3988C8B2A12943D2C1B2A02003AA67
:108C00001023FFF75BFD3080398810313980202830
:108C100037D103AD07A92846FFF78CFEE97B8842D0
:108C2000E5D128785528E2D14748007800280299F4
:108C300000D1014607988842D9D240490A68962156
:108C400051430B9A824208D90818904219D30BA9B4
:108C50000E222046FFF70BFBC9E78918814210D38B
:108C600007A90E222046FFF702FB0BA80A99818173
:108C700007980B9008980C9009980D9038880190EF
:108C8000B5E72078617809020818A178E278120225
:108C9000511809040818401C24D100200190388084
:108CA000A020B02103AA1023FFF708FD3080202860
:108CB00018D103AD0BA92846FFF73CFEE97B88429B
:108CC00010D1287855280DD11F480078002800D1F0
:108CD00002900B980299884204D20BA90E222046DA
:108CE000FFF7C5FA2078617809020818A178E278C0
:108CF0001202511809040818401C0CD10020E0721F
:108D0000A07260722072E071A07160712071E070D9
:108D1000A070607020700198388020786178090216
:108D20000818A178E27812025118090408180749B6
:108D3000086030880FB0F0BD701101005C2B00207E
:108D4000622B0020582B00205B2B0020682B00207A
:108D5000F0B581B000910646214800250570002A33
:108D60002ED01446C036631B71190F200840102204
:108D7000101A834200D303461A480278102A01D001
:108D8000042A1AD1C809FE2707405F2F13D80127EC
:108D9000B8436038C0B29E3282420CD3009A521956
:108DA000C9B2DFB23B46FFF789FC0F490880ED19D5
:108DB000A542D8D304E0082000E004200A49088036
:108DC000094801880020042902D0082900D0012088
:108DD00003490870411E8841400001B0F0BDC04603
:108DE0006E2B00205A2B00206C2B00200A4A0123F6
:108DF00013700A4A10700A4A11600A4A0021116071
:108E0000042801D105218901102801D11D208101EB
:108E1000054801807047C0465B2B00205A2B00207C
:108E20005C2B0020682B0020602B0020F0B587B061
:108E3000994D00262E80994B1B688B4224D1994C6A
:108E40002188202925D1029000920196964C002776
:108E50002760964D964E2878062809D806F0E2F944
:108E60002068401C2060B042F5D38D480421018069
:108E70002F70904C20880107029B31D08848202118
:108E80000180854D019E0BE001204002844908804D
:108E900006E003A8FFF762FE208081488021018060
:108EA0007F4800883F2807DD874988420BDC40283F
:108EB00012D0802810D010E004280DD008280AD045
:108EC000202809D009E001214A02904204D0C902B9
:108ED000884201D001E002262E80288807B0F0BD2C
:108EE000A128019E00D32780009A012A6A4D1ED135
:108EF000187B012856D1DF719F715F711F711F733D
:108F0000587B012804D1DF729F725F721F725F73FA
:108F100003AF38461946FFF79CFDF87320880028F8
:108F200046D01038C1B2A02003AA102344E0002A82
:108F3000B6D1614801780029B2D00270187859780A
:108F4000090208189978DA781202511809040818E9
:108F50005A490978002901D00F21C943884233D2E8
:108F6000274603AC20461946FFF773FDE0733978B6
:108F7000A02010232246FFF7E6FB029A484908800A
:108F800008288DD13888103038801078517809023F
:108F900008189178D2781202511809040818484923
:108FA00008607DE7597B012911D10128A3D0A7E7EB
:108FB000A02003AA10230146FFF7C5FB384908800B
:108FC0003D48009901706BE70120C0025EE73D4813
:108FD0000078012812D103AC20461946FFF739FD6D
:108FE000E073A020B02110232246FFF7ACFB2C49F0
:108FF00008800828E4D133480770E1E718785978E9
:10900000090208189978DA78120251180904081828
:109010002B490968214A12685118884203D2204816
:1090200040210180CCE725490978002901D00F2192
:10903000C94388422DD203AF384619461C46FFF774
:1090400008FDF8731B480178A02010233A46FFF76B
:109050007AFB134908800828B2D1164908881030D5
:1090600008802078617809020818A178E278120255
:109070005118090408181249086008490A6815219E
:109080005143FFF75DF800299AD101200D4908707E
:1090900096E70120C00291E7742B00205C2B002092
:1090A000722B0020582B0020782B00206F2B0020E3
:1090B000818D5B00622B0020642B00205B2B002045
:1090C000682B0020702B0020FF010000F0B585B058
:1090D0000646434C0027278004921018414A128804
:1090E000904241D201910397404F00200290386096
:1090F0003F4C404D2078052809D806F093F8386891
:10910000401C3860A842F5D33748042101800298FA
:1091100020703948018839480278102A01D0042A81
:1091200032D188190346C033049C651A0F240440C9
:109130001020001B854200DB0546DC09603C01264F
:109140003002E7B27F09052F12D3B443E6B29E3254
:10915000B242234C039F0DD301984218D9B2EBB20F
:109160003046FFF7F0FA05E01F482021018011E0AA
:109170001B4C039F1C49088008280BD1E8B21E4AEB
:1091800011880818108005E0012080021649088027
:10919000134C039F144800881F2809DD202813D092
:1091A00001210A0290420FD0890288420CD00CE0C3
:1091B000042809D0082808D10F480088049988425B
:1091C00001D3022700E001272780208802210143E4
:1091D000022902D1084900220A8005B0F0BDC0462C
:1091E000742B0020602B0020722B0020782B002095
:1091F0006F2B0020818D5B007C2B00205A2B0020E0
:10920000F0B585B0044600200190042C6FD20BF01D
:10921000F7FA002801D10BF073FB0020009000BF8B
:109220000098401C00900BF0EBFA03900398002884
:1092300003D0484900988842F2D30398002856D1B9
:10924000042145480BF0BEFA4448454908802101F5
:10925000444A515C4900404A505A41490A88012118
:10926000090300F055F902900120049020013D49C6
:1092700040184078002801D100264BE020013949F0
:1092800040184078012802D13548068842E0200184
:1092900034494018407802282AD120014018057925
:1092A0002901304A515C49002B4A505A2C490A88FE
:1092B0000121090300F02CF9064628012A49431828
:1092C0002801284940180289280140180021C76850
:1092D0003046B84706462801224BC018C2882801EC
:1092E000C0188178304600F087F8064612E02DE07D
:1092F00020011C4940184078032804D02001401860
:109300004078132804D1200116494018868801E0CE
:10931000002004900498002818D020011249431816
:109320002001104940180289200140183146C768C1
:109330000298B847019020010A4BC018C28820014A
:10934000C0188178019800F057F80190019805B095
:10935000F0BD000050C300000A0100208813000087
:1093600004010020F0F3010030F40100F8B50546D7
:109370000E4614460020009001211C4801751C482F
:10938000007888431A490870084680780821084305
:109390001749887000208871084600780121084329
:1093A0001349087008460572002717E01048007836
:1093B000802108430E49087000BF0E48007D002838
:1093C000FBD000200B4908750948C0892080A41CE7
:1093D0000748C1890098081800907F1CB742E5D360
:1093E00031460098FEF7ACFE80B2F8BD4061004007
:1093F000005004404060004010B50346012908D1E8
:10940000094CA41A9C4202D99C18A0B20BE0064851
:1094100009E0022906D1934202DD9C1AA0B202E0C3
:10942000002000E0184610BDFFFF000010B5044604
:109430000121202001F0D0FF0020324908700121D5
:1094400031480175002031490875152014F030FFAE
:109450002C488078E17808432A498870084680784B
:1094600021780843274988702078802806D108464B
:109470000079E17949000843224908712148807840
:10948000E17A08431F498870A078002803D1084674
:10949000007908710FE0A078012806D119480079F9
:1094A000602108431749087105E0164800798021BA
:1094B00008431449087113488079217908431149F8
:1094C000887108468079617908430E498871207A4D
:1094D000C872607A88720846007838218843094942
:1094E0000870084600786178C9000843054908708B
:1094F000A07A0873084600780121084301490870E2
:1095000010BD000000500440406100404060004039
:10951000F8B504460E461746002E01D100250FE08F
:10952000A64201DC3D460BE00094009C20467843B7
:10953000009031460098FEF703FE0090009885B237
:109540002846F8BD0146042904D28A00024BD218ED
:10955000508800E000207047AC2400200146042918
:1095600003D28A00024B985C00E0002070470000A4
:10957000AC240020FFB587B004460898844203DA83
:109580000A988068002802D12448019042E0089897
:10959000001B82B20292002625460A9880680021AC
:1095A0002F463A463346049605910690FEF722FE72
:1095B00005460E46002328463146029AFEF7EAFD8C
:1095C00005460E46304600210A46494050400143B8
:1095D00002D0124801901DE003950A98C068039DCF
:1095E000A84202D30020019014E00A98C1680398B1
:1095F000401A039009990398FEF7A2FD039003987F
:10960000000C0004002802D00448019002E00398F6
:1096100080B2019001980BB0F0BD0000FFFF000088
:1096200010B5084800788021884306490870012158
:1096300005480175002005490875152014F038FE0D
:1096400010BD0000005004404061004040600040F8
:10965000F8B505460E4614461F4621462846FEF735
:1096600085FD80B2F8BD0000FFB587B006460A98B8
:109670004068002801D1029035E00A9801684068EE
:1096800008180390002534460021274603980695C4
:109690000491059038462946049B059AFEF7AAFDD9
:1096A00004460D460A984068024600230190204671
:1096B0002946FEF76FFD04460D4600232046294645
:1096C000099AFEF767FD04460D46284607492140E2
:1096D000002359405840014303D00448C04302903E
:1096E00001E0A0B2029002980BB0F0BD0000FFFFB5
:1096F00010B5FE4800688079030014F0BFFD07052F
:109700009ED8F5F4F3F2F100F848006840790300C0
:1097100014F0B4FD0805138A2A8A468A638A10F079
:109720006BFF0020F1490968C873F0480068407970
:10973000401CEE49096848717DE0ED494969EB4AF2
:109740001268D27A885C10F0CFFFE8480068407950
:10975000401CE64909684871E44800684079401CAB
:10976000E2490968487166E009F068FB002810D1F9
:1097700010F0BAFFDD4800684079401CDB490968F9
:109780004871DA4800684079401CD8490968487136
:1097900005E010F05BFF0020D449096848714AE0F9
:1097A00009F04CFB002811D1112010F09DFFCF488B
:1097B00000684079401CCD4909684871CB48006871
:1097C0004079401CC9490968487105E010F03EFF26
:1097D0000020C649096848712DE009F02FFB0028D8
:1097E0001BD1C2480068C07A401CC0490968C872D1
:1097F000BE480068C07ABE49097888420DDB002067
:10980000BA490968C872B94909684862B748006826
:109810008079401CB5490968887110F017FF002055
:10982000B2490968487106E010F010FF0020AF4906
:109830000968487100BF00BF32E3AC480068407C53
:10984000002817D0AA48C068002803D0A848C168DB
:10985000192088470020A54909684862A348006884
:109860008079401CA1490968887100209F490968D6
:1098700048711BE09D480068406A282807D29B4831
:109880000068406A401C9949096848620EE000205F
:10989000964909684862954800688079401C934958
:1098A000096888710020914909684871F8E28F4879
:1098B00000684079030014F0E1FC080518A42FA407
:1098C0004CA480A410F098FE002088490968C87351
:1098D000864800684079401C84490968487197E0CF
:1098E000D4E2C7E230E25DE194E0814949697F4A10
:1098F0001268D27A885C10F0F7FE7C4800684079E4
:10990000401C7A4909684871784800684079401CD1
:109910007649096848717BE009F090FA002811D176
:10992000012010F0E1FE714800684079401C6F4949
:10993000096848716D4800684079401C6B490968A6
:10994000487105E010F082FE0020684909684871FE
:109950005EE009F073FA002828D164490968C97AE1
:1099600024225143634A12688918604A1268D27BE4
:10997000885C10F0B9FE5D480068C07B401C5B4904
:109980000968C87359480068C07B242814D3574815
:1099900000684079401C554909684871534800687F
:1099A0004079401C51490968487105E010F04EFEAD
:1099B00000204E49096848712AE009F03FFA002862
:1099C00018D14A480068C07A401C48490968C872E2
:1099D00046480068C07A4649097888420ADB002078
:1099E00042490968C872414800688079401C3F4973
:1099F0000968887110F02AFE00203C490968487106
:109A000006E010F023FE002038490968487100BFC5
:109A100000BF45E2354800684079030014F02EFC91
:109A20000A0614B92BB948B978B995B910F0E4FD14
:109A300000202E490968C8732C4800684079401CF2
:109A40002A4909684871ABE029494969274A1268DF
:109A5000D27A885C10F048FE244800684079401CA7
:109A6000224909684871214800684079401C1F4913
:109A70000968487194E009F0E1F9002811D14A2001
:109A800010F032FE194800684079401C17490968F7
:109A90004871164800684079401C144909684871AB
:109AA00005E010F0D3FD002010490968487177E007
:109AB00009F0C4F9002824D1FF2010F015FE0B484E
:109AC0000068C07B401C09490968C87307480068E2
:109AD000C07B24281BD3054800684079401C0349FB
:109AE0000968487101480068407905E0D007002006
:109AF000402B0020CC070020401CEA49096848712F
:109B000005E010F0A3FD0020E6490968487147E030
:109B100009F094F9002811D1FF2010F0E5FDE1488B
:109B200000684079401CDF4909684871DD480068D9
:109B30004079401CDB490968487105E010F086FD5A
:109B40000020D849096848712AE009F077F900280F
:109B500018D1D4480068C07A401CD2490968C8723C
:109B6000D0480068C07AD049097888420ADB0020D2
:109B7000CC490968C872CB4800688079401CC94943
:109B80000968887110F062FD0020C64909684871B3
:109B900006E010F05BFD0020C2490968487100BF73
:109BA00000BF7DE1BF4800684079030014F066FB08
:109BB0000C0715C32CC349C366C382C39FC310F0EF
:109BC0001BFD0020B7490968C873B6480068407992
:109BD000401CB44909684871B4E0B3494969B14AC5
:109BE0001268D27A885C10F07FFDAE480068407938
:109BF000401CAC4909684871AA4800684079401C7B
:109C0000A849096848719DE009F018F9002811D1A8
:109C1000772010F069FDA34800684079401CA149F5
:109C2000096848719F4800684079401C9D4909684F
:109C3000487105E010F00AFD00209A490968487152
:109C400080E009F0FBF8002811D10C2010F04CFD49
:109C5000944800684079401C9249096848719148CD
:109C600000684079401C8F490968487105E010F090
:109C7000EDFC00208B490968487163E009F0DEF8CB
:109C8000002810D110F030FD864800684079401C53
:109C9000844909684871834800684079401C8149BB
:109CA0000968487105E010F0D1FC00207D49096881
:109CB000487147E009F0C2F8002811D1132010F0D4
:109CC00013FD784800684079401C7649096848715E
:109CD000744800684079401C72490968487105E081
:109CE00010F0B4FC00206F49096848712AE009F0BF
:109CF000A5F8002818D16B480068C07A401C694953
:109D00000968C87267480068C07A6749097888425C
:109D10000ADB002063490968C872624800688079DC
:109D2000401C60490968887110F090FC00205D4972
:109D30000968487106E010F089FC0020594909685B
:109D4000487100BF00BFABE056480068407903008F
:109D500014F094FA080513872A874787638710F061
:109D60004BFC00204F490968C8734E480068407991
:109D7000401C4C49096848717AE04B494969494A95
:109D80001268D27A885C10F0AFFC464800684079CF
:109D9000401C444909684871424800684079401CA9
:109DA00040490968487163E009F048F8002811D17A
:109DB000492010F099FC3B4800684079401C394923
:109DC00009684871374800684079401C354909687E
:109DD000487105E010F03AFC0020324909684871EA
:109DE00046E009F02BF8002810D110F07DFC2D483A
:109DF00000684079401C2B4909684871294800686F
:109E00004079401C27490968487105E010F01EFCA4
:109E100000202449096848712AE009F00FF8002859
:109E200018D120480068C07A401C1E490968C872D1
:109E30001C480068C07A1C49097888420ADB002067
:109E400018490968C872174800688079401C15498C
:109E50000968887110F0FAFB0020124909684871FE
:109E600006E010F0F3FB00200E490968487100BFBE
:109E700000BF15E000200B4909688871094909688D
:109E80004871062007490968C87009E010F0DEFB38
:109E9000002004490968487102490968887100BFB7
:109EA00000BF10BDD0070020402B002010B56A482D
:109EB00000684079030014F0E1F9090610C627C6CE
:109EC00044C6608EC60010F097FB63480068407976
:109ED000401C614909684871BCE0604949695E4AB3
:109EE0001268D27A885C10F0FFFB5B48006840790A
:109EF000401C594909684871574800684079401C1E
:109F0000554909684871A5E008F098FF002811D16B
:109F10007F2010F0E9FB504800684079401C4E4912
:109F2000096848714C4800684079401C4A490968F2
:109F3000487105E010F08AFB002047490968487124
:109F400088E008F07BFF002810D110F0CDFB4248DC
:109F500000684079401C4049096848713E480068E3
:109F60004079401C3C490968487105E010F06EFBDF
:109F700000203949096848716CE008F05FFF00284B
:109F800022D135480068C07A401C33490968C8723C
:109F900031480068C07A3149097888420FDB0020D7
:109FA0002D490968C8722C4800684079401C2A492C
:109FB00009684871002028490968486208E00020C3
:109FC00025490968487103E0002023490968487160
:109FD00010F03CFB3EE020480068407C002816D092
:109FE0001E48C068002803D01C48C1681920884753
:109FF00000201949096848621749096848711649DB
:10A0000009688871052014490968C8701AE0124867
:10A010000068406A282807D20F480068406A401C40
:10A020000D49096848620DE000200B490968486243
:10A030000949096848710849096888710520064975
:10A040000968C87006E010F001FB002002490968A9
:10A05000487100BF00BF10BDD0070020402B00207A
:10A0600010B50024F7480068807A01287ED1F548B1
:10A070000068C07900287AD0F2480068807900280A
:10A0800004D0012874D0022873D191E1ED48006812
:10A09000007B24286ED2EB480068C07901287AD171
:10A0A000002475E0E7480068C07A24214843E64967
:10A0B00009684018E3490968097B415CE148006888
:10A0C000C07A24225043E14A12688018DD4A12689F
:10A0D000127B805C814229D0DA480068C07A242152
:10A0E0004843DA4909684018D6490968097B415C48
:10A0F000D4480068C07A24225043D34A126880189A
:10A10000D04A1268127B8154CE480068407B2428D4
:10A1100005D3CC480068007BCA4909684873C94820
:10A120000068007BC7490968887308E0C548006873
:10A13000407B242803D20120C24909688871C148A4
:10A140000068007B401CBF4909680873BD4800686F
:10A15000007B242808D3BB480068407B242803D216
:10A160000120B84909688871B64805E0D3E1CDE11E
:10A1700069E0BAE138E00EE00068007B242804D2F0
:10A18000B04800688079012800D103E0601CC4B2A7
:10A19000242C87D356E0002413E0AA480068C07A34
:10A1A00024214843A94909684018015DA548006871
:10A1B000C07A24225043A44A126880180155601CBA
:10A1C000C4B2242CE9D300209E4909684873232097
:10A1D0009C490968887301209A490968887124207C
:10A1E0009849096808732DE00020964909680873AA
:10A1F00094480068C07A401C92490968C872914826
:10A200000068C07A92490978884217DB8D48006857
:10A21000007C012804D102208A490968887106E07F
:10A22000002088490968887186490968C87100203A
:10A2300084490968C8728349096808740020814903
:10A240000968487161E17F4800684079030014F0B3
:10A2500015F8080513A62AA651A68EA6012079494D
:10A260000968087410F0C8F9764800684079401C05
:10A2700074490968487199E075494969714A1268D9
:10A28000D27A885C10F030FA6E4800684079401C41
:10A290006C49096848716B4800684079401C6949FD
:10A2A0000968487182E008F0C9FD00281BD16549A2
:10A2B0000968497B491CC8B210F016FA6148006869
:10A2C000407B60490968C8735E4800684079401C5B
:10A2D0005C49096848715B4800684079401C5949ED
:10A2E0000968487105E010F0B1F900205549096886
:10A2F00048715BE008F0A2FD00282BD151490968A4
:10A30000C97A24225143504A126889184D4A12686A
:10A31000D27B885C10F0E8F94A480068C07B401C9A
:10A3200048490968C87347480068C07B45490968BF
:10A33000897B88421ADD434800684079401C4149C6
:10A34000096848713F4800684079401C3D490968E8
:10A3500048710BE010F07AF93A480068407B3949BF
:10A360000968C87300203749096848711EE008F081
:10A3700065FD00280CD133490968887124203149D2
:10A380000968C8732F49096848732E49096888739A
:10A3900010F05CF900202B490968487106E010F0C4
:10A3A00055F9002027490968487100BF00BFACE09B
:10A3B000244800684079030013F060FF08050F8E01
:10A3C000268E4C8E688E10F017F91E480068407972
:10A3D000401C1C490968487185E01D494969194AB2
:10A3E0001268D27A885C10F07FF9164800684079CC
:10A3F000401C144909684871124800684079401CA3
:10A400001049096848716EE008F018FD002811D164
:10A41000492010F069F90B4800684079401C09494F
:10A4200009684871074800684079401C0549096877
:10A43000487105E010F00AF90020024909684871E6
:10A4400051E00000D0070020CC070020C807002002
:10A45000402B002008F0F2FC002810D110F044F945
:10A460009C4800684079401C9A490968487199489D
:10A4700000684079401C97490968487105E010F070
:10A48000E5F800209349096848712CE008F0D6FCF3
:10A4900000281AD18F480068C07A401C8D4909688D
:10A4A000C8728C480068C07A8B49097888420CDBF6
:10A4B000002088490968C8728649096888718549F9
:10A4C0000968487183490968C87110F0BFF8002015
:10A4D00080490968487106E010F0B8F800207D490D
:10A4E0000968487100BF00BF0FE010F0AFF800200E
:10A4F0007849096848717749096888717549096818
:10A50000087374490968C87200BFE2E0002071490D
:10A5100009688872DDE06F480068807A0228F4D10B
:10A520006C480068007A002879D06A480068407951
:10A53000030013F0A3FE0B0711BB25BB41545EBB08
:10A540007590BB0010F058F8624800684079401CD4
:10A55000604909684871B7E05F494969087810F0B7
:10A56000C3F85C4800684079401C5A490968487142
:10A57000584800684079401C564909684871A3E072
:10A5800008F05CFC002810D110F0AEF851480068CB
:10A590004079401C4F49096848714E48006840792D
:10A5A000401C4C490968487105E010F04FF8002044
:10A5B00048490968487187E008F040FC002807D145
:10A5C000444800684079401C42490968487103E0EA
:10A5D000002040490968487110F038F874E010F024
:10A5E0000BF83C4800684079401C3A4909684871BA
:10A5F0006AE0394949690978491CC8B210F074F811
:10A60000344800684079401C324909684871314833
:10A6100000684079401C2F490968487154E054E0B3
:10A6200008F00CFC00280FD10FF0B8FF2949096889
:10A630008870012010F02CF8264800684079401CF2
:10A6400024490968487105E010F000F8002021490C
:10A650000968487138E01F480068807811280CD1DB
:10A6600000201C4909680872AA201A4909688870E4
:10A67000002018490968487011E0164800684078C1
:10A68000401C144909684870124800684078032843
:10A6900005D308F073FC00200E49096848700FF0DC
:10A6A000D5FF00200B49096848710DE00FF0CEFF7F
:10A6B0000020084909684871064909684870AA20BD
:10A6C00004490968887000BF03E000200149096857
:10A6D000887210BDD0070020402B002010B5024624
:10A6E0009000074BC018405C002802D00320C043F4
:10A6F00010BD01209300024C1B1958540020F7E7AD
:10A70000E826002070B5002508E06D1C1B48854236
:10A7100002D20AF021F901E0002503E00AF070F806
:10A720000028F2D100BF022100200AF077F80321AF
:10A7300000200AF073F8052100200AF06FF80721C5
:10A7400000200AF06BF8002408E00020A1000C4A69
:10A750005054A10089184880601CC4B2042CF4D362
:10A7600001200849087000204870052088700020EA
:10A77000C87005480549088070BD000050C300003E
:10A78000AC240020060100208813000004010020F2
:10A79000F8B58D480078030013F070FD0604051627
:10A7A0003D5EFDFC0EE10AF0ABF800208649C87062
:10A7B000487008468078002802D10320087002E023
:10A7C000022081490870FDE07F488078002804D08D
:10A7D0007D488078401E7C4988700AF011F8002876
:10A7E0000BD10AF08DF800207749C87008468078B0
:10A7F00000280FD1032008700CE07348C078401C7B
:10A800007149C8700846C078052803D30520087030
:10A810000AF0A2F8D6E009F0F3FF00280ED10421D7
:10A820006A4809F0CFFF00206749C870487068483F
:10A83000684908800420644908700CE06248C078C8
:10A84000401C6149C8700846C078052803D305201C
:10A8500008700AF081F8B5E05B49497809015E4A61
:10A86000515C4900594A505A5A490A880121090342
:10A87000FEF74EFE009001255348407800015649EE
:10A8800040184078002801D100243CE04E48407830
:10A890000001514940184078012802D14D480488F0
:10A8A00031E04948407800014B494018407802287F
:10A8B00012D1454949780901474A89180879FEF7B4
:10A8C00041FE0446404949780901434A89180879FC
:10A8D000FEF744FE054616E03B48407800013E493D
:10A8E00040184078032806D03748407800014018C7
:10A8F0004078132806D13448407800013649401882
:10A90000848800E00025002D2FD02F4840780001DA
:10A91000324943182C48407800012F4940180289D9
:10A9200029484078000140182146C7680098B84778
:10A930000646254840780001274BC018C2882248A7
:10A9400040780001C01881783046FEF755FD064674
:10A950001D484078800022494018468001201A494D
:10A96000497889001E4A50540AE000201649497867
:10A9700089001B4A89184880134949788900505436
:10A9800011484078401C1049487008464078042817
:10A9900009D301E013E007E009F0B2FF00200A4903
:10A9A0004870032008700DE009F02AFF002803D149
:10A9B00001200549087001E009F0CEFF02E0FFF731
:10A9C000A1FE00BF00BFF8BD060100200A01002063
:10A9D0008813000004010020F0F3010030F40100AE
:10A9E000AC24002010B509F0D5FE002405E00020BD
:10A9F000A100074A5054601CC4B2042CF7D30020B5
:10AA0000044908700520887003480449088010BD77
:10AA1000AC2400200601002088130000040100205F
:10AA200070B50446002000F0AFF8002000F0DAF81E
:10AA3000002000F09BF8002000F0C4F8002000F097
:10AA400087F8002000F0AEF800BF012000F08EF87B
:10AA5000012000F0B7F8002521E0002000F086F882
:10AA6000002000F0AFF880202040002806D0012010
:10AA700000F08AF8012000F0B5F805E0002000F0B1
:10AA800083F8002000F0AEF800BF012000F06EF85F
:10AA9000012000F097F86006040E681CC5B2082D6E
:10AAA000DBDB012000F054F8012000F07BF870BDE2
:10AAB00070B504460D46012000F066F8012000F054
:10AAC00091F8002000F052F8002000F07BF8002000
:10AAD00000F03EF8002000F065F800BF012000F013
:10AAE00045F8012000F06EF8002628E0002000F074
:10AAF0003DF8002000F066F880202040002803D0B8
:10AB0000012000F041F802E0002000F03DF8802034
:10AB10002840002803D0012000F064F802E0002063
:10AB200000F060F800BF012000F020F8012000F0E4
:10AB300049F86006040E6806050E701CC6B2082EA1
:10AB4000D4DB012000F004F8012000F02BF870BDE8
:10AB500010B50446002C04D08121032009F08AFF9F
:10AB600003E08021032009F085FF10BD10B50446E5
:10AB7000002C04D08121042009F07CFF03E0802117
:10AB8000042009F077FF10BD10B50446002C04D056
:10AB90008121022009F06EFF03E08021022009F0EC
:10ABA00069FF10BD10B50446002C04D08121044873
:10ABB00009F060FF03E08021014809F05BFF10BD50
:10ABC0000107000010B50446002C05D081210720A4
:10ABD000000209F04FFF04E080210720000209F085
:10ABE00049FF10BD10B50446002C04D08121044853
:10ABF00009F040FF03E08021014809F03BFF10BD50
:10AC00000207000010B5F920FFF70AFF8820FFF7C0
:10AC100007FF9020FFF704FF9820FFF701FF0821AE
:10AC20000846FFF745FFE820FFF7FAFE1221084625
:10AC3000FFF73EFFA020FFF7F3FE70210846FFF765
:10AC400037FFA820FFF7ECFE70210846FFF730FF22
:10AC5000B020FFF7E5FE70210846FFF729FFB82076
:10AC6000FFF7DEFE00210846FFF722FFC020FFF7B6
:10AC7000D7FE00210846FFF71BFFC820FFF7D0FED4
:10AC800000210846FFF714FFD020FFF7C9FE2F214F
:10AC90000846FFF70DFFD820FFF7C2FE2F21084618
:10ACA000FFF706FFE020FFF7BBFE2F210846FFF766
:10ACB000FFFE4020FFF7B4FE00210846FFF7F8FE34
:10ACC0000A20FFF7ADFE002405E000210846FFF74B
:10ACD000EFFE601CC4B25A2CF7DB00240AE000200F
:10ACE0000B4908550B4908550B4908550B490855A0
:10ACF000601CC4B25A2CF2DB8120FFF791FE0020C9
:10AD0000074908708870C8700871487010BD00004D
:10AD1000EC21002046220020A0220020FA22002060
:10AD2000D000002010B58020FFF77AFE10BD000093
:10AD30000020044908700120034908700020487071
:10AD400070470000D5000020D000002010B5484812
:10AD5000007800287AD046488078030013F08EFAF5
:10AD60000604434A535A687E414800794149085CC9
:10AD70003F490979404A515C884209D13C480079F1
:10AD80003E49085C3A4909793D4A515C88421BD0EA
:10AD9000374800793749085C35490979364A5054B3
:10ADA000334800793549085C31490979344A5054AF
:10ADB0002F48C078002803D004202D49887011E066
:10ADC00001202B4988700DE000202949C8700846F1
:10ADD0000079401C0871084600795A2802DB0020DF
:10ADE0000871087041E04020FFF71AFE0220204958
:10ADF00088703AE01E4A11791079FFF759FE032056
:10AE00001B49887031E00A20FFF70AFE0420184928
:10AE100088702AE0164A1279194B995C144A127903
:10AE2000154B985CFFF744FE0520114988701CE023
:10AE30000F480079401C0E490871084600795A28CD
:10AE400005DB002008710870C87003E00EE00120E7
:10AE50000749C87000200649887006E000200449B0
:10AE600008708870C870087100BF00BF10BD000076
:10AE7000D0000020EC21002046220020A02200204B
:10AE8000FA22002010B50FF0F1FF012811D10E4871
:10AE90000078052806D1FF22A5320021012011F0FB
:10AEA000CFFC0FE04B22D2000021012011F0C8FCA2
:10AEB00008E00020054988804880002211460120D2
:10AEC00011F0BEFC10BD00001E0100201C0000207F
:10AED000002003490872487088704860704700007D
:10AEE000D00C002058221152704710B504460121A1
:10AEF000022000F071FA0021022000F06DFA10BD6E
:10AF0000014600205322525C10231A40002A08D028
:10AF10005322525C0C231A409210032A18D10320AA
:10AF200016E05422525A0123DB031A40002A0ED0A5
:10AF30005322525C0C231A409210032A05D053224C
:10AF4000525C9207920F032A01D1022000E00120F7
:10AF500070470246002058239B5A0B40002B01D01B
:10AF6000012000E000207047014600226020405A86
:10AF7000FF231B0218400005020F1001014BC018EF
:10AF8000704700000055044010B5002A0AD056232F
:10AF90001B5A0C0223435624235256231B5A8B431D
:10AFA000235209E056231B5A0C02A3435624235272
:10AFB00056231B5A0B43235210BD0000F8B504461C
:10AFC0000D46012700263448844203D10121022086
:10AFD00000F002FA2878401EA0702088FF2101317D
:10AFE000084320802088400840002080A878401E28
:10AFF000C1B25A20015568790007000CE9790902AD
:10B000000843A97908435C210853288981B240206C
:10B010000153A868C000C10C42200153A88981B225
:10B0200044200153E868C000C10C46200153288A1F
:10B0300081B2482001532869C000C10C4A20015345
:10B04000A88A81B24C2001536869C000C10C4E200F
:10B0500001535020005B297909020843502108530D
:10B060005020005B297988435021085300E0761C6A
:10B070005020005B4007400F2979884202D00748E2
:10B080008642F4D15020005B4007400F2979884266
:10B0900000D000273846F8BD00540440FFFF0000F0
:10B0A00030B5034600201C898C4209DD082A05D2F0
:10B0B00018244C431D682C19A05C02E0002000E01D
:10B0C000002030BD10B5024613898B4205DD1823E0
:10B0D0004B431468E318987C00E0002010BD014643
:10B0E000FF22C889C007C00F00280AD00120C881EC
:10B0F00000E0521EC889C007C00F002801D0002AF6
:10B10000F7D1C889C007C00F00280FD10220C8811D
:10B110000420C881487A400840004872487A3823A1
:10B120009843487200204872012070470020FCE7D5
:10B130000246507A012318435072507A0B78DB0094
:10B1400018435072087A012808D1888850814868CD
:10B15000000C0123DB031843908108E0087A0028E3
:10B1600005D15081486880001A4B18409081487A78
:10B17000012804D1507A40231843507206E0487ADF
:10B18000002803D1507A4023984350720878002851
:10B1900011D1C87A1072087B1070487B5070887B80
:10B1A0009070CB7BD370087C10714B7C5371887C82
:10B1B0009071CB7CD371887A002803D00120C00223
:10B1C000D08101E00820D081FF200130D081012012
:10B1D00070470000FC1F0000002904D0427A802341
:10B1E0001A43427203E0427A80239A4342727047C4
:10B1F00030B5024600200F4B5024A45A0D022C43B8
:10B200005025AC525024A45A8C43AC5200E05B1E33
:10B210005024A45A6407640F8C4201D0002BF6D14D
:10B220005024A45A6407640F002C01D0002000E0D1
:10B23000012030BDFFFF0000827A80231A40802A5F
:10B2400000D081727047000070B5044600250023CD
:10B25000002D02D00126602006530420C881888971
:10B260000126F6033040002808D00120107288899A
:10B27000C004C0084E893043506006E000201072C0
:10B2800088890F4E304080105060087AD0720023B9
:10B2900004E0CE5C10460C30C6545B1CD07A984259
:10B2A000F7DCC88904263040002804D1C889F6029A
:10B2B0003040002801D0002070BDD07AFCE70000AB
:10B2C000FC1F0000027C80231A40802A00D00174F9
:10B2D000704710B50246FF23D089C007C00F002871
:10B2E0000AD00120D08100E05B1ED089C007C00FCA
:10B2F000002801D0002BF7D1D089C007C00F00284B
:10B3000001D0002010BD507A012420435072507AA1
:10B310003824A0435072C87A1072487A00280FD19E
:10B32000087B1070487B5070887B9070CC7BD47009
:10B33000087C10714C7C5471887C9071CC7CD471E9
:10B34000FF200130D0814000D081107ADAE7000080
:10B35000F8B504460D460020002C00D100BF002A9D
:10B3600000D100BF012C01D141263043012A01D177
:10B3700012263043022C01D1C0263043022A01D1CB
:10B3800030263043134E307076788027BE43114FFD
:10B390007E70012C08D1FF2100BF0E4EB3781E46EF
:10B3A0000E4033468B42F8D10A4E76784027BE4392
:10B3B000084F7E70012A0BD10026009603E000BFE3
:10B3C000009E761C0096FF276937009EBE42F6D984
:10B3D000F8BD000000040240002905D0054A12789B
:10B3E0000243044B1A7004E0024A12788243014B74
:10B3F0001A70704720040240002905D0054A927E49
:10B400000243044B9A7604E0024A927E8243014B47
:10B410009A7670470008024001200649087000BF74
:10B4200004480078802108400028F9D00120024912
:10B4300008707047000C0240A401002070B503465C
:10B4400014460020002B01D1C0B202E00546803531
:10B45000E8B2012902D1051DE8B206E0022903D1B4
:10B4600005460835E8B200E0C0B2012C02D1851CC7
:10B47000E8B200E0C0B2084DA870AD7801263543AF
:10B48000054EB570002201E000BF521C7D252D0144
:10B49000AA42F9D970BD0000000C024070B500242A
:10B4A0002448007920210840002801D0224D3FE0A7
:10B4B00000F046F805462148007880210840002821
:10B4C00036D01E4880780840002801D01A4D02E08E
:10B4D00000F036F80546194880780007840F022CE2
:10B4E00001DBAD0804E0012C01D16D0800E000BFD4
:10B4F000124880788007C00F002801D02D0101E09C
:10B500000C2045430D4800784007840F002C02D1E1
:10B51000601CC4B207E0032C03D1601C4006040E7B
:10B5200001E06006040E21462846FCF709FE0546A8
:10B53000284670BD0004024000127A00000C024050
:10B5400000B5C0229178F82211401C4A12781143AC
:10B55000EA2923D00ADC0A46E03A130012F08EFEF4
:10B560000A181C20242A2A2A2A161A2AED291FD052
:10B5700004DCEB2916D0EC291CD117E0F02903D00C
:10B58000F82917D10E4817E00E4815E00E4813E0D1
:10B590000E4811E00E480FE00E480DE00E480BE09B
:10B5A0000E4809E00E4807E00E4805E00E4803E0AB
:10B5B0000E4801E00D4800BF00BF00BD201C024046
:10B5C0000090D003006CDC020048E80100366E01F8
:10B5D0000024F400001BB70000127A00808D5B008D
:10B5E00000093D00C0C62D0080841E0040420F00AF
:10B5F00010B50446204600F05FFD002010BD00009D
:10B6000010B590211348FCF74BFE12481249086010
:10B6100012484860062008810020887206220F49DF
:10B620000D4800F04BFA00210B48FFF705FE802182
:10B630000B48FCF735FE0A480A4948600A4B0422C9
:10B640000A49084800F0CBFB55210648FFF73AFEAF
:10B6500010BD0000480800202808002060F001000C
:10B66000D808002034080020F1B50000F0EF0100F8
:10B670000C4A127812060B4B5B781B041A43094BD9
:10B680009B781B021A43074BDB781A43104642088B
:10B690004240D20083085A401146034A5140034AAF
:10B6A000116070471B0700200102000020070020E6
:10B6B000F8B504460F46A07A4006400E002874D123
:10B6C0000025ACE01820684321680818407C012858
:10B6D0003CD101211820684322681018017400260B
:10B6E0000CE018206843216808180830815D182094
:10B6F0006843226810188155701CC6B2082EF0D31A
:10B70000002118206843226810180174182068432B
:10B71000226810184174182068432268101841618B
:10B72000182068432268101881742C2068436168CF
:10B730000818406A002809D018236B432268D018E3
:10B740002C236B436268D218516A884718206843DB
:10B75000216808184069FF21C94388425DD8182034
:10B760006843216808184069C11918206843226895
:10B7700010184161182068432168081841692C207D
:10B780006843626810188069814246D31820684374
:10B7900021680818807C55283FD05521182068431F
:10B7A000226810188174002624E03CE018206843C9
:10B7B00021680818805D2C21694362685118103196
:10B7C000895D08401821694322685118885518205E
:10B7D000684321680818805D2C216943626851180C
:10B7E0000831895D0843182169432268511888553A
:10B7F000701CC6B2082ED9D32C2068436168081883
:10B80000806A002809D018236B432268D0182C23A3
:10B810006B436268D218916A8847681C85B2208998
:10B82000A84200DD4EE7F8BD10B50446002013F035
:10B8300089F8022841D121480078002802D101204E
:10B840001E4908701D48007801281FD11B48407808
:10B85000401C1A49487021465A20FCF771FC1749D0
:10B860004978884229D800201449487008468078D1
:10B87000401C8870084680780A2803D3002088700E
:10B8800002200870002013F08DF816E00B480078B5
:10B89000022812D109484078401C084948702146C6
:10B8A0007D20C000FCF74CFC04494978884204D84C
:10B8B00000200249487013F075F810BD7800002090
:10B8C00000B587B0002168460171042141710C4820
:10B8D0000290411003910B49049105910A4806908A
:10B8E000FFF78EFE01A813F0C1F800F02FFB00F067
:10B8F0000FF80021054809F029F907B000BD000044
:10B90000FFFF1F00FFFFFF1F45BB000002050000F7
:10B9100010B5FF2002306549486000200872012000
:10B92000087000204872012088726148FFF7D7FB39
:10B930005E495F48FFF7FCFB01215D48FFF74CFCC7
:10B940005C485A49486000200872012008700020B5
:10B9500048720120887256481030FFF7C0FB5349E7
:10B9600053481030FFF7E4FB012151481030FFF736
:10B9700033FC5048401E4D494860002008720120A9
:10B980000870002048720120887249485030FFF743
:10B99000A6FB464946485030FFF7CAFB0121444800
:10B9A0005030FFF719FC4348C13840494860002037
:10B9B00008720120087000204872012088723C48FB
:10B9C0004030FFF78CFB394939484030FFF7B0FB76
:10B9D000012137484030FFF7FFFBFF201230334989
:10B9E0004860002008720120087000204872012081
:10B9F00088722F486030FFF772FB2C492C4860306A
:10BA0000FFF796FB01212A486030FFF7E5FBFF2096
:10BA1000213026494860002008720120087000206B
:10BA20004872012088722248A030FFF758FB1F4956
:10BA30001F48A030FFF77CFB01211D48A030FFF715
:10BA4000CBFB3F20400119494860002008720120CB
:10BA50000870002048720120887215482030FFF7D6
:10BA60003EFB124912482030FFF762FB01211048CB
:10BA70002030FFF7B1FB10480C49486000200872E5
:10BA80000120087000204872012088720848303078
:10BA9000FFF725FB054906483030FFF749FB012138
:10BAA00003483030FFF798FB10BD0000E42500206C
:10BAB0001055044002040000DF070000F0B50B46FB
:10BAC000144643600481002136E0002216E02C2554
:10BAD0004D4346687519AD5C18274F430668F61943
:10BAE000B5542C254D4346687519AD5C18274F4356
:10BAF0000668F6190836B554551CEAB2082AE6D38A
:10BB0000002518274F430668F619357418274F4348
:10BB10000668F619757418274F430668F619B57448
:10BB200018274F430668F619F57418274F4306681F
:10BB3000F61975614D1CA9B205898D42C5DC002539
:10BB40008572F0BD70B50446606800F01FFE0546C2
:10BB5000E27A23460C332946094800F0DFFD094903
:10BB60006068884203D0491C6068884206D1E17A47
:10BB7000A28890B222460C3202F06EFD70BD000029
:10BB800028080020DF070000F8B5054600262C46EF
:10BB9000002C07D000BF03E0FF20A055701CC6B2E8
:10BBA000082EF9D304F04EFCC000082108400746D7
:10BBB0002068884338432060F8BDF8B50546002664
:10BBC0002C46002C07D000BF03E0FF20A055701CBE
:10BBD000C6B2082EF9D304F0ABFC07122088000A85
:10BBE00000023843208004F0A3FC0002FF21090278
:10BBF00008400746208888433843208004F07EFDB3
:10BC000007126088000A00023843608004F076FD65
:10BC10000002FF2109020840074660888843384334
:10BC20006080F8BDFEB5054600260020019001F0B9
:10BC30001DFD0A210090FCF783FA074604F036FC4C
:10BC40000A210090FCF792FA80B201902C46002C59
:10BC500007D000BF03E0FF20A055701CC6B2082E1D
:10BC6000F9D30721090620688843019909120906BA
:10BC7000072212061140084320606068000A000293
:10BC80000199C9B208436060FF21090260688843D6
:10BC9000390C0902FF2212021140084360601102B0
:10BCA00060688843390A0904120211400843606041
:10BCB00060680002000A3906090E09060843606040
:10BCC00004F0B4FBC007C00FC0070090206840001C
:10BCD000400800990843206003F058FE0007000F59
:10BCE000009020680009000100990843206003F0DB
:10BCF00047FE022806D10121090720688843401821
:10BD0000206004E00121090720688843206004F0D6
:10BD100053FB0001F02108400090206888430099FF
:10BD20000843206004F01AFCFF2806DDFF21090407
:10BD300020688843401820600BE004F00FFC0004EA
:10BD4000FF210904084000902068884300990843B7
:10BD50002060FEBDFEB505460026002001900027AC
:10BD600004F0D0F964210090FCF700FA80B2019051
:10BD7000002001F08DFC87B22C46002C07D000BFBC
:10BD800003E0FF20A055701CC6B2082EF9D320682E
:10BD9000000A00020199C9B208432060FF2109048A
:10BDA0002068884339120904FF2212041140084315
:10BDB000206020680002000A3906090E09060843BF
:10BDC000206003F0E9FD28300002FF21090208404D
:10BDD000009020688843009908432060FEBDFFB5AD
:10BDE00081B004460F460025002600200090276001
:10BDF000039820810498E0600020207400BF9DE03B
:10BE00001C206843216808586A01616888501C201A
:10BE100068432168081880686A0161688918486069
:10BE20001C2068432168081840686A016168891805
:10BE300088601C20684321680818C0686A0161682E
:10BE40008918C8601C20684321680818007C6A01B2
:10BE50006168891808741C20684321680818407CB0
:10BE60006A016168891848741C20684321680818B1
:10BE7000807C6A016168891888831C206843216876
:10BE80000818C07C6A0161688918887400206A01FA
:10BE900061688918C8741C206843216808184068C4
:10BEA000002813D01C20684321680818C07C002893
:10BEB00005D1401E6A0161688918C8831AE0002014
:10BEC000C0436A0161688918C88313E01C20684375
:10BED00021680818C07C002805D000206A0161682C
:10BEE0008918C88306E000206A0161688918C88340
:10BEF00001200090002607E000216A016068801898
:10BF000014308155701CC6B2690160684018808B7E
:10BF1000B042F1DC1C206843216808184069002801
:10BF20000AD06B016268D218104614301C236B4390
:10BF30002268D21851698847681CC5B22089A84276
:10BF400000DD5DE7009805B0F0BD000000B58BB0E6
:10BF500056480790002108A801706846017608A895
:10BF60004170002052498872082108A8C170002041
:10BF700004E0002209A90A54411CC8B208A9C978E2
:10BF80008142F6DC4B48FFF7AAF806A94948FFF7BB
:10BF9000CFF84648401C0790002108A80170684669
:10BFA000017608A84170002041498872082108A83C
:10BFB000C170002004E0002209A90A54411CC8B243
:10BFC00008A9C9788142F6DC3A484030FFF787F883
:10BFD00006A938484030FFF7ABF84520000107902C
:10BFE000002108A801706846017608A84170002069
:10BFF0002F498872082108A8C170002004E000229F
:10C0000009A90A54411CC8B208A9C9788142F6DCC2
:10C0100028485030FFF763F806A926485030FFF74C
:10C0200087F8112040010790002108A80170684698
:10C03000017608A8417000201D498872082108A8CF
:10C04000C170002004E0002209A90A54411CC8B2B2
:10C0500008A9C9788142F6DC16482030FFF73FF87E
:10C0600006A914482030FFF763F8FD20C0000290B5
:10C070000021684601730171417381730821C17306
:10C08000002004E0002204A90A54411CC8B26946F9
:10C09000C97B8142F6DC07481030FFF720F801A980
:10C0A00004481030FFF744F80BB000BDEE06000066
:10C0B000E42500208055044030B585B004460025B5
:10C0C00020680190A1796846C172617941720021AE
:10C0D0000172017000BF05E020460830415D03A8F1
:10C0E00041556D1C6846C07AA842F5D81121490116
:10C0F0000198401A1BD023210901401A11D011497F
:10C100004018002802D0012817D104E069460E48E3
:10C11000FFF7DFF812E069460B484030FFF7D9F827
:10C120000CE0694608485030FFF7D3F806E069464E
:10C1300005482030FFF7CDF800E000BF00BF05B094
:10C1400030BD000062FDFFFF80550440F0B585B0B2
:10C1500004460F4600250026207C4006400E552848
:10C160007ED100BF76E1690160684018807C0028BC
:10C1700077D169016068401840686A016168891870
:10C180008968884209D26901606840184068C0190E
:10C190006A016168891848605AE16901606840185D
:10C1A000C068AF49884208D8690160684018C06813
:10C1B000401C6A0161688918C8606901606840189C
:10C1C000C07C002821D1002607E000216A016068B8
:10C1D000801814308155701CC6B26901606840181F
:10C1E000808BB042F1DC1C2068432168081840694C
:10C1F00000280AD06B016268D218104614301C2344
:10C200006B432268D21851698847690160684058B9
:10C210000090690160684018017C68460171002146
:10C220004171690160684018017F68468171690148
:10C2300060684018417C6846C171002608E06901C9
:10C24000606840181430815D02A88155701CC6B228
:10C25000690160684018808BB042F0DCE06801E062
:10C26000FCE01DE0002806D06846E16888476A01C6
:10C2700061688918C874690160684018C07C00282A
:10C2800004D16A01616889184860E1E06901606869
:10C2900040184068C01B6A01616889184860D7E08F
:10C2A00069016068401880680028EED06901606804
:10C2B0004018C08B0028E8D0690160684018C08B26
:10C2C0006A0161688918C968884207D16901606894
:10C2D0004018C08B6249C94388427DD169016068BA
:10C2E000401840686A01616889188968884209D2E3
:10C2F0006901606840184068C0196A01616889185E
:10C300004860A5E000206A016168891848606901F9
:10C3100060684018C0685249884208D8690160685E
:10C320004018C068401C6A0161688918C86000260E
:10C3300007E000216A016068801814308155701C84
:10C34000C6B2690160684018808BB042F1DC1C20E5
:10C35000684321680818406900280AD06B016268A8
:10C36000D218104614301C236B432268D21851692E
:10C37000884769016068405800906901606840180A
:10C38000017C6846017100214171690160684018B3
:10C39000017F68468171690160684018417C684688
:10C3A000C171002608E06901606840181430815DA1
:10C3B00002A88155701CC6B2690160684018808B64
:10C3C000B042F0DCE068002808D06846E1688847A1
:10C3D0006A016168891800E015E0C8746901606845
:10C3E0004018C07C002804D16A016168891848603F
:10C3F0002EE06901606840184068C01B6A016168EE
:10C400008918486024E01C206843216808184068A7
:10C4100000280FD00020C0436A0161688918C883D2
:10C420001C2068432168081840686A0161688918FF
:10C43000886008E000206A0161688918C8836A0181
:10C4400061688918886000206A0161688918C8607D
:10C45000681CC5B22089A84200DD84E605B0F0BDA5
:10C460000000FFFF7CB500BF19212C480078FBF7C6
:10C4700067FE04462A4860432A4A811800220120A8
:10C480000BF0F2FC20460A2250436430001981B2BE
:10C49000002201200DF0A8FA01200A22624312199D
:10C4A000D1B20A22624312190090D0B201231A4677
:10C4B00008F026FE64220721002006F057FB012029
:10C4C000009001900B20604382B20B20604381B248
:10C4D000002301200CF0C0FD6F20604381B20120D9
:10C4E0000DF028FD104860430246032101200AF0A8
:10C4F000BDFB002505E0012128460AF0F1FA681C81
:10C50000C5B20F2DF7DB21460B2251436431C8B26F
:10C510000DF074FF0DF05CFF7CBD00007300002087
:10C52000672B0000A0860100FCB101000020054936
:10C5300008700549087005490870054908700549E3
:10C540000870704774000020750000207300002000
:10C550007200002071000020F0B589B000BF00BF5C
:10C5600000BF00BF00BF00BF00BF00BF00BF00BFD3
:10C5700003215C480078FBF7F9FD5B4948430290D2
:10C5800003210120029A0AF071FB05215548007829
:10C59000FBF7D6FD0446E1B201200AF033F903218E
:10C5A00050480078FBF7E2FD0B214843643080B22D
:10C5B0000690E1B201231846069A09F07BF8494932
:10C5C00009788A0088180621FBF7D0FDFF21F53194
:10C5D000484380B207900798FBF7C8FDC7B23946B9
:10C5E000012009F04BFD03213E480078FBF7BEFD1A
:10C5F0000B214843643080B2089000220120089942
:10C600000DF0F2F9032137480078FBF7AFFD374909
:10C6100048433749401803900022012003990BF04A
:10C6200023FC03212F480078FBF7A0FD0B21484392
:10C6300080B2049003212B480078FBF797FD0B2173
:10C64000484386B20120F1B20090049AD0B201238F
:10C650001A4608F055FD64220721002006F086FAEC
:10C66000032120480078FBF781FD0B21484385B268
:10C670000120009000232A46294601900CF0ECFC92
:10C68000032118480078FBF771FD6F21484380B201
:10C690000590012005990DF04DFC164800783C28C6
:10C6A00005DA14480078401C1249087002E03C206A
:10C6B000104908700F4800781D2805DC09480078EB
:10C6C000401C084908700BE006480078002802D199
:10C6D0000449087004E003480078401E01490870CE
:10C6E00009B0F0BD74000020FCB10100672B000010
:10C6F000A086010075000020002000BF06E0002198
:10C70000044A1154044A1154411CC8B25A28F6DB99
:10C7100070470000EC210020A0220020FFB581B06E
:10C7200004460F463D462089A8422DDD1820684367
:10C7300021680818007C002826D1002609E004980A
:10C74000815D182068432268101808308155701CDC
:10C75000C6B2082EF3D301211820684322681018AE
:10C7600041742C20684361680818006A00280BD0C7
:10C7700018236B432268D218104608302C236B43D1
:10C780006268D218116A884705B0F0BD01460620DC
:10C79000104BCA1A99420FD008DCCA1FFA3A002A75
:10C7A00012D0102A0AD01F2A10D10BE0C02A07D0BD
:10C7B000C12A0BD100200BE0012009E0022007E094
:10C7C000032005E0042003E0052001E0062000BF6F
:10C7D00000BF70474103000010B504467D21C90029
:10C7E00061430846322103F02FFC10BD0148006868
:10C7F00070470000500000200148006870470000AA
:10C800004C00002010B505490988652251430846AF
:10C810006421FBF7ABFC80B210BD00005A00002081
:10C8200001480078704700005F0000200148007850
:10C83000704700005800002010B50EF017FB0128CB
:10C840002CD100F063F8012000F066F803F060FCE2
:10C85000044600F043F803F007FE044600F04AF8EF
:10C8600003F07EFF012805D100F03EF8012000F022
:10C8700047F805E0002000F037F8002000F040F80D
:10C8800000201349086013480068134988421ED2EB
:10C8900010480068801C0F49086018E000200D490E
:10C8A00008600B4800680C49884204D208480068B8
:10C8B000801C07490860002000F028F8012000F0E3
:10C8C0002BF8002000F00AF8002000F013F810BD4B
:10C8D000500000204C000020FFFFFF7F014908802E
:10C8E000704700005A00002001490870704700009E
:10C8F0005F00002001490880704700005C000020B4
:10C90000014908707047000060000020014908706C
:10C91000704700005800002001490870704700006F
:10C920005E0000200021014A117170470060004044
:10C93000002201494A757047006000400022014909
:10C940004A767047006000400021014A117270472A
:10C95000006000400021014A1173704700600040F0
:10C960000021014A11747047006000400021014A13
:10C9700011757047006000400021014A1176704730
:10C9800000600040002201494A7370470060004087
:10C99000002201494A7470470060004010B51C4CE9
:10C9A0001C49206888421ED106221B49201DFBF726
:10C9B00082FC002817D10D22184920460A30FBF7C7
:10C9C0007AFC00280FD10622154920461730FBF7C4
:10C9D00072FC002807D10622124920461D30FBF7C1
:10C9E0006AFC00280DD000F077FE0A480E49086066
:10C9F000074812F008F90C4A2421054812F02EF9D4
:10CA000004E0242221460848FBF731FC10BD000059
:10CA1000000250007AA7A55A3107002037070020EE
:10CA20002B07002025070020B82A002000200849F5
:10CA3000087008490870012007490870002007495C
:10CA400008700748074908600020074908707047C8
:10CA50001307002012070020150700201A070020E6
:10CA600025060000440700202407002010B50446D6
:10CA7000912044430A212046FBF762FB0446641DD3
:10CA8000204610BD70B5A8B0054600240026A021A0
:10CA90006846FBF705FC00F09FFC1E490A6814215C
:10CAA0006943505000211B48026814206843101845
:10CAB00041601848026814206843101881601548C6
:10CAC0004068002824D000BF17E06006060E282E1C
:10CAD00000D316E00F480168142060430858B100E5
:10CAE0006A4650500B48016814206043081841689A
:10CAF000701C80001150601CC4B20648007AA0422D
:10CB0000E3DC00BF6200034869464368022098479F
:10CB100028B070BD082B002030B5A9B00024002536
:10CB2000A02101A8FBF7BCFB00BF25E06006050EB5
:10CB300000F052FC1F490A68142161435050002143
:10CB40001C480268142060431018416019480268AC
:10CB50001420604310188160282D0BD215480168FD
:10CB6000142060430858A90001AA50500021681CF5
:10CB700080001150601CC4B20E48007AA042D5DC7F
:10CB80000C484068002813D00A48007A4000282842
:10CB900006D30848282201A943680220984707E0E5
:10CBA0000448007A4200034801A9436802209847DC
:10CBB00029B030BD082B002010B50EF057F9012820
:10CBC0007ED1FFF719FE5549884216D20F205449ED
:10CBD0004871887108468078002801D10520487086
:10CBE0004F488078052802D100204D494870002028
:10CBF0004B4908724872087035E0FA20484948717C
:10CC000088714849088803F059FB46488078002815
:10CC10000CD14349087008464079C87008468079AD
:10CC2000087100208870487048721CE001203C495F
:10CC300008700846407A022805D101204872002079
:10CC4000C87008710FE03648407A00280BD10220E6
:10CC50003349487208464078887008464079C87061
:10CC60000846807908712E4880782D494978884295
:10CC700013DD00202A49C87008460079401C08715D
:10CC8000084600798979884222DB0020244908710E
:10CC900008468078401E88701AE021488078204934
:10CCA0004978884214DA00201D4908710846C07886
:10CCB000401CC8700846C0784979884208DB00E00B
:10CCC0001EE000201649C87008468078401C887015
:10CCD00014488078002803D10120114908721BE014
:10CCE00010480088732803DB02200D49087213E006
:10CCF0000C48008870280FDC0020094908720BE0FE
:10CD000000200749087008464079C87008468079B5
:10CD1000087100200872487210BD0000B80B0000B6
:10CD2000580900207C0000200020044988704870C9
:10CD3000C8700871087248727047000058090020D6
:10CD40000020064908808870054988704870FA20DC
:10CD5000C870087100200872487270477C0000207B
:10CD60005809002070B503F003FA044603F012FAE4
:10CD700005460EF07BF801282ED105211A48FEF752
:10CD8000A1F9552804D1002018498870088027E0AF
:10CD9000012D04D1002015498870088020E0012071
:10CDA000124988701248844202DB201A84B200E0E3
:10CDB00000240A212046FBF7D9F9052901DB601D73
:10CDC00084B20C48844200DD04460A212046FBF769
:10CDD000CDF90649088003E00020044988700880E6
:10CDE000FFF7EAFE70BD0000280800207C0000204C
:10CDF000AA0A0000C60700001CB5002000900190A0
:10CE000000F0EAFA0B49086000200B490968086045
:10CE10000A48006800280CD00749096808680A21F8
:10CE2000FBF78EF90090012269460520034B1B6831
:10CE300098471CBDE0070020D4070020DC07002035
:10CE400000200849488008490880084908800849A6
:10CE500008700849887208490880488001200871D4
:10CE6000704700003400002024000020260000202D
:10CE7000280000200C0800202C000020F8B503F04A
:10CE800059F9074603F068F90090FFF7CFFC012835
:10CE900060D10521C548FEF715F9552802D0009844
:10CEA000012807D10020C2490870C2490880C24940
:10CEB000887256E0BE480078002810D10120BC4995
:10CEC00008703D462846E917890F091889030D0C9B
:10CED000BA48854200DD0546B648058041E0B648BF
:10CEE000807A4000B4490F520846867A0EE07000FE
:10CEF000B1490D5A701E4000085A7100AE4A505296
:10CF0000701E400011460D52701EC6B2002E08DD84
:10CF10007000A949095A701E4000A74A105A814260
:10CF2000E5DBA548807A401CA34988720846807AD0
:10CF3000052816DB002088720846C5882846E917B0
:10CF4000890F09188D109D48854200DD05469948D6
:10CF5000058006E0002096490870964908809649A9
:10CF600088729448058896480088A84257DA944801
:10CF70000088281A84B292480079012827D1904865
:10CF80004088A0420BDA8E4840880A308C4948809D
:10CF900008464088A04204DD0846448001E08848F5
:10CFA0004480874844882046E117890F09188C106F
:10CFB0000A2C00DA0A248248008800198049088077
:10CFC00008460088A84201DD08460580CDE07C487F
:10CFD0004088142805DD7A4840881438784948800C
:10CFE00002E0002076494880754844882046E117D1
:10CFF000890F09188C100A2C03DA01207049087176
:10D00000B3E06F480088A04205DD6D480088001B32
:10D010006B490880A9E0002069490880A5E06848BC
:10D020000088A84259DD66480088401B84B26448E5
:10D030000079012827D162484088142805DD60481E
:10D04000408814385E49488002E000205C494880EE
:10D050005B4844882046E117890F09188C100A2C78
:10D0600003DA0220564908717FE05548008800190C
:10D0700053490880084600885049884275DD0846B3
:10D080004F49088071E04E484088A0420BDA4C4876
:10D0900040880A304A49488008464088A04204DD5A
:10D0A0000846448001E0464844804548448820467C
:10D0B000E117890F09188C100A2C00DA0A2440485D
:10D0C00000882919884202DA3D4805804DE03C4835
:10D0D0000088001B3A49088047E0394844882046C8
:10D0E000E117890F09188C100A2C3EDD344840885E
:10D0F000142805DD3248408814383149488002E060
:10D1000000202F4948802E4844882046E117890F87
:10D1100009188C102A480079012813D10A2C03DA47
:10D1200002202749087120E0254800880019244979
:10D130000880084600882149884216DD08462049B3
:10D14000088012E00A2C03DA01201D4908710CE066
:10D150001B480088A04205DD19480088001B1849BB
:10D16000088002E0002016490880164800885028F0
:10D1700004DC134800881349088016E01048008832
:10D1800010490988884204DD0D4800880D4908804F
:10D190000BE00B4800880B490988081A84B2502C10
:10D1A00003DB0748008807490880F8BD28080020ED
:10D1B00028000020240000200C080020E02E0000A1
:10D1C0002C0000202600002010B5044664204443B3
:10D1D000A1212046FAF7B4FF0446204610BD000006
:10D1E0007CB5002400200190009000F03FFA054635
:10D1F0000A21FAF7A5FF044601226946042000F03F
:10D200006DFC0098401C002814D17D20C00020181F
:10D2100011490860084600680190012201A9032015
:10D2200000F09AFC0120009001226946042000F0E1
:10D2300093FC0FE0009801280CD17D2000012018FC
:10D2400005490860084600680190012201A90320F1
:10D2500000F082FC7CBD00002801002010B50120F8
:10D260000F49087000200F49096808600D490968D6
:10D2700048600C490968886000F07EF9FFF7BCFD42
:10D28000FFF74AFC08480068002807D0012205483B
:10D29000016808310020044B1B68984710BD00004E
:10D2A000AD070020A8070020A407002010B51848EB
:10D2B00000681849884229D117480068002804D01E
:10D2C000154800688047154908701548006800280F
:10D2D00004D013480068804712490870124800685B
:10D2E000002804D010480068804710490880104882
:10D2F0000068002805D00E48006880470D49088066
:10D3000002E00D480B49088000F078F810BD0000DD
:10D31000B80700207856341294070020AC0700208C
:10D3200098070020AE0700209C070020B0070020CF
:10D33000A0070020B20700201027000010B500232E
:10D34000174C2360174C2370174C2370174C237015
:10D35000174C2380174C2380174C2370174C1368ED
:10D360002360174C53682360164C93682360164C57
:10D37000D3682360154C1369236000280CD0144B2C
:10D380001860134C0B682468A3600023104C2468B9
:10D3900023600F4C246863600E4B014C236010BD6A
:10D3A000B8070020B4070020AC070020AE0700201B
:10D3B000B0070020B2070020AD070020940700202E
:10D3C000980700209C070020A0070020A407002049
:10D3D000A80700207856341205480068054988429D
:10D3E00003D105480068806870470020C043FBE710
:10D3F000B807002078563412A807002070B5002422
:10D40000002500263048007801285CD12F4800789C
:10D41000002858D12E480078012854D12D4805887D
:10D420002D490988694308462C49FAF789FE85B2D7
:10D43000E1200001854207D81921694308460921E6
:10D44000FAF77EFE044600E0244C25480068006898
:10D4500000192349096808602148006800682049CC
:10D4600009684968884207D31D48006800681C495C
:10D4700009684968461A0AE01948006840680021AE
:10D48000C943081A1649096809684018461C154816
:10D49000864218D3344601462046FAF751FE044628
:10D4A0000F48006841680F48604308180C49096834
:10D4B000486001200C49087009480068806800191C
:10D4C00007490968886070BDAC070020AD070020DF
:10D4D000AE070020B0070020B20700201027000090
:10D4E000A8070020A0860100B407002000220C4BF2
:10D4F0001A600C4B0A681A600B4B4A681A600B4B97
:10D500008A681A600A4BCA681A600A4B0A691A606C
:10D51000002801D0084A1060084A014B1A60704781
:10D52000B807002094070020980700209C070020DF
:10D53000A0070020A4070020A80700207856341276
:10D5400010B50A48006800280ED009480078012864
:10D550000AD10020064908700122064801680831F6
:10D560000020024B1B68984710BD0000A407002054
:10D57000B4070020A80700201CB5002000900190EF
:10D580000024FFF729FF04460E48006804600020CD
:10D590000C49096848600B49096888600A480068B6
:10D5A00000280DD007480068006800900548006812
:10D5B00040680190022269460120034B1B6898478E
:10D5C0001CBD0000BC070020C0070020F8B50546C0
:10D5D0000C4616460027002D17D00E480560FFF7B1
:10D5E000FBFE07462068B84203D90A480068076076
:10D5F00003E008492068096808600649606809680E
:10D6000048600449A0680968C8600348066000F0E3
:10D6100005F8F8BDBC070020C007002070B5002445
:10D620000025FFF7D9FE04460F4800680068A042B5
:10D6300000D903E00C4800680068251A0A48006811
:10D640004068401908490968886007480068806890
:10D6500005490968C968884205D903480068C06857
:10D6600001490968886070BDBC0700200148006856
:10D6700080687047BC070020002801D0024A106073
:10D68000024A116070470000BC070020C00700205C
:10D6900001461048026814204843101882680D485B
:10D6A0000368142048431818C06882420BD90948FF
:10D6B0000268142048431018C26806480368142002
:10D6C0004843181882600348026814204843101821
:10D6D00080687047082B0020002005E019490A5C8B
:10D6E00019490A54411CC8B20628F7DB002006E09D
:10D6F00016490A5C1449891D0A54411CC8B20D28F8
:10D70000F6DB002006E012490A5C0F4913310A5487
:10D71000411CC8B20628F6DB002006E00D490A5C71
:10D72000094919310A54411CC8B20628F6DB002009
:10D7300005E0002204491F310A54411CC8B20128E7
:10D74000F7DB704731070020BC2A00203707002094
:10D750002B0700202507002010B500200549086090
:10D76000486008724872887202F072FE0149C872FD
:10D7700010BD00006409002070B50024002502F0EF
:10D7800067FE6549C87202F049FD044602F050FD8B
:10D790000546FFF74BF8012874D101215F48FDF7DA
:10D7A00091FC552807D100205B4908724872086037
:10D7B00048608872AFE0FF2C01D0FF2D63D1FF2CB1
:10D7C0002AD1FF2D28D00020534908720120487229
:10D7D00053480860FF201430684348604868662159
:10D7E000FAF7AEFC4C494860084640684C4988420C
:10D7F00002D908464849486047484068AA2803D3E8
:10D8000045484068FA2803D901204349887282E0DC
:10D810000020414988727EE0FF2C2AD0FF2D28D1BC
:10D8200001203D490872002048723D484860FF20B1
:10D8300014306043086008686621FAF781FC3649B5
:10D840000860084600683649884202D908463249CD
:10D85000086031480068AA2803D32F480068E628EA
:10D8600003D901202C49887255E000202A4988728A
:10D8700051E02B48284908604860002088720872EF
:10D88000487248E040E00120234908724872FF20B6
:10D8900014306043086008686621FAF751FC1E499D
:10D8A0000860084600681E49884202D908461A499D
:10D8B0000860FF20143068431749486048686621B3
:10D8C000FAF73EFC1449486008464068144988420B
:10D8D00002D90846104948600F480068AA280BD3AF
:10D8E0000D480068E62807D80B484068AA2803D3EB
:10D8F00009484068FA2803D90120074988720AE0DC
:10D9000000200549887206E0002003490872487229
:10D9100008604860887270BD6409002028080020F3
:10D92000DE030000FFB583B006460D46174600240F
:10D930000020029000BF1420784380190190002E2F
:10D9400057D00198002854D02B4806602A490698E1
:10D9500048600846077200BF45E0FFF73DFD0290B2
:10D96000200129580298814204D820012858401CDF
:10D97000002806D1204902980A68142161435050BA
:10D9800006E0200129581C48026814206043115009
:10D99000200140194068401C002807D1002116488A
:10D9A0000268142060431018416008E0200140190B
:10D9B000416811480268142060431018416020013A
:10D9C000401981680C480268142060431018C16037
:10D9D00020014019017B0848026814206043101898
:10D9E0000161601CC4B20448007AA042B5DC00F0BA
:10D9F00005F807B0F0BD0000082B002070B500242A
:10DA000000250026FFF7E8FC054600BF4EE02A4847
:10DA10000168142060430858A84239D82648016894
:10DA20001420604308582E1A2348016814206043CC
:10DA300008184068811920480268142060431018B3
:10DA400081601D48016814206043081881681A48E5
:10DA50000268142060431018C068814224D9164817
:10DA600001681420604308180069002803D020468C
:10DA7000FFF708F818E01048016814206043081800
:10DA8000C1680D48026814206043101881600BE0E3
:10DA900009480168142060430818406806490A686C
:10DAA0001421614351188860601CC4B20248007A96
:10DAB000A042ACDC70BD0000082B002010B500BFF8
:10DAC00014244C432318002805D0002B03D0024C0B
:10DAD00020606260217210BD082B0020F8B5054659
:10DAE0000E4614462B0010F0C9FB0504121920271E
:10DAF0002E001748FBF732F8164908701448FAF759
:10DB0000E7FB07466421FAF71BFB30601CE0A0042A
:10DB1000020C31461020FBF71BF915E0A004020CA3
:10DB200031463020FBF714F90EE0A004020C314618
:10DB30005020FBF70DF907E0A004020C31467020DD
:10DB4000FBF706F900E000BF00BF0020F8BD0000B1
:10DB5000CE230020D900002070B505460E4614469D
:10DB60002B0010F08BFB05041C232A313800306891
:10DB7000002802D1FAF790FE10E064223168514388
:10DB800008461649FAF7AEFB002015490870012235
:10DB900064211248FBF74AF9114908701CE0A004FF
:10DBA000020C31461020FBF791FA15E0A004020C9C
:10DBB00031463020FBF78AFA0EE0A004020C314611
:10DBC0005020FBF783FA07E0A004020C31467020D6
:10DBD000FBF77CFA00E000BF00BF70BDC02300204F
:10DBE000D800002000B5AFB050211BA8FAF758FBB1
:10DBF00000201A90142115A8FAF752FB0020129069
:10DC0000139014901190402101A8FAF749FB0020CD
:10DC10003F49086001221BA9FFF760FF1B98401CC9
:10DC2000002801D11A9001E01B981A9039481590EC
:10DC300039481690394817900020189038481990A4
:10DC400015AA1AA93748FFF779FB02221CA901205F
:10DC5000FFF744FF1C98401C002801D1129001E0FE
:10DC60001C9812901C98401C002801D1139001E0D0
:10DC70001D9813902C48149012A92C48199AFFF75C
:10DC8000A5FC08221EA90220FFF728FF1E98401CB1
:10DC9000002801D1019001E01E9801901F98029088
:10DCA00023480390012069460874801E059021498D
:10DCB0000791012101A80177881E09901D490B9148
:10DCC000012109A80173881E0D901A490F910121A5
:10DCD0000DA80173042201A91748199BFFF722FE22
:10DCE00001221BA90320FFF7F9FE14491B980860C5
:10DCF0001B98401C002806D1FF20F5300860012247
:10DD00000320FFF729FF0E48014908602FB000BD2E
:10DD1000DC0000202DC8000021C8000005C800005C
:10DD200059DB00005423002076841E00602300206D
:10DD30000F2700009F86010070230020280100208B
:10DD4000A33AA55A00B585B014216846FAF7A8FA97
:10DD500000200F4908600F4800900F4801900F48BD
:10DD60000290002003900E48049069460D48FFF78A
:10DD7000BDFB0D480499FFF77FFC04210B48049A72
:10DD8000FFF79CFE0A480249086005B000BD00008C
:10DD9000DC0000202DC8000021C8000005C80000DC
:10DDA00059DB000054230020602300207023002052
:10DDB000A33AA55A00200B4908800B4908800B495B
:10DDC000088001200A49087000200A4908730A499E
:10DDD000088048800120087100200649488008809A
:10DDE000704700003C0000203E0000204000002062
:10DDF000420000201808002044000020FEB502F078
:10DE0000D3F9009002F0DAF90190FEF70FFD012836
:10DE10006BD10521D448FDF755F9552807D10020CD
:10DE2000D2490870D2490880D249888067E00198B9
:10DE3000012807D10020CD490870CD490880CD497F
:10DE400088805CE0C9480078002808D10120C749D3
:10DE50000870009D0A206843C54908804FE000987B
:10DE600081B2C448007B4200C248801D8152801F9D
:10DE7000067B11E07100BF48801D455A701E4100AD
:10DE8000BC48801D415A72008152701E4100B94841
:10DE9000801D4552701EC6B2002E0ADD7100B548C5
:10DEA000801D415A701E4200B248801D805A814236
:10DEB000E0DBB048007B401CAE4908730846007B9D
:10DEC000032807DB00200873084605890A206843F9
:10DED000A74908800020A74908804880A4480088F6
:10DEE00088800120A149087009E000209F4908703E
:10DEF0009F4908809F4908804880087388809C4813
:10DF000005889D480088A84256D29B480088281A58
:10DF100084B299480079012826D197484088A042C8
:10DF20000BDA95484088801C934948800846408811
:10DF3000A04204DD0846448001E08F4844808E48BA
:10DF4000448803212046FAF711F984B2022C00DA42
:10DF500002248948008800198749088008460088FB
:10DF6000A84200D90D80CDE083484088062805DD11
:10DF700081484088801F8049488002E000207E4917
:10DF800048807D48448803212046FAF7EFF884B2A0
:10DF9000022C03DA012078490871B3E07648008842
:10DFA000A04205DD74480088001B73490880A9E081
:10DFB000002071490880A5E06F480088A84259D91F
:10DFC0006D480088401B84B26B480079012827D136
:10DFD00069484088062805DD67484088801F6649F3
:10DFE000488002E000206449488063484488032157
:10DFF0002046FAF7BBF884B2022C03DA02205E490D
:10E0000008717FE05C48008800195B490880084679
:10E0100000885A49884275DD08465749088071E0F2
:10E0200055484088A0420BDA53484088801C52492A
:10E03000488008464088A04204DD0846448001E04C
:10E040004D4844804C48448803212046FAF78EF816
:10E0500084B2022C00DA0224474800882919884239
:10E0600002D245490D804DE043480088001B4249DB
:10E07000088047E04048448803212046FAF776F8B4
:10E0800084B2022C3EDD3C484088062805DD3A4833
:10E090004088801F3849488002E000203649488087
:10E0A0003548448803212046FAF760F884B23248A4
:10E0B0000079012813D1022C03DA02202E490871BD
:10E0C00020E02D48008800192B4908800846008868
:10E0D0002A49884216DD08462749088012E0022CAA
:10E0E00003DA0120244908710CE023480088A0428B
:10E0F00005DD21480088001B1F49088002E0002040
:10E100001D4908801C4800881D490988884203DA97
:10E11000194800880F2804DA174800881849088031
:10E120000AE01548008816490988081A0F2803DBF9
:10E130001148008812490880114807880B48007868
:10E1400000280DD06C20474364213846F9F7F8FFCA
:10E1500007460A48874200D907460A490F8002E06D
:10E16000002008490880FEBD280800204200002049
:10E170003C0000201808002044000020C6070000D2
:10E18000400000203E000020002007490880074989
:10E19000088007490880488001200871002005494F
:10E1A00048800880704700003E00002040000020AA
:10E1B000440000201808002000200249087002498D
:10E1C00008707047880000208900002010B5FEF715
:10E1D0002DFB012813D103210C48FCF773FF5528B0
:10E1E00005D100200A4908700A4908700CE002F0C5
:10E1F00029F80749087001200649087004E000204A
:10E20000034908700349087010BD00002808002069
:10E210008800002089000020F0B5A9B004460E4611
:10E220000025002700202890A0216846FAF738F83A
:10E23000FFF7D2F826490A68142161435050244858
:10E240000168142060430818C068B0420CD220480E
:10E250000168142060430818C1681D480268142032
:10E2600060431018416005E01948016814206043BC
:10E270000818466016484068002826D0002517E098
:10E280006806070E282F00D316E0114801681420F5
:10E2900068430858B9006A4650500D480168142078
:10E2A000684308184168781C80001150681CC5B28A
:10E2B0000748007AA842E3DC00BF6A0004486946C8
:10E2C00043680220984701202890289829B0F0BD83
:10E2D000082B002010B500F0EDFD00F0D7F80EF08F
:10E2E000DBFF00F00DFB00F001F810BD70B54148F8
:10E2F0000078912800D070BD00F0BEF8012876D1DA
:10E300003D4800883D49088008468078F0218843D0
:10E3100020303A4988700846807800090001354964
:10E32000097A0907090F0843344988703148807A0F
:10E33000401E3049887208460089401C0881084602
:10E340000089C988884216DA08202C49887200247E
:10E350000EE0284841882848001D415C2748C01C21
:10E36000015524484088401C22494880601CC4B2A2
:10E37000072CEEDB2DE01F4800891E49C988884222
:10E380001CD11C4800791B498978401AC5B2681C09
:10E390001A49887200240EE0164841881648001D6C
:10E3A000415C1648C01C015512484088401C114968
:10E3B0004880601CC4B2AC42EEDB0AE000F006FD0F
:10E3C00000200C4908700C490888092100F0B8F9B0
:10E3D00091E7012000F0BCFC084A917A1088921C59
:10E3E00000F070F905490888002100F0C1F800BF6D
:10E3F00081E700006C2800200828002098270020D2
:10E400001B49097E002932D01949897E0C225143CB
:10E41000174A515A174A118000200CE01449897E8E
:10E420000C225143124A8918891C0A5C1149891C23
:10E430000A54411CC8B20828F0DB0D49897E0C2221
:10E4400051430B4A8918897A0A4A91720121D17283
:10E450000749097E491E064A11761146897E491CE4
:10E4600091761146897E022901DB00219176704761
:10E47000642700208C2700200349487B012802D113
:10E480000021014A517370477C28002010B53348A1
:10E490004068002861D13148007B03000FF0EEFE98
:10E4A00007590512212E3D4A59002D4800780028B1
:10E4B00007D000202A4908702A490888012100F065
:10E4C0003FF947E026480078002809D00020244979
:10E4D000087025494A8808880123091D00F040F981
:10E4E00038E01F480078002807D000201C49087039
:10E4F0001C490888022100F023F92BE01848007815
:10E50000002809D000201649087017494A88088851
:10E510000923091D00F024F91CE0114800780028A7
:10E5200007D000200E4908700E490888092100F024
:10E5300007F90FE00A480078002809D000200849B0
:10E54000087009494A8808880323091D00F008F962
:10E5500000E000BF00BF00F039FC10BD7C280020A7
:10E560006C28002008280020A42700207047000005
:10E5700070B504460D4634480088A04263D1002D92
:10E5800061D13248007822284ED004DC20283DD0CA
:10E59000212856D141E0902802D0912851D115E090
:10E5A0002A48C08801280AD100202849087000F0B4
:10E5B0000DFC27490888002100F0C2F805E003207F
:10E5C00000F0C6FBA020214908703BE01F480089ED
:10E5D0001E49C98888420AD100201C49087000F0F1
:10E5E000F5FB1B490888002100F0AAF80DE0174848
:10E5F000807A002806D000F0E9FB1449087B00F07F
:10E6000089FB02E0032000F0A3FB1BE0062000F0E2
:10E610009FFB11200D49087014E0062000F098FBC4
:10E6200011200A4908700DE000200849087000F028
:10E63000CDFB08494A8808880923091D00F090F895
:10E6400000E000BF00BF70BD802700206C280020C4
:10E6500008280020A427002070B50346184C247E0B
:10E66000022C00DB70BD164C647E0C256C43144DEF
:10E670002B5300200AE0155C114C647E0C26744379
:10E680000F4EA419A41C2554441CE0B28842F2D3B6
:10E690000B4C647E0C267443094EA419A1723446B7
:10E6A000247E641C35462C762C46647E641C6C7675
:10E6B0002C46647E022C01DB00246C7600BFD1E77F
:10E6C00064270020F0B585B007460D4616461A4867
:10E6D0000780002406E031781748801C0155761C1D
:10E6E000601CC4B2AC42F6DB2C4605E0AA211248FD
:10E6F000801C0155601CC4B2082CF7DB0E48008852
:10E70000019008216846C1720021417201720170B6
:10E71000002406E00848801C015D03A80155601C28
:10E72000C4B2082CF6DB69460448FCF7D2FD012090
:10E730000149887205B0F0BD802700209055044043
:10E7400070B504460D46294620460EF0D1FC70BD3A
:10E7500070B504460D46294620460EF0D7FC70BD24
:10E76000F8B504460D4616461F463B463246294636
:10E7700020460EF0CCFCF8BDF8B507460E4615460F
:10E780005C480078002804D009213846FFF7D8FFFC
:10E79000F8BD002D01D0602D04DD09213846FFF7BA
:10E7A000CFFFF5E7544807804580002406E0317824
:10E7B0005148001D0155761C601CC4B2AC42F6DB0A
:10E7C00000204C49487008468580FF2088727F20D1
:10E7D00008730846808808282EDA0120C880084679
:10E7E0008088488001200881434800884349088088
:10E7F00008468078F0218843404988700846807830
:10E80000000900013B4909790907090F08433B4901
:10E81000887038480079401C8872002407E0364828
:10E82000001D015D3548C01C0155601CC4B2314853
:10E830008088A042F3DC4AE00721681CF9F796FCC7
:10E84000002907D0072128460830F9F78FFC29490D
:10E85000C88005E00721681CF9F788FC2549C880B5
:10E860000620244948800120088123480088234944
:10E87000088008468078F021884310301F4988704E
:10E8800008468078000900011A4989880905090F9E
:10E8900008431A49887008464088FF2109028843C6
:10E8A000144989880902FF221202114008431349C2
:10E8B000488008208872002407E00F48001D015D91
:10E8C0000E48001D0155601CC4B2062CF5DB01206A
:10E8D00000F03EFA094A917A1088921CFFF7F2FE86
:10E8E000902004490870054908880021FFF740FE80
:10E8F00000BF4DE76C280020082800209827002042
:10E9000010B5FFF77DFD1448C07A002822D01248C8
:10E9100080780009002806D0012807D002280AD0F4
:10E92000032810D10CE000F09DF90FE000F09EF8F4
:10E9300000F05AFA0AE000F011F800F055FA05E08C
:10E9400000F000F902E0FFF711FE00BF00BF002059
:10E950000149C87210BD00008C27002010B5404846
:10E960000078112800D010BD3E4800883F214901A1
:10E97000884200D0F7E73B4880780007000F38490D
:10E98000097A0907090F88420CD000203449087021
:10E9900000F01CFA34494A8808880423091DFFF74F
:10E9A000DFFEE0E72E480089401C2D49088108461B
:10E9B000807A401E887208460089C98888421BDA1E
:10E9C0002848807A082800D0CDE700240EE02548AA
:10E9D000C01C015D224842882348001D8154204804
:10E9E0004088401C1E494880601CC4B2072CEEDBE6
:10E9F000062000F0ADF930E01948808818494988B0
:10EA0000401A1849897A884203DA1648807A082819
:10EA100000D0A8E700240EE01248C01C015D104899
:10EA200042881148001D8154601CC4B20C484088C3
:10EA3000401C0B4948800A48408809498988884217
:10EA4000EADB00200649087000F0C0F906494A8850
:10EA500008880023091DFFF783FE00BF83E700003D
:10EA60006C2800208C270020A427002070B5324895
:10EA7000007880210840802800D170BD2F48008890
:10EA80003F214901884200D0F7E72C48807A0828C6
:10EA900000D0F2E72948807805072D0F2D0227487E
:10EAA0004088000A0543082D00DAE6E700202249E5
:10EAB000487006204880084685800120088108208B
:10EAC00088720020C8728988481C0721F9F74EFB1C
:10EAD000002909D018498988084608300721F9F724
:10EAE00045FB1549C88007E013498988481C072160
:10EAF000F9F73CFB1049C88010480088104908808D
:10EB000008464580002407E00C48001D015D0C48C4
:10EB1000001D0155601CC4B2062CF5DB042000F07A
:10EB200017F9102004490870054A51881088FFF72A
:10EB30000FFE00BFA1E700006C2800208C270020FA
:10EB4000A427002010B544480078A02808D04248E7
:10EB50000078912804D040480078A12800D010BD4A
:10EB60003E4800883F21490188420AD03C49088834
:10EB70000921FFF7E5FD00F029F90020364908706A
:10EB8000EDE73648807A08280AD0354908880921F7
:10EB9000FFF7D6FD00F01AF900202F490870DEE7D4
:10EBA0002E4880780007000F002804D0012825D0C7
:10EBB000022843D12EE028484078002800D048E0C1
:10EBC0002648C078002803D101202349487003E07B
:10EBD0002248C078204988721F480078912803D0C5
:10EBE0001E4800791C49087391201B49087000F0E9
:10EBF000EDF81949087B00F08DF82AE016484078B6
:10EC0000002800D025E0A12013490870032000F05F
:10EC10009FF81EE010484078002800D019E00E4808
:10EC20000078A02809D10E4908880821FFF788FD3F
:10EC300000F0CCF80020084908700AE0084908886C
:10EC40000521FFF77DFD00F0C1F8002002490870A2
:10EC500000BF00BF00BF82E76C2800208C27002087
:10EC60000828002010B52848007880210840802816
:10EC700000D110BD24480078002806D02348008821
:10EC80003F214901884200D0F3E72048807A1F499C
:10EC900089780907090F884203DD1C48807A082813
:10ECA00000D0E6E7194880780007000F002805D05B
:10ECB000164880780007000F072800DDD9E71348C1
:10ECC000008813490880114880780007000F4880A9
:10ECD000002407E00D48C01C015D0D48001D0155D2
:10ECE000601CC4B20A484088A042F3DC00200649F8
:10ECF000087000F06BF806494A8808880023091D4F
:10ED0000FFF72EFD00BFB4E76C2800208C27002001
:10ED1000A42700207F2805DC7D21C90041430A4A41
:10ED200091600DE0F12808DBF92806DC0107090FE6
:10ED300064225143044A916002E00449024A91600E
:10ED40000221014A517370477C28002018F001000D
:10ED500000B503000FF092FA0729050B11171D23C8
:10ED600029000121144A11731449516022E0022143
:10ED7000114A1173114951601CE003210E4A1173AD
:10ED80000F49516016E004210B4A11730D4951607F
:10ED900010E00521084A1173002151600AE00621A4
:10EDA000054A11730849516004E00021024A1173B9
:10EDB000516000BF00BF00BD7C280020A86100009A
:10EDC000F824010028230000F04902000020014936
:10EDD000087370477C280020024909880918014AF5
:10EDE000118070477C28002010B52F48007810282B
:10EDF00018D12E48408860280ADD2D488078000907
:10EE00000001801C2A49887022202749087025E0CB
:10EE10002748807800090001254988702020224970
:10EE200008701BE020480078112816D11E48807A0F
:10EE3000002800D010BD1C484078002800D0F9E719
:10EE40000820194988721A48807800090001184979
:10EE5000887020201449087000E0EBE7FD20C00016
:10EE60001349088008468078F021884330301049E3
:10EE700088700846C0780020C870084600791420C1
:10EE80000871032088720220FFF762FF084A917A16
:10EE90001088921CFFF716FC054908880021FFF72F
:10EEA00067FB00BFC6E700006C280020A4270020F5
:10EEB00098270020244A118852888A4242D0224A48
:10EEC00052888A4204DA204A52888A1A90B207E0AD
:10EED0001D4A52880023DB439A1A521C521890B2E2
:10EEE000194A5180127B002A10D0174A5268002A12
:10EEF0000CD0154A5268824205D9134A5268121A38
:10EF0000114B5A6002E000220F4B5A600E4A527BAE
:10EF1000022A17D10C4A9268002A0CD00A4A926839
:10EF2000824205D9084A9268121A074B9A6002E099
:10EF30000022054B9A60044A9268002A02D10122FD
:10EF4000014B5A73704700007C280020FEB5002753
:10EF50000020029001900090002500260024FDF77B
:10EF600065FC012879D10021A748FCF7ABF85528AA
:10EF700008D1A6480178A648F9F792F90020A349DC
:10EF8000087040E101F072F9074601F083F9029040
:10EF900001F076F9019001F087F9009001F05CF939
:10EFA0009C490870F020384000110A2805DBF02049
:10EFB00038400011C01C054303E0F0203840001128
:10EFC00005432D023807000F0A2804DB3807000F1D
:10EFD000C01C054302E03807000F05432D02F02155
:10EFE0000298084000110A2805DB02980840001129
:10EFF000C01C054304E0F0210298084000110543BD
:10F000002D0202980007000F0A2805DB029800076E
:10F01000000FC01C054303E002980007000F0543E2
:10F02000F0210198084000110A2805DB01980840EA
:10F030000011C01C064304E0F021019808400011B3
:10F040000643360201980007000F0A2806DB0198E4
:10F050000007000FC01C064304E0CCE00198000745
:10F06000000F06433602F0210098084000110A28DC
:10F0700005DB009808400011C01C064304E0F021A5
:10F080000098084000110643360200980007000F60
:10F090000A2805DB00980007000FC01C064303E0A8
:10F0A00000980007000F06435A480078002811D145
:10F0B00000240AE00020A100554A5050A100564A01
:10F0C0005050A100554A5050641C482CF2D30020E7
:10F0D00053490870524800784E490978884218DA36
:10F0E000002D16D04E4802784B49284600F0D8F83B
:10F0F00000280ED14A480078800047490D50484802
:10F100000078401C4649087008460178424800F0E3
:10F11000D8F8434800783F490978884218DA002E29
:10F1200016D03F4802783C49304600F0B9F8002834
:10F130000ED13B480078800037490E50384800789F
:10F14000401C3749087008460178334800F0B9F888
:10F15000334800782F49097888420EDD002407E003
:10F160000020A1002C4A5050A1002C4A5050641C91
:10F17000482CF5D300202A490870294800782549F1
:10F18000097888423FD100240FE0A00022490858A6
:10F19000A100224A50500020A1001F4A50501B4895
:10F1A00001781E4800F08DF8641C1D4800788442E8
:10F1B000EBD31848007815490870002018490870EA
:10F1C000002413E0A00012490858A100134A515826
:10F1D00088420AD0A00011460858A1000C4A50509D
:10F1E0000A480178104600F06CF8641C0748007863
:10F1F0008442E7D307E0054801780548F9F750F85D
:10F20000002002490870FEBD28080020820000206E
:10F21000B00B002080000020900A00207009002020
:10F220008100002010B505F06BFD10BD00BF7047D8
:10F2300010B504468020204301460320400205F01B
:10F2400019FC10BD10B510210320400205F012FC7E
:10F2500010BD000010B50224024805F05BFC044616
:10F26000204610BD0106000010B50021014805F040
:10F2700001FC10BD0106000010B5044680202043AB
:10F280000146024805F0F6FB10BD00000106000033
:10F2900010B51021014805F0EDFB10BD010600007E
:10F2A00030B503460C460021002000BF06E08D006B
:10F2B00065599D4200D101204D1CE9B29142F6DB17
:10F2C00030BDF8B505460E4600240EE0601CC7B2FE
:10F2D00007E0BA005119A200501900F00AF8781C92
:10F2E000C7B2B742F5DB601CC4B2701EA042EDDCB1
:10F2F000F8BD10B503680C68A34203D90A68036817
:10F300000B60026010BD70B505460024FFF71EFEBD
:10F3100070BD00002E480078401C2D4908702D4813
:10F320000078401C2B4908702B480078401C2A4963
:10F3300008702A480068401C284908600846006890
:10F34000FF219131884202D90020244908602048D9
:10F350000078C82802D900201D4908701D4800788F
:10F36000842802D900201B4908701B4800785028C7
:10F3700002D9002018490870194818490968405CEA
:10F3800018490870184812490978405C17490870F4
:10F39000174810490978405C1649087016480E490C
:10F3A0000978405C15490870154809490978405C9E
:10F3B00014490870144806490978405C13490870DC
:10F3C000134803490978405C1249087070470000EF
:10F3D000530700205407002055070020580700203D
:10F3E00083F701004C07002013F901004D070020AE
:10F3F000DBF901004E07002027FB01005007002029
:10F400005FFA01004F07002077FB01005107002041
:10F410003FFC01005207002010B50446204600F0D2
:10F4200049FA204600F002F810BD000010B504466D
:10F43000B148007800287DD1B0480088B0498842A2
:10F4400078DAB048007800284FD0AF48007800281C
:10F4500003D0AA480088AD490880AD48007800284C
:10F4600018D1A6480188A94800881930814206D3DE
:10F470000120A7490870A1480088A44908809F4836
:10F480000088A249098888421CDA9C4800889F4964
:10F49000088017E09D48018898480088193081420B
:10F4A00006D300209A49087094480088974908803C
:10F4B0009248008895490988884203DD8F48008872
:10F4C0009249088092480078002857D191480078E6
:10F4D000042803D08C480078002807D0874800888B
:10F4E000822803DA05208B490870A1E0894800785A
:10F4F000032803D084480078002809D07F4800887A
:10F50000FF211931884203DA0420824908708FE014
:10F5100080480078022803D07B48007800280AD071
:10F5200076480088FF21AF31884204DA0320794908
:10F5300008707DE0DFE077480078012803D072484A
:10F540000078002808D06D4800887349884203DAA3
:10F550000220704908706BE06E480078002803D0E4
:10F5600069480078002863D0644800883721090181
:10F5700088425DDA01206749087059E064480078E4
:10F58000012855D163480078012803D05E480078EF
:10F59000002809D05948008837210901884203DB37
:10F5A00000205C49087043E05A480078022803D0E4
:10F5B00055480078002808D05048008856498842AD
:10F5C00003DB01205349087032E0524800780328D9
:10F5D00003D04D480078002809D048480088FF2112
:10F5E000AF31884203DB02204A49087020E04948D5
:10F5F0000078042803D044480078002809D03F4808
:10F600000088FF211931884203DB0320414908703B
:10F610000EE040480078052803D03B4800780028D9
:10F6200006D036480088822802DB04203949087059
:10F63000FDF7E2F8394988425DD33948006800197E
:10F640003749086030480078002808D000202E494B
:10F650000870334908602F4800783249087000F07C
:10F6600057FD00281FD12E4800682F49884239D302
:10F6700000202B4908602B480078264909788842E9
:10F6800005DA28480078401C264908702AE02548F9
:10F69000007820490978884224DD22480078401EFD
:10F6A000204908701EE01E4800682049884219D38E
:10F6B00000201B4908601B480078164909788842D9
:10F6C00005DA18480078401C164908700AE0154809
:10F6D000007810490978884204DD12480078401EFD
:10F6E000104908700F4800780A490978884202D109
:10F6F00000200B49086010BD0B0000200200002014
:10F700001027000012000020080000200400002044
:10F710000A0000200600002076020000B80B00005E
:10F720001800002007000020C05D0000407E05009A
:10F7300000200B4908700B49087001200A49087025
:10F740000A49087000200A4908700A4908700A49E5
:10F7500008800A4908800A4908800A4908707047E9
:10F7600006000020070000200800002009000020FB
:10F770000A0000200B0000200C0000200E000020DA
:10F78000100000201200002000200B4908700B49D7
:10F79000087001200A4908700A49087000200A49C7
:10F7A00008700A4908700A4908800A4908800A490D
:10F7B00008800A49087070470600002007000020F2
:10F7C00008000020090000200A0000200B00002093
:10F7D0000C0000200E00002010000020120000206D
:10F7E000F1B500272D480078002804D00320F9F750
:10F7F000A9FE2B4908802B480088192847D30020F0
:10F800002849088028480078142829D20320F9F7CD
:10F8100099FE0746002407E060002449085AB842D0
:10F8200000DD05E0601CC4B21F4800788442F3DBB1
:10F8300000BF1D48057808E0681E40001B49085AB3
:10F8400069001A4A5052681EC5B2A542F4DC600035
:10F8500016490F5214480078401C1349087016E0EE
:10F860000026052405E060001049085A8619601C2E
:10F87000C4B20F2CF7D30A213046F8F761FC0849CF
:10F8800008800020084908700120094908700548CF
:10F8900001880098081803490880F8BD0900002075
:10F8A000020000201600002000000020E4070020D5
:10F8B0001200002023490988234A91422BDB0021B2
:10F8C000224A1180224A118022490988AF2212015E
:10F8D000914207DC20490978002916D01D49098882
:10F8E000914212DD02211D4A117000211C4A117043
:10F8F00005211C4A11700021174A117001211A4A72
:10F9000011700021194A11701AE01249098809186A
:10F91000104A118014E000210C4A11800D4A118018
:10F920000B490988124A914205DD00210B4A1170EA
:10F93000094A117004E0064909880918044A11802F
:10F940007047000002000020102700000E00002079
:10F950000C00002010000020090000200B000020F7
:10F960000600002007000020080000200A000020F8
:10F97000B80B0000014800787047000058090020CB
:10F980000148007A7047000058090020014880783B
:10F9900070470000580900200148008870470000A7
:10F9A0007C000020F8B500230025009500240022EB
:10F9B00000BF94E001259D40ACB20D882540009524
:10F9C000009DA5426FD11A468D79012D0DD1464D6E
:10F9D00003263602AD192D5C012696403543424E72
:10F9E00003273F02F61935540CE03F4D032636023B
:10F9F000AD192D5C01269640B5433B4E03273F02CF
:10FA0000F6193554CD78002D4ED1374D60352D5C2B
:10FA1000CE78002E01D1012600E000269640B543A5
:10FA2000314E603635548D78002D2ED12E4D19264D
:10FA30007601AD192D5C8E78002E01D1012600E0F3
:10FA400000269640B543284E19277F01F6193554F4
:10FA50000D79002D0ED1244D50352D5C0E79002EE0
:10FA600001D1012600E000269640B5431E4E5036D7
:10FA7000355423E01C4D50352D5C0E7996403543AE
:10FA8000EEB2194D50352E5418E0174D1926760157
:10FA9000AD192D5C8E7896403543134E19277F01A2
:10FAA000F61935540AE018E00F4D60352D5CCE781C
:10FAB00096403543EEB20C4D60352E544D79012DF4
:10FAC0000AD1094D30352D5C012696403543EEB202
:10FAD000054D30352E5400E000BF5D1CABB2082B45
:10FAE00000DA67E7F8BD000000000440FFB50746F4
:10FAF00015461E4600243846019900F01FF80028DC
:10FB000002D0012004B0F0BD00240CE00A206043C4
:10FB10000949085CB04204D12946204600F05EF84D
:10FB200007E0601C84B20A2060430349085C002897
:10FB3000ECD100BF0020E5E7B00100200246002A1A
:10FB400003D1402901DD01207047032A03D1022996
:10FB500001DD0120F8E7042A03D1202901DD01207D
:10FB6000F2E7052A03D1202901DD0120ECE70C2A68
:10FB700003D1102901DD0120E6E70D2A05D1012975
:10FB800003DD402901DA0120DEE70E2A03D1202916
:10FB900001D10120D8E70020D6E7000010B5064AC1
:10FBA00003231B02D218125C8A43034B0324240252
:10FBB0001B191A5410BD00000000044010B5064A7D
:10FBC00003231B02D218125C0A43034B03242402B2
:10FBD0001B191A5410BD00000000044070B5024605
:10FBE0000020B1E00A2353435A4C1B195B1C44000C
:10FBF00004191B199B788B427DD10A235343554C22
:10FC00001B195B1C440004191B195B78082B33D1AA
:10FC10000A2353434F4C1B195B1C440004191B5708
:10FC20004D4C4E4D6419E35C012423430A24544394
:10FC3000484D6419641C450045196457464D474EAC
:10FC4000AD192B550A235343424C1B195B1C44002E
:10FC500004191B57404C35466419E35C02242343C6
:10FC60000A2454433B4D6419641C450045196457EC
:10FC7000394DAD192B5564E00A235343354C1B19FC
:10FC80005B1C440004191B195B78092B34D10A232F
:10FC90005343304C1B195B1C440004191B572E4C5A
:10FCA0002E4D6419E35C402423430A245443294D18
:10FCB0006419641C450045196457274D274EAD193A
:10FCC0002B550A235343234C1B195B1C4400041976
:10FCD0001B57214C35466419E35C8024A3430A2456
:10FCE00054431C4D6419641C4500451964571A4D52
:10FCF000AD192B5525E025E00A235343154C1B195C
:10FD00005B1C440004191B57134C144D6419E35C2D
:10FD10000A2454430F4D6419641C450045196419A5
:10FD200065780124AC402343DCB20A235343094DD8
:10FD30005B195B1C450045195B57074D074EAD1914
:10FD4000EC5404E0431CD8B2032800DA4AE700BFB1
:10FD500070BD0000B00100200000044075080000E4
:10FD6000F8B50024FCF762FD012861D100F030FBFA
:10FD7000044664220721002002F0F8FE012C21D164
:10FD800000F0A4FB00280ED000F056FB054600F062
:10FD900047FB0646012003460246294600903046AE
:10FDA00005F0AEF950E000F047FB054600F038FBE7
:10FDB000064601200023024629460090304605F001
:10FDC0009FF941E0022C21D100F080FB00280ED0E9
:10FDD00000F032FB054600F023FB064601200346F7
:10FDE000024629460090304605F08AF92CE000F0E2
:10FDF00023FB054600F014FB0646002001231A46AB
:10FE000029460090304605F07BF91DE000F05EFBCE
:10FE1000054600F011FB064600F002FB07460120F4
:10FE200003462A4631460090384605F069F90BE052
:10FE30000020034602460146009005F061F90022C9
:10FE40000721104602F092FEF8BD0000F0B585B023
:10FE5000002473480078012824D1FCF7E7FC01282E
:10FE600012D1FCF7FFFA00BF0BE0182C02D1601C86
:10FE7000C4B204E064222146002002F077FE601C38
:10FE8000C4B2242CF1DBC8E0FCF736FC002406E009
:10FE900000222146104602F069FE601CC4B2242CE8
:10FEA000F6DBBAE0FCF7C2FC01287DD1FCF7A4FC2C
:10FEB0005C4988427FD35C480088032805DA5A48A9
:10FEC0000088401C5849088011E0002056490880ED
:10FED00000F0ACFA064600F0C7FA07460A21F8F728
:10FEE0002FF9054632462946012009F07DFD00F034
:10FEF0001BFC064600F0C2FB0A210390F8F720F92C
:10FF0000054600F093FA07463246294607F0ACFF53
:10FF1000FFF726FF00F050FA05462946012006F0BB
:10FF200071FC00F09BFA0646FF21F531F8F71EF947
:10FF3000C5B22946012006F0A1F8FFF71BFD0546D2
:10FF4000FFF72AFD0646FFF721FD07462B463246FE
:10FF50003946012005F0AEFB00F0E0F805462946E1
:10FF6000012009F0E7FF00F0A3FB054600F0BAFA14
:10FF7000064600F06DFA074600F0A0FB039000F083
:10FF8000B7FA3B4600960195029001460120039A7C
:10FF900009F062F800F066FB054600F05DFB0646DE
:10FFA00000F066FB074601E008E004E02A4631461F
:10FFB00006F05CFE31E0FCF7CFFA2EE0FCF79CFB8C
:10FFC00000222321104602F0D1FD002222211046FA
:10FFD00002F0CCFD00220721104602F0C7FD0022EE
:10FFE0000821104602F0C2FD00220921104602F04D
:10FFF000BDFD00220A21104602F0B8FD00221321A7
:020000040001F9
:10000000104602F0B3FD00221121104602F0AEFDB1
:1000100000221221104602F0A9FD05B0F0BD00003B
:1000200001010020B80B00007600002001490860A3
:10003000704700008007002002480068401C01490A
:10004000086070477C070020F3B581B006460020A9
:100050000E49086000F01EF8044600F01BF8054643
:100060002F1B3046029903F025FD00900AE000F0B6
:1000700011F805462F1B06480068002802D00448E6
:100080000068804700988742F1D3FEBD7C070020BE
:100090008007002001480068704700007C070020AE
:1000A0000B490978012901D101200FE0084909789D
:1000B000022901D1022009E005490978032901D16B
:1000C000042003E00121024A117001207047000062
:1000D0001507002010B5094B1B8899B20A12C8B247
:1000E000D3433133064C2370C34323336370134629
:1000F0005633A37003467133E37010BD44070020EC
:100100001B070020014800887047000024000020E1
:1001100001480088704700003C000020014800783A
:1001200070470000880000200148007870470000F8
:100130008900002010B5002205210648FAF7B0FF1B
:100140000402012205210348FAF7AAFF201880B211
:1001500010BD00002808002010B506220521034824
:10016000FAF79EFFC006C00F10BD0000280800204F
:1001700010B5042205210648FAF792FF0402052271
:1001800011460348FAF78CFF201880B210BD00001A
:100190002808002010B5062205210248FAF780FF42
:1001A000C01110BD2808002010B502220521024808
:1001B000FAF776FF10BD00002808002010B50622CF
:1001C00005210348FAF76CFF8006C00F10BD000040
:1001D0002808002010B5042202210348FAF760FF26
:1001E000C007C00F10BD00002808002010B5052270
:1001F00002210348FAF754FFC007C00F10BD0000EA
:100200002808002010B5002204210348FAF748FF0F
:100210004006400F10BD00002808002010B5002245
:1002200001210248FAF73CFF10BD00002808002019
:1002300010B5012211460248FAF732FF10BD000046
:100240002808002010B5022203210248FAF728FFEF
:1002500010BD00002808002010B50322002102482C
:10026000FAF71EFF10BD00002808002010B500227C
:1002700011460248FAF714FF10BD000028080020BC
:1002800010B5042200210248FAF70AFF10BD000051
:100290002808002010B5012200210248FAF700FFCB
:1002A00010BD00002808002010B5052200210248DA
:1002B000FAF7F6FE10BD000028080020322815DAF3
:1002C0003C498978012903DD01213A4A517070E0E7
:1002D00038498978002905DD2F286ADC0021354A54
:1002E000517066E00021334A517062E03E2817DA0F
:1002F000322815DB2F498978022903DD02212D4A96
:10030000517056E02B498978012905DD3B2850DCE6
:100310000121284A51704CE00121264A517048E0E1
:10032000502817DA3E2815DB22498978032903DD96
:100330000321204A51703CE01E498978022905DDDD
:100340004D2836DC02211B4A517032E00221194A45
:1003500051702EE0622817DA502815DB154989788C
:10036000042903DD0421134A517022E011498978E0
:10037000032905DD5F281CDC03210E4A517018E0BB
:1003800003210C4A517014E073280FDA62280DDB48
:1003900008498978042905DD70280ADC0421054A0A
:1003A000517006E00421034A517002E00521014A20
:1003B00051707047580900200148007870470000CC
:1003C000070000200148007870470000F00000207E
:1003D0000148007870470000EF000020F8B50026C3
:1003E00000240025FDF742F907460A21F7F7A8FE89
:1003F000054609480068854200D303E006480068C6
:10040000461B34467D200001844200D30446034845
:1004100004600068F8BD00002801002024010020CD
:100420000148007870470000F90000200148007979
:1004300070470000E8000020014840787047000045
:10044000F90000200148807970470000E800002092
:100450000148407970470000E8000020014800880A
:10046000704700002600002010B50024FFF7DEFFD3
:1004700000280AD10A4800880A49884202DB084657
:10048000074908800648048808E005480088FCF70A
:100490009BFE84B20448844200DB0446204610BD23
:1004A0003E000020C6070000CE04000000200549E1
:1004B0000988054A914202DB1146024A118001492E
:1004C000088870473E000020C607000001480078F9
:1004D000704700004D070020014800787047000079
:1004E0004F0700200148007A70470000640900208F
:1004F00070B500240D48C07A01280CD10B4908685A
:10050000FCF7B4FA05466421F7F71AFE84B2632CAF
:100510000ADD632408E005480088401D84B20A21F2
:100520002046F7F723FE84B2204670BD6409002000
:1005300070B5002407490868FCF798FA05460A21B7
:10054000F7F7FEFD84B20448844200DD04462046ED
:1005500070BD000064090020DE03000010B5002417
:100560000A2103480088F7F701FE84B2204610BD37
:100570000200002001480078704700000B000020B6
:1005800010B50024044804F0C5FA002801D0012465
:1005900000E00024204610BD0307000010B5002431
:1005A000054804F0B7FA002802D00120044601E013
:1005B0000020044610BD00000507000010B500240F
:1005C000054804F0A7FA002802D00120044601E003
:1005D0000020044610BD00000707000010B50024ED
:1005E000062004F097FA002801D0012400E000243E
:1005F000204610BD10B50024054804F08BFA0028F1
:1006000002D00120044601E00020044610BD000095
:100610000607000010B50024044804F07BFA002807
:1006200001D0012400E00024204610BD0305000095
:1006300010B50024044804F06DFA002801D001240C
:1006400000E00024204610BD040500000148807A27
:10065000704700006409002001488078704700005E
:10066000D00C00200148406870470000D00C0020EA
:100670000148407870470000D00C002070B500247D
:10068000FFF7D4FE002803D1FCF7F0FF04460DE08D
:10069000FFF7CCFE012806D1FCF7E8FF0546FCF782
:1006A00093FD044602E0FCF7E1FF0446204670BDDE
:1006B0000148407A704700006409002070B50024AA
:1006C0000D48C07A01280CD10B494868FCF7CEF9D7
:1006D00005466421F7F734FD84B2632C0ADD6324F8
:1006E00008E005488088401D84B20A212046F7F7BB
:1006F0003DFD84B2204670BD6409002070B5002421
:1007000007494868FCF7B2F905460A21F7F718FDD2
:1007100084B20448844200DD0446204670BD0000D7
:1007200064090020DE03000070B50024FFF77EFEA0
:10073000002803D1FCF7ACFF04460FE0FFF776FE7C
:10074000012807D10020FCF7A3FF0546FCF73CFD7C
:10075000044603E00020FCF79BFF0446204670BDE2
:1007600001480078704700004200002070B505463F
:100770000024032D00D170BD002D01D0012D1BD10F
:1007800081210320800204F075F98021134804F0D0
:1007900071F932211248FFF757FC002409E0A2004A
:1007A000104BD2189178A200985A04F063F9601C9B
:1007B000C4B23B2CF3DB0FE0022D0DD1002409E085
:1007C000A200094BD2189178A200985A04F052F96D
:1007D000601CC4B23B2CF3DB00BFCCE70206000078
:1007E000A086010018EE010004EF0100F8B5002119
:1007F00000240023002200BF0AE001258D40ABB297
:1008000005881D402C469C4200D10A464D1CA9B2C9
:100810001029F2DB0588FF2D1FDC284D6D7E068830
:10082000B543264E757635462D7E0688B543234E54
:10083000357635466D7E8678F607F60F9640354359
:100840001E4E757635462D7E867802273E40760808
:1008500096403543194E357622E0184DED7E0688D8
:10086000B543164EF5763546AD7E0688B543134E34
:10087000B5768578ED07ED0F1646083EB5400F4E6C
:10088000F67E35430D4EF5768578022635406D08A7
:100890001646083EB540094EB67E3543074EB5763E
:1008A0000025009505E000BF6D462D786D1CEEB269
:1008B00000966D462D78012DF5D9F8BD206B0440CA
:1008C000C107C90F002905D00021394A1171002242
:1008D00038490A7102210140002905D00021344A1B
:1008E0001172002233490A7204210140002905D007
:1008F00000212F4A117300222E490A73082101405A
:10090000002905D000212A4A1174002229490A74BD
:1009100010210140002905D00021254A117500222F
:1009200024490A7520210140002905D00021204AD0
:10093000117600221F490A7640210140002904D087
:1009400000221B494A711B494A718021014000293C
:1009500004D0002216494A7216494A72FF21013119
:100960000140002904D0002211494A7311494A73F9
:10097000012149020140002904D000220C494A7497
:100980000C494A74012189020140002904D0002247
:1009900007494A7507494A750121C90201400029E2
:1009A00004D0002202494A7602494A767047000084
:1009B0000060004000610040C107C90F002905D058
:1009C00001223C490A7100213B4A11710221014078
:1009D000002905D0012237490A720021364A1172D6
:1009E00004210140002905D0012232490A73002167
:1009F000314A117308210140002905D001222D49F7
:100A00000A7400212C4A117410210140002905D0DC
:100A1000012228490A750021274A11752021014029
:100A2000002905D0012223490A760021224A1176A5
:100A300040210140002905D001221E494A710022AF
:100A40001D494A7180210140002905D00122194920
:100A50004A72002218494A72FF21013101400029DF
:100A600005D0012213494A73002213494A73012118
:100A700049020140002905D001220E494A74002292
:100A80000D494A74012189020140002905D0012243
:100A900008494A75002208494A750121C9020140E6
:100AA000002905D0012203494A76002202494A76EC
:100AB00070470000006100400060004010B50C4825
:100AC0000078002803D00B4A50689168884708488E
:100AD0004078002803D0084A506891688847044845
:100AE0008078002803D0054A50689168884710BD77
:100AF0000060004000030020800400200006002069
:100B000010B508480079002803D0074A10695169D8
:100B1000884704484079002803D0044A5068916807
:100B2000884710BD00600040000300208C040020B6
:100B300010B50848007A002803D0074AD069116A26
:100B400088470448407A002803D0044A50689168D6
:100B5000884710BD0060004000030020980400207A
:100B600010B50848007B002803D0074A906AD16A74
:100B700088470448407B002803D0044A50689168A5
:100B8000884710BD0060004000030020A40400203E
:100B900010B50848007C002803D0074A506B916BC1
:100BA00088470448407C002803D0044A5068916874
:100BB000884710BD0060004000030020B004002002
:100BC00010B50848007D002803D0074A106C516C0E
:100BD00088470448407D002803D0044A5068916843
:100BE000884710BD0060004000030020BC040020C6
:100BF00010B50848007E002803D0074AD06C116D5C
:100C000088470448407E002803D0044A5068916811
:100C1000884710BD0060004000030020C804002089
:100C200010B50848407F002803D0074A50689168F3
:100C300088470448007F002803D0044A906DD16D96
:100C4000884710BD00600040D4040020000300204D
:100C500010B508484078002803D0074A50689168CA
:100C6000884704480078002803D0044A506E916EEB
:100C7000884710BD20600040E004002000030020F1
:100C800010B509480079002803D0084A106F516F49
:100C900088470548001D4078002803D0044A506862
:100CA0009168884710BD00002060004000030020CC
:100CB000EC04002010B5034AD06F78329168884761
:100CC00010BD00000003002010B5024A5068916872
:100CD000884710BD8403002010B50948007C002817
:100CE00003D0084A5068916888470548103040781A
:100CF000002803D0044A50689168884710BD00005E
:100D000020600040900300201005002010B5024A2A
:100D100050689168884710BD9C03002010B5024AB6
:100D200050689168884710BDA803002010B5094895
:100D3000007F002803D0084A50689168884705481A
:100D40001C304078002803D0044A506891688847D6
:100D500010BD000020600040B403002034050020D6
:100D600010B50C480078002803D00B4A50689168F1
:100D7000884708484078002803D0084A506891689E
:100D8000884704488078002803D0054A5068916855
:100D9000884710BD40600040C0030020400500208F
:100DA000C006002010B50D480079002803D00C4A79
:100DB0005068916888470948001D4078002803D092
:100DC000084A5068916888470448001D80780028C8
:100DD00003D0054A50689168884710BD40600040C4
:100DE000CC0300204C050020CC06002010B50D4897
:100DF000007A002803D00C4A506891688847094857
:100E000008304078002803D0084A50689168884725
:100E1000044808308078002803D0054A506891685B
:100E2000884710BD40600040D803002058050020CE
:100E3000D806002010B50D48007B002803D00C4ACE
:100E400050689168884709480C304078002803D0E2
:100E5000084A50689168884704480C308078002818
:100E600003D0054A50689168884710BD4060004033
:100E7000E403002064050020E406002010B50D48BE
:100E8000007C002803D00C4A5068916888470948C4
:100E900010304078002803D0084A5068916888478D
:100EA000044810308078002803D0054A50689168C3
:100EB000884710BD40600040F0030020700500200E
:100EC000F006002010B5024A50689168884710BDAE
:100ED000FC03002010B50948007E002803D0084A12
:100EE000506891688847054818304078002803D03A
:100EF000044A50689168884710BD00004060004077
:100F0000080400208805002010B50948007F00284B
:100F100003D0084A50689168884705481C304078DB
:100F2000002803D0044A50689168884710BD00002B
:100F300040600040140400209405002010B50848CB
:100F40000078002803D0074A506891688847044811
:100F50004078002803D0044A50689168884710BD43
:100F60006060004020040020A005002010B5094862
:100F70000079002803D0084A5068916888470548DE
:100F8000001D4078002803D0044A506891688847C3
:100F900010BD0000606000402C040020AC05002063
:100FA00010B50948007A002803D0084A50689168B3
:100FB0008847054808304078002803D0044A506824
:100FC0009168884710BD0000606000403804002030
:100FD000B805002010B5024A50689168884710BDD6
:100FE0004404002010B5024A50689168884710BD3B
:100FF0005004002010B50948007D002803D0084A9D
:10100000506891688847054814304078002803D01C
:10101000044A50689168884710BD00006060004035
:101020005C040020DC05002010B50948007E002883
:1010300003D0084A506891688847054818304078BE
:10104000002803D0044A50689168884710BD00000A
:101050006060004068040020E805002010B50948E1
:10106000007F002803D0084A5068916888470548E7
:101070001C304078002803D0044A506891688847A3
:1010800010BD00006060004074040020F4050020E2
:1010900010B5FE4800688079002806D001286ED07F
:1010A00002286DD003286CD104E2F848006840792A
:1010B00003000DF0E3F80A0614BC2BBC47BC67BC68
:1010C0009BBC09F099FA0020F0490968C873EF4801
:1010D00000684079401CED4909684871AEE0EC4970
:1010E0000969EA4A1268D27A885C09F0FDFAE74891
:1010F00000684079401CE54909684871E348006888
:101100004079401CE1490968487197E001F096FE7A
:10111000002810D109F0E8FADC4800684079401C4A
:10112000DA4909684871D94800684079401CD749B4
:101130000968487105E009F089FA0020D349096877
:1011400048717BE001F07AFE002811D1012009F0FE
:10115000CBFACE4800684079401CCC4909684871F8
:10116000CA4800684079401CC8490968487105E0D0
:1011700009F06CFA0020C549096848715EE05FE03B
:10118000FEE0A3E101F05AFE002828D1BF4909681A
:10119000C97A24225143BF4A12688918BB4A12688F
:1011A000D27B885C09F0A0FAB8480068C07B401C7C
:1011B000B6490968C873B5480068C07B242814D3B1
:1011C000B24800684079401CB04909684871AF488E
:1011D00000684079401CAD490968487105E009F094
:1011E00035FA0020A9490968487127E001F026FE78
:1011F000002815D1A5480068C07A401CA349096899
:10120000C872A2480068C07AA1490978884207DB01
:1012100000209E490968C87201209C4909688871AC
:1012200009F014FA002099490968487106E009F0AC
:101230000DFA002095490968487100BF00BF4FE1D1
:1012400092480068407903000DF018F808051391E2
:101250002A914791709109F0CFF900208B490968D4
:10126000C8738A4800684079401C884909684871F9
:1012700084E087490969854A1268D27A885C09F056
:1012800033FA824800684079401C804909684871F7
:101290007E4800684079401C7C49096848716DE0CF
:1012A00001F0CCFD002811D1262009F01DFA774865
:1012B00000684079401C75490968487173480068A6
:1012C0004079401C71490968487105E009F0BEF990
:1012D00000206E490968487150E001F0AFFD002818
:1012E0001DD1012009F000FA68480068C07B401C4D
:1012F00066490968C87365480068C07B242814D310
:10130000624800684079401C6049096848715F483C
:1013100000684079401C5D490968487105E009F0A2
:1013200095F9002059490968487127E001F086FDC8
:10133000002815D155480068C07A401C53490968F7
:10134000C87252480068C07A51490978884207DB60
:1013500000204E490968C87202204C49096888710A
:1013600009F074F9002049490968487106E009F05C
:101370006DF9002045490968487100BF00BFAFE022
:1013800042480068407903000CF078FF0805138B91
:101390002A8B478B638B09F02FF900203B490968A2
:1013A000C8733A4800684079401C38490968487158
:1013B0007EE037490969354A1268D27A885C09F0BB
:1013C00093F9324800684079401C304909684871F7
:1013D0002E4800684079401C2C490968487167E034
:1013E00001F02CFD002811D1252009F07DF92748B6
:1013F00000684079401C2549096848712348006805
:101400004079401C21490968487105E009F01EF93E
:1014100000201E49096848714AE001F00FFD0028CC
:1014200010D109F061F9194800684079401C17494A
:1014300009684871154800684079401C13490968DB
:10144000487105E009F002F9002010490968487167
:101450002EE001F0F3FC002815D10C480068C07A9A
:10146000401C0A490968C87208480068C07A0849DF
:101470000978884207DB002004490968C872032004
:1014800002490968887109F0E1F805E0D0070020F9
:10149000402B0020CC070020002012490968487129
:1014A00006E009F0D3F800200E490968487100BF32
:1014B00000BF15E000200B490968887109490968D7
:1014C0004871062007490968C87009E009F0BEF8AC
:1014D000002004490968487102490968887100BF01
:1014E00000BF10BDD007002010B56A4800684079E1
:1014F00003000CF0C3FE090610C627C644C6608E62
:10150000C60009F079F8634800684079401C6149D9
:1015100009684871BCE0604909695E4A1268D27A7C
:10152000885C09F0E1F85B4800684079401C594943
:1015300009684871574800684079401C5549096856
:101540004871A5E001F07AFC002811D14F2009F084
:10155000CBF8504800684079401C4E4909684871F2
:101560004C4800684079401C4A490968487105E0C8
:1015700009F06CF8002047490968487188E001F0DB
:101580005DFC002810D109F0AFF8424800684079AE
:10159000401C4049096848713E4800684079401C39
:1015A0003C490968487105E009F050F800203949C4
:1015B000096848716CE001F041FC002822D13548EF
:1015C0000068C07A401C33490968C8723148006815
:1015D000C07A3149097888420FDB00202D4909681B
:1015E000C8722C4800684079401C2A490968487133
:1015F000002028490968486208E000202549096858
:10160000487103E0002023490968487109F01EF879
:101610003EE020480068407C002816D01E48C06884
:10162000002803D01C48C1681920884700201949A8
:10163000096848621749096848711649096888713C
:10164000052014490968C8701AE012480068406A09
:10165000282807D20F480068406A401C0D490968D5
:1016600048620DE000200B49096848620949096891
:101670004871084909688871052006490968C870D9
:1016800006E008F0E3FF002002490968487100BF46
:1016900000BF10BDD0070020402B002010B5002453
:1016A000F7480068807A01287ED1F5480068C07943
:1016B00000287AD0F24800688079002804D00128F8
:1016C00074D0022873D191E1ED480068007B242892
:1016D0006ED2EB480068C07901287AD1002475E009
:1016E000E7480068C07A24214843E6490968401861
:1016F000E3490968097B415CE1480068C07A24221B
:101700005043E14A12688018DD4A1268127B805CFF
:10171000814229D0DA480068C07A24214843DA4956
:1017200009684018D6490968097B415CD4480068BB
:10173000C07A24225043D34A12688018D04A1268D3
:10174000127B8154CE480068407B242805D3CC48C6
:101750000068007BCA4909684873C9480068007B73
:10176000C7490968887308E0C5480068407B242899
:1017700003D20120C24909688871C1480068007B12
:10178000401CBF4909680873BD480068007B2428D5
:1017900008D3BB480068407B242803D20120B84905
:1017A00009688871B64805E0D3E1CDE169E0BAE1A6
:1017B00038E00EE00068007B242804D2B0480068BE
:1017C0008079012800D103E0601CC4B2242C87D3A7
:1017D00056E0002413E0AA480068C07A2421484358
:1017E000A94909684018015DA5480068C07A24220B
:1017F0005043A44A126880180155601CC4B2242CBE
:10180000E9D300209E490968487323209C49096850
:10181000887301209A4909688871242098490968C9
:1018200008732DE000209649096808739448006801
:10183000C07A401C92490968C87291480068C07A11
:1018400092490978884217DB8D480068007C01289E
:1018500004D102208A490968887106E0002088497D
:101860000968887186490968C87100208449096837
:10187000C872834909680874002081490968487161
:1018800061E17F480068407903000CF0F7FC08052F
:1018900013A62AA651A68EA60120794909680874C4
:1018A00008F0AAFE764800684079401C744909682F
:1018B000487199E075490969714A1268D27A885C61
:1018C00008F012FF6E4800684079401C6C490968B6
:1018D00048716B4800684079401C69490968487143
:1018E00082E001F0ABFA00281BD165490968497B09
:1018F000491CC8B208F0F8FE61480068407B6049A6
:101900000968C8735E4800684079401C5C490968F2
:1019100048715B4800684079401C59490968487122
:1019200005E008F093FE00205549096848715BE026
:1019300001F084FA00282BD151490968C97A242280
:101940005143504A126889184D4A1268D27B885C0C
:1019500008F0CAFE4A480068C07B401C4849096834
:10196000C87347480068C07B45490968897B88423D
:101970001ADD434800684079401C414909684871B4
:101980003F4800684079401C3D49096848710BE0B8
:1019900008F05CFE3A480068407B39490968C87322
:1019A00000203749096848711EE001F047FA002815
:1019B0000CD1334909688871242031490968C873FA
:1019C0002F49096848732E490968887308F03EFE5C
:1019D00000202B490968487106E008F037FE002016
:1019E00027490968487100BF00BFACE0244800687F
:1019F000407903000CF042FC08050F8E268E4C8EB9
:101A0000688E08F0F9FD1E4800684079401C1C49AA
:101A10000968487185E01D490969194A1268D27A36
:101A2000885C08F061FE164800684079401C144943
:101A300009684871124800684079401C10490968DB
:101A400048716EE001F0FAF9002811D1252008F064
:101A50004BFE0B4800684079401C094909684871F1
:101A6000074800684079401C05490968487105E04D
:101A700008F0ECFD002002490968487151E00000BF
:101A8000D0070020CC070020C8070020402B0020F2
:101A900001F0D4F9002810D108F026FE644800684F
:101AA0004079401C62490968487161480068407982
:101AB000401C5F490968487105E008F0C7FD002037
:101AC0005B49096848712CE001F0B8F900281AD187
:101AD00057480068C07A401C55490968C872544884
:101AE0000068C07A5349097888420CDB00205049CD
:101AF0000968C8724E49096888714D49096848717A
:101B00004B490968C87108F0A1FD002048490968DF
:101B1000487106E008F09AFD0020454909684871BF
:101B200000BF00BF0FE008F091FD002040490968A8
:101B300048713F49096888713D49096808733C4903
:101B40000968C87200BF71E00020394909688872CD
:101B50006CE037480068807A022867D13448006812
:101B6000007A00285ED0324800684079002804D00E
:101B700001280CD0032846D11BE008F03DFD2C487D
:101B800000684079401C2A490968487149E00020F2
:101B900008F0AAFD264800684079401C24490968DD
:101BA0004871234800684079401C21490968487100
:101BB00037E008F0EBFC002812D11D48006840789F
:101BC000401C1B4909684870194800684078032880
:101BD00012D301F0D3F900201549096848700BE0D1
:101BE0000020134909680872AA2011490968887001
:101BF00000200F490968487008F028FD00200C49B2
:101C0000096848710DE008F021FD002008490968C5
:101C10004871074909684870AA2005490968887011
:101C200000BF03E0002002490968887210BD00006F
:101C3000D0070020402B0020F8B504460D460026B2
:101C40000C2060431D49085C002801D00120F8BD2C
:101C50000C2060431949401885600C2060434018EF
:101C60008068002801D10120F1E701210C206043A8
:101C7000124A115400222046E317DB0E1B185B1199
:101C80005B01E31A9B000E4FDB19E717FF0E3F19AC
:101C90007F11DA550CF024FB00222046E317DB0EFF
:101CA0001B185B115B01E31A9F00064BFB18E7173B
:101CB000FF0E3F197F11DA553046C8E700030020B8
:101CC000006000400061004000BFFEE70948008856
:101CD000401C08490880084600880749884208DDFA
:101CE00006480078002804D00846024908800120F0
:101CF00088707047E4000020DC050000EF00002041
:101D000010B50B488078012810D10A4800780128C6
:101D100002D1094802F0D0FC06480078022802D11E
:101D2000054802F0C9FC00200249087010BD0000FF
:101D3000E4000020EF000020F900002070470000C0
:101D400010B500F005FE012803D1002001490880EC
:101D5000887010BDE4000020F0B505460E46174619
:101D600000243A463146284600F000FE00BF42E01B
:101D700000202101394A126850522101374A126865
:101D80008918488000212001344A12688018818017
:101D90002001324A12688018C18020012F4A12683F
:101DA0008018017220012D4A1268801841722001AA
:101DB0002A4A1268801881722001284A1268801805
:101DC000C17200202101254A126889180873002178
:101DD0002001224A126880184173002021011F4A05
:101DE000126889188873002120011C4A1268801823
:101DF000C173601CC4B21A484078A042B8DC6420A9
:101E00001849096808807D20C00016490968488083
:101E100015481449096888807D2000011149096826
:101E2000C88010490968088110480E49096848812E
:101E30000F480C490968888140000A490968C8812F
:101E40003220084909680882FF20F53005490968F1
:101E50004882044909688882F0BD0000900700208C
:101E6000840700208C0700204C040000102700008D
:101E70003075000038B5002404E0002013490855EF
:101E8000601C84B2282CF8D301216846417001708F
:101E90006A460F490D48FFF75FFF7D21C9003220D8
:101EA00000F054F90B490C4800F06EF90948643011
:101EB00000F000F90748C83000F00CF9074800F0BE
:101EC0001FF9074800F032F938BD0000DC2300207C
:101ED00088F3010028230000B80B00005424000000
:101EE0001027000013480078002803D10120114971
:101EF00008701EE00F480078012803D102200D4928
:101F0000087016E00B480078022803D10320094925
:101F100008700EE007480078032803D10420054923
:101F2000087006E003480078042802D10020014927
:101F300008707047EF000020F8B500240025002647
:101F40003648007800281ED135480078002803D193
:101F500001203349087016E031480078012803D188
:101F600002202F4908700EE02D480078022803D186
:101F700003202B49087006E029480078032802D185
:101F80000020274908702548007801280ED1012437
:101F90001725002623480123324629460090204673
:101FA00001F0C0FD1F4802F087FB36E01B480078B7
:101FB00002280FD101243B2500261A48401C01238A
:101FC000324629460090204601F0ACFD154802F04B
:101FD00073FB22E01148007803280DD1FEF726FAA2
:101FE000002803D101201049087102E000200E49A9
:101FF00008710CF015F910E00848007804280CD19D
:10200000FEF726FA002803D101200749487102E0B3
:102010000020054948710CF003F9F8BDEF000020DD
:10202000F0000020F9000020E800002010B5044670
:1020300023000CF023F9093306090C0D0E0F313281
:102040003600FFF779FF2DE0FFF74CFF2AE029E08B
:1020500028E027E001F03CFD1348007803280ED16A
:102060001248007800280AD1FEF7ECF9002803D1C5
:1020700001200F49887102E000200D4988710A484B
:102080000078012805D109480078002801D1FAF725
:1020900043FD09F0B7FF05E004E003E0FFF716FE9B
:1020A00000E000BF00BF10BDF0000020EF000020E6
:1020B000E800002001460020054A126852898A4241
:1020C00001DC012002E0024A126811817047000021
:1020D0008C07002001460020084A126812898A42B3
:1020E00001DB012009E0054A126892898A4201DC7D
:1020F000012002E0014A1268518170478C070020DC
:1021000001460020084A126852898A4201DB0120F8
:1021100009E0054A1268D2898A4201DC012002E006
:10212000014A1268918170478C0700200146002007
:10213000054A126892898A4201DB012002E0024AC4
:102140001268D181704700008C07002002460020F1
:102150000C4B1B681B8A934201DD012010E08A4270
:1021600001DB01200CE0074B1B689B888B4201DCE4
:10217000012005E0034B1B681A80024B1B68598045
:10218000704700008C070020024600200C4B1B68A3
:102190001B8A934201DD012010E08A4201DB01200D
:1021A0000CE0074B1B685B88934201DB012005E0D4
:1021B000034B1B689A80024B1B68D9807047000054
:1021C0008C07002070B5044600250C206043FE49B2
:1021D000096840184068002807D00C216143FA4A7A
:1021E000126889184868804705460C206043F64904
:1021F0000968085C002873D10C206043F249096823
:1022000040188068002874D02001F04909684018FF
:10221000C07A02280AD1032D08D10C206043EA4A73
:102220001268801881680120884762E02001E74930
:1022300009684018C07A02280AD1042D08D10C2060
:102240006043E14A1268801881680220884750E0A4
:102250002001DE4909684018C07A02280AD1052DFC
:1022600008D10C206043D84A126880188168032086
:1022700088473EE02001D54909684018C07A022805
:102280000AD1062D08D10C206043CF4A126880186D
:102290008168042088472CE02001CC490968401857
:1022A000C07A02280AD1072D08D10C206043C64A03
:1022B000126880188168052088471AE02001C34908
:1022C00009684018C07A02280BD1082D09D10C20CA
:1022D0006043BD4A1268801881680620884708E07C
:1022E0000DE00C206043B84A126880188168002015
:1022F00088472001B54909684018C5720CE30C20D5
:102300006043B1490968085C012873D10C2060431F
:10231000AD49096840188068002874D02001AB4995
:1023200009684018C07A03280AD1022D08D10C2070
:102330006043A54A1268801881680120884762E0DE
:102340002001A24909684018C07A04280AD1022D48
:1023500008D10C2060439C4A1268801881680220D2
:10236000884750E02001994909684018C07A05283B
:102370000AD1022D08D10C206043934A12688018BC
:102380008168032088473EE0200190490968401891
:10239000C07A06280AD1022D08D10C2060438A4A4F
:1023A000126880188168042088472CE02001874942
:1023B00009684018C07A07280AD1022D08D10C20DC
:1023C0006043814A126880188168052088471AE0B6
:1023D00020017E4909684018C07A08280BD1022DD7
:1023E00009D10C206043784A126880188168062061
:1023F000884708E00DE00C206043734A126880189B
:102400008168002088472001704909684018C5721A
:1024100082E20C2060436C490968085C0228F7D10D
:10242000002D7DD1200169490968085A6849096869
:10243000098A884275DA200164490968085A0A3015
:1024400081B22001614A1268115220015F49096876
:10245000085A5F490968098A884231DB20015B49D3
:102460000968401840885A4909680988884227DB6A
:10247000200156490968401840885549096849882B
:1024800088421DDC00202101504A126889184880CA
:1024900020014E4909684018807A0028B8D10C20E4
:1024A000604349490968401880680028B0D00C2072
:1024B0006043454A126880188168012088472BE2F2
:1024C000200142490968085A41490968098A884235
:1024D0009EDB20013D490968401840883C49096855
:1024E0008988884294DB200138490968401840886F
:1024F00037490968C98888428ADC00202101334AAB
:102500001268891848802001304909684018807A8B
:102510000028D4D10C2060432B490968401801E001
:1025200063E00BE080680028C9D00C206043264A95
:1025300012688018816802208847EDE1002021019F
:10254000224A1268891848802101204A1268891895
:10255000C872002120011D4A12688018C180200124
:102560001A4A1268801841722001184A12688018AD
:102570008172184801782001144A1268801801728B
:1025800000202101114A12688918888021010F4A10
:1025900012688918087321010C4A12688918487357
:1025A00021010A4A12688918887300212001074A0C
:1025B00012688018C1730C206043034909684018F1
:1025C00080680028B9D007E0880700209007002025
:1025D0008C070020840700200C206043CF4A12683B
:1025E000801881680020884796E1012DA5D120013F
:1025F000CB4909684018C07AA84225D000212001A3
:10260000C74A12688018418000202101C44A12681C
:102610008918C8802001C24909684018C572C1489C
:1026200000782101BE4A12688918487200202101F1
:10263000BB4A126889188880BA4801782001B84AD4
:1026400012688018017267E12001B54909684018D5
:10265000007AB4490978884220D0B2480078210134
:10266000AF4A1268891808722001AD4909684018FC
:10267000407AAC490978884209D02001A849096804
:10268000401880882101A64A12688918C880002154
:102690002001A34A12688018818012E02001A0491D
:1026A000096840188088A04988420AD220019C49C4
:1026B0000968401880880A302101994A12688918EF
:1026C00088802001964909684018408896498842C8
:1026D0000AD2200192490968401840880A30210135
:1026E0008F4A12688918488020018D49096840186E
:1026F000407A8C490978884205D001202101884A16
:102700001268891888722001854909684018408834
:10271000864909680988884204DB00212001804A33
:102720001268115220017E4909684018807A0028F9
:102730007ED10C20604379490968401880680028E0
:1027400077D02001764909684018408877490968A0
:102750000989884214DB2001714909684018007B0F
:1027600000280DD10C2060436C4A126880188168E3
:102770000320884701202101694A126889180873DB
:1027800020016749096840184088684909684989F3
:10279000884214DB2001624909684018407B002808
:1027A0000DD10C2060435D4A1268801881680420B6
:1027B0008847012021015A4A12688918487320016C
:1027C00057490968401840885849096889898842EA
:1027D00014DB2001524909684018807B00280DD184
:1027E0000C2060434D4A1268801881680520884794
:1027F000012021014A4A126889188873200148493A
:1028000009684018408849490968C989884210DB2D
:102810002001434909684018C07B00287CD10C2066
:1028200060433E4A1268801881680620884701E0AC
:1028300007E03BE001202101394A12688918C8737A
:102840006AE02001364909684018407A01282ED1F3
:102850003448007802282AD12001314909684018FB
:10286000C08832490968498A884255DB20012C49D1
:102870000968401880882D490968898A88424BDB9D
:102880000C2060432549096840188068002843D01F
:102890000C206043214A126880188168072088470D
:1028A000002021011E4A12688918487234E0200174
:1028B0001B4909684018407A02282DD11948007830
:1028C000012829D12001164909684018C0881749F4
:1028D0000968898A88421FDB20011149096840186C
:1028E000808812490968498A884215DB0C206043B8
:1028F0000A4909684018806800280DD00C20604300
:10290000064A126880188168082088470020210143
:10291000034A12688918487270BD000088070020B9
:102920009007002084070020F0FF00008C070020A3
:1029300010B5002400BF04E02046FFF743FC601CF4
:10294000C4B202484078A042F6DC10BD84070020E3
:1029500010B50024044802F0DDF8002800D000E0A3
:102960000124204610BD00000304000010B5074BF1
:1029700014781C7054785C70054B1960054B186016
:1029800003461833044C236010BD00008407002068
:10299000880700208C0700209007002010B504460F
:1029A000012C09D164220C21002000F0DFF8012164
:1029B000022004F095F808E000220C21104600F0F7
:1029C000D5F80021022004F08BF810BD10B50024CA
:1029D00004210848F8F776FB552801D1012407E0C7
:1029E000042000F0E7FF002801D0002400E00124CB
:1029F000204610BD2808002010B50446012C09D13E
:102A000064221C21002000F0B1F80121062004F00E
:102A100067F808E000221C21104600F0A7F800210A
:102A2000062004F05DF810BD10B50024062000F06B
:102A3000C1FF002801D0012400E00024204610BD81
:102A400010B50446012C09D164221721002000F0A2
:102A50008DF80121042004F043F808E0002217213A
:102A6000104600F083F80021042004F039F810BD6E
:102A700000200449097A002901D0012000E000204B
:102A800070470000D00C002010B50446022C1CD169
:102A900000220D21104600F069F8FDF717FD00280F
:102AA00009D064220B21002000F060F801210D20E4
:102AB00004F016F847E000220B21104600F056F80B
:102AC00000210D2004F00CF83DE0032C1CD1002265
:102AD0000B21104600F04AF8FDF7F8FC002809D059
:102AE00064220D21002000F041F801210D2003F0A7
:102AF000F7FF28E000220D21104600F037F80021F2
:102B00000D2003F0EDFF1EE0012C0ED164220D21FB
:102B1000002000F02BF800220B21104600F026F8D0
:102B200001210D2003F0DCFF0DE000220D211046F5
:102B300000F01CF800220B21104600F017F80021CD
:102B40000D2003F0CDFF10BD10B50024FCF718FFD9
:102B5000022801D1022406E0FCF712FF012801D16E
:102B6000032400E00124204610BD000010B5064BF0
:102B70001B78834207DD242905D224234343034CD9
:102B800024681B195A5410BD402B0020C807002090
:102B900010B574480068407903000BF06FFB0B0719
:102BA00011D325D35A6D77D38DA8D30007F024FD18
:102BB0006C4800684079401C6A4909684871CFE058
:102BC00069494969087807F08FFD664800684079CF
:102BD000401C644909684871624800684079401C9B
:102BE000604909684871BBE000F028F9002811D15C
:102BF0007F2007F079FD5B4800684079401C594907
:102C000009684871574800684079401C554909686F
:102C100048711DE0534800684078401C51490968DC
:102C2000487050480068407803280BD300204D4975
:102C300009684870AA204B490968887003204949EF
:102C40000968C87007F002FD00204649096848710C
:102C500086E000F0F3F8002807D142480068407988
:102C6000401C40490968487103E000203D4909685B
:102C7000487107F0EBFC73E007F0BEFC39480068D0
:102C80004079401C37490968487169E0364949690B
:102C90000978491CC8B207F027FD3248006840791E
:102CA000401C3049096848712E4800684079401C32
:102CB0002C490968487153E000F0C0F800280FD192
:102CC00007F06CFC274909688870012007F0E0FCD8
:102CD000244800684079401C22490968487105E091
:102CE00007F0B4FC00201F490968487138E01D480E
:102CF0000068807818280CD102201A4909680870E9
:102D00000020184909684870042016490968C870ED
:102D100011E0144800684078401C12490968487066
:102D2000104800684078032805D300F027F90020F8
:102D30000C490968487007F089FC002009490968B6
:102D400048710DE007F082FC0020064909684871CF
:102D5000044909684870AA2002490968887000BFC0
:102D600000BF10BDD0070020402B002010B5314817
:102D700000684079002804D001280CD0032848D1ED
:102D80001DE007F039FC2B4800684079401C2949B8
:102D9000096848714BE028490969087807F0A4FCE4
:102DA000244800684079401C22490968487121483C
:102DB00000684079401C1F490968487137E000F0FD
:102DC0003DF800280CD101201A490968087000203C
:102DD000184909684870042016490968C87011E04C
:102DE000144800684078401C12490968487011482E
:102DF00000684078032805D300F0C0F800200D4992
:102E00000968487007F022FC00200A4909684871E7
:102E10000DE007F01BFC00200649096848710549D0
:102E200009684870AA2003490968887000BF00BF7C
:102E300010BD0000D0070020402B002010B507F087
:102E4000A5FB04461F4800680078002838D01D48BC
:102E50000068C078042833D3002C09D10021194818
:102E60000068C07A8200174800681430815027E05B
:102E700014480068C07A8100124800681430405835
:102E80001149884211D20F480068C07A81000D486C
:102E9000006814304058401C0A490968C97A8A0001
:102EA00008490968143188500AE000F067F80021E9
:102EB00004480068C07A82000248006814308150DB
:102EC000204610BDD0070020B80B000000B587B029
:102ED0000120694608710848029008480390084894
:102EE0000490084805900848069001A9074800F09A
:102EF0000FF807B000BD000035320100014D0100A0
:102F000009E40100E9F30100E8F301003C2400209A
:102F1000F8B506460F46002400253946304600F035
:102F2000EFF900BF14E000250EE0002124206043EB
:102F30000B4A12688018415524206043094A1268E0
:102F400080184155681CC5B2242DEED3601CC4B254
:102F500005480078A042E6DC00F010F8F8BD00005B
:102F6000C8070020CC070020402B00200120024988
:102F70000968087170470000D007002010B500F004
:102F800073F9002003490968087002490968C8708C
:102F900010BD0000D007002007480068C078062850
:102FA00008D105480068C079002803D101200249F2
:102FB0000968C87170470000D007002010B5554857
:102FC0000068C07803000BF059F908671D1A171440
:102FD000110E056650484068002803D04E484168ED
:102FE0000020884793E000F0E5F890E000F0C6F894
:102FF0008DE000F0D1F88AE0FFF7B8FE87E0FFF738
:10300000C7FD84E044484068002803D04248416836
:10301000012088473F480068407C00281AD03E487D
:10302000C068002803D03C48C168C82088470020F9
:10303000384909684862374800680078002804D099
:10304000042034490968C87024E002203149096825
:10305000C8701FE02F480068406A401C2D4909686D
:1030600048622C480068406A7D21C900884211D31B
:10307000002028490968486226480068007800282E
:1030800004D0042023490968C87003E002202149C4
:103090000968C8703BE000BF1F484068002803D0A3
:1030A0001D484168002088471A480068407C002875
:1030B00013D01948C068002803D01748C168C82039
:1030C0008847002013490968486212480068C078A0
:1030D000401C10490968C87018E00E480068406A32
:1030E000401C0C49096848620A480068406A7D2112
:1030F000C90088420AD30020064909684862054889
:103100000068C078401C03490968C87000BF00BF50
:1031100010BD0000D0070020402B002010B515483E
:103120000068C078072824D0012012490968487433
:1031300008E011488068002802D00F49886880475D
:10314000FFF73CFF0B480068C0780628F1D109481A
:103150000068007A0028ECD106480068C079002891
:10316000E7D104480068807A0028E2D10149096863
:10317000487410BDD0070020402B002010B5054832
:1031800000680078012802D1FDF782FF01E0F6F720
:10319000AFFA10BDD007002010B5054800680078D0
:1031A000012802D1FEF7A0F901E0F6F77FFE10BD7D
:1031B000D007002010B51D480068807A002829D16A
:1031C0001A480068007A002803D0022017490968CD
:1031D000887216480068C079002803D0012013497E
:1031E00009688872114800680079012812D100200E
:1031F0000E49096808710D490968887207200B4952
:103200000968C8700A484068002803D00848416827
:1032100000208847054800680078012802D1FEF7A1
:103220003DFA01E0F6F71CFF10BD0000D0070020BA
:10323000402B002010B504462146084801F086FCCA
:1032400007480078002805D1002C03D0322105481A
:10325000FCF7FAFE0248047010BD000001030000F4
:103260000201002050C30000002024490968487072
:10327000AA2022490968887000202049096848620C
:103280001E49096808711D49096848711B49096888
:1032900088711A490968C87118490968087217497C
:1032A0000968887215490968C87214490968087361
:1032B00024201249096848731049096888730F4926
:1032C0000968C87300200D49096808740B4909682A
:1032D00048740A490968887408490968C874074924
:1032E0000968486100210548006881610348006859
:1032F000C16102480068016270470000D0070020E9
:1033000010B50A780D4B1860034628330C4C236027
:1033100024235343044628341B190A4C23600A4CC7
:103320004B6863608B68A360CB68E3604B69636143
:103330000B6923610B78237010BD0000D0070020BB
:10334000C8070020CC070020402B00200748006859
:10335000C078062808D105480068007A002803D103
:10336000012002490968087270470000D007002058
:1033700010B50446012C09D1642220210020FFF75A
:10338000F5FB0121084603F0ABFB08E000222021F9
:103390001046FFF7EBFB0021012003F0A1FB10BD5D
:1033A00010B50024032000F005FB002801D0012403
:1033B00000E00024204610BD10B50446032C0ED1B9
:1033C000642215210020FFF7D1FB002214211046B2
:1033D000FFF7CCFB01210E2003F082FB39E0022C29
:1033E0001CD1FDF773F8002809D0642214210020B5
:1033F000FFF7BCFB01210E2003F072FB08E0002266
:1034000014211046FFF7B2FB00210E2003F068FBE9
:10341000002215211046FFF7A9FB1AE0012C0ED15E
:10342000642214210020FFF7A1FB01210E2003F0EC
:1034300057FB002215211046FFF798FB09E00022F8
:1034400015211046FFF792FB002214211046FFF7CA
:103450008DFB10BD10B50024F9F7CEF9094988425B
:103460000DD3FDF787F8002807D1FCF7A5FF012849
:1034700001DD032404E0022402E0022400E0012430
:10348000204610BDB80B000010B50446012C09D130
:1034900064221D210020FFF769FB0121002003F0B9
:1034A0001FFB08E000221D211046FFF75FFB0021F3
:1034B000084603F015FB10BD10B50024022000F0F3
:1034C00079FA002810D0012410480078052805DA80
:1034D0000E480078401C0D49087015E005200B4986
:1034E0000870002048700FE0002408484078052844
:1034F00005DA06484078401C0449487004E005207D
:103500000249487000200870204610BD1E010020AE
:1035100010B50446012C09D164221E210020FFF7BA
:1035200025FB0121092003F0DBFA08E000221E211F
:103530001046FFF71BFB0021092003F0D1FA10BD54
:1035400070B5002400250026FCF744FE0546FCF774
:103550004DFE064602210848F7F7B4FD552800D174
:1035600008E0012E01D1002404E0012D01D1012445
:1035700000E00024204670BD2808002010B5044655
:10358000012C09D164221F210020FFF7EFFA01214D
:10359000082003F0A5FA08E000221F211046FFF7DB
:1035A000E5FA0021082003F09BFA10BD70B5002554
:1035B0000024FCF747FE044603210C48F7F782FD80
:1035C000552803D101200A4908800AE0762C03DA45
:1035D00001200749088004E0782C02DB0020044920
:1035E000088003480588284670BD00002808002090
:1035F0002001002010B50446012C09D164222121AC
:103600000020FFF7B3FA0121072003F069FA08E070
:10361000002221211046FFF7A9FA0021072003F01C
:103620005FFA10BD10B50024FCF7D8FE002801D1C8
:10363000012400E00024204610BD10B50446012CF2
:1036400009D1642216210020FFF790FA01210320FE
:1036500003F046FA08E0002216211046FFF786FA2A
:103660000021032003F03CFA10BD10B50024052012
:1036700000F0A0F9002801D0012400E00024204639
:1036800010BD10B50446012C09D164221921002077
:10369000FFF76CFA0121052003F022FA3CE0022C2E
:1036A00017D1FCF713FF002809D06422192100204C
:1036B000FFF75CFA0121052003F012FA2CE000224A
:1036C00019211046FFF752FA0021052003F008FAED
:1036D00022E0032C17D1FCF7FFFE002809D064225A
:1036E00019210020FFF742FA0121052003F0F8F923
:1036F00012E0002219211046FFF738FA00210520B8
:1037000003F0EEF908E0002219211046FFF72EFA27
:103710000021052003F0E4F910BD000010B50024DD
:10372000FCF790FE01282FD104211948F7F7CAFCB5
:10373000552801D1012428E0FCF764FD01280BD0B5
:10374000FCF760FD022807D0FCF75CFD032803D0DE
:10375000FCF758FD052801D1012416E0FCF752FDC5
:10376000042801D1022410E0FCF74CFD062801D109
:1037700003240AE0FCF746FD002803D0FCF742FDD5
:10378000072802D1002400E00024204610BD0000DC
:103790002808002010B50446012C0ED164221B21FC
:1037A0000020FFF7E3F900221A211046FFF7DEF9A7
:1037B00001210A2003F094F91EE0022C0ED16422AC
:1037C0001A210020FFF7D2F900221B211046FFF733
:1037D000CDF901210A2003F083F90DE000221A211E
:1037E0001046FFF7C3F900221B211046FFF7BEF970
:1037F00000210A2003F074F910BD10B50024FCF775
:1038000025FF012801D1012400E00224204610BD3B
:1038100010B5F9F70BF80446204610BD10B5034B60
:1038200007220349034800F013F910BD11380100C5
:1038300094F301000424002070B506465C488068BB
:10384000002804D05A4988688047054600E00025D2
:103850000024A6E0564841680C20604308184088C0
:10386000A84207D0524841680C206043081840889D
:1038700002287DD14E4841680C20604308188068BA
:1038800000280CD04A494A680C21614351188868C5
:10389000804747490968E2008918487009E04448B0
:1038A00041680C206043095C41480068E2008018D0
:1038B00041703F480068E100401840783C49096881
:1038C000E200895C88420FD039480068E100401866
:1038D000417837480068E200815400203449096883
:1038E000E200891848605AE031480068E100401859
:1038F00041782F4842680C2060431018407881427C
:103900001FD12B480068E1004018416828484268F0
:103910000C2060431018808881420BD8244800682E
:10392000E10040184068801921490968E2008918BF
:10393000486034E001201E490968E2008918488087
:103940002DE01B480068E1004018416818484268B3
:103950000C2060431018C08881420DD814480068BC
:10396000E10040184068811911480068E20000E059
:1039700009E08018416012E000200D490968E2006A
:10398000891848800BE0002009490968E20089187D
:103990004880002106480068E20080184160601CF1
:1039A00084B203488089A04200DD53E770BD000067
:1039B000F82A00200146064A92898A4205DD044A17
:1039C0001268CB00D218508800E000207047000039
:1039D000F82A0020002000BF14E00D494A680C219D
:1039E00041435118498801290AD10021084A126827
:1039F000C300D2185180064A1268C300D218516021
:103A0000411C88B2024989898142E6DC7047000086
:103A1000F82A0020002000BF13E00C494A680C215E
:103A2000414351184988002909D1084A1268C30046
:103A3000D2185180054A1268C300D2185160411C47
:103A400088B2024989898142E7DC7047F82A002060
:103A5000F0B504460020164DAB6069602C60AA8169
:103A600000BF1FE0124D6E680C254543755D104E7A
:103A70003668C700F61975700D4D6E680C25454304
:103A8000755D0B4E3668C700F5550025084E366843
:103A9000C700F6197580064E3668C700F6197560BE
:103AA000451CA8B2024DAD898542DBDCF0BD0000AB
:103AB000F82A002070B505460E46002E05D0314686
:103AC0002846F4F73DFB044600E02C46204670BD36
:103AD00010B5FCF783FC002809D1054800780328BD
:103AE00005D104480078002801D1F9F779FB10BD11
:103AF000F0000020EF000020012003498871002021
:103B00000249087070470000E8000020EF00002024
:103B10000020034908714871012088717047000036
:103B2000E800002070B5049C2578914216DD01283C
:103B30000AD18D4206DAFF26F61AAE420ED3EE18EF
:103B4000F5B20BE0154609E0022807D1954204DDE5
:103B50009D4203DBEE1AF5B200E00D46257070BD04
:103B60000D4A4168516081699161C168D160416AC3
:103B70005162016A11620168116041695161816895
:103B80009160C169D16101691161816A916200210D
:103B9000024A117070470000142B0020C407002057
:103BA00010B5FFF717FFF8F7C1FC00210148F7F740
:103BB00089FB10BD3408002010B5F8F7B7FCFFF7FB
:103BC00029FF08F061FC08F0FDFCFBF7B1FDFAF7F6
:103BD000F3FAFFF791FFF9F7A7F8F7F779F955210D
:103BE0000148F7F76FFB10BD340800201CB500201A
:103BF0003849087006F0B0FC0020FCF7B7FD0AF069
:103C000065FEF7F75DFE55213348F7F75BFBF8F7E4
:103C1000C5FEF6F777FDF6F7F5FFE12040020AF062
:103C200097FA00F08BFAF7F753F906F077FEF8F7FA
:103C30007DFCFAF7BFF8F9F703F9F9F781F8FFF718
:103C4000EDFDFEF717F9FFF741F9F9F7CBFFFBF7A9
:103C50009BFDFAF7B1FA214AFF219131002008F0CB
:103C600079FD1E4AFF219131012008F073FD0022E9
:103C70001146104608F0B2FC00220121104608F05F
:103C8000ADFC00220221104608F0A8FC00221146DB
:103C9000012008F0A3FC08F0DDFB08F093FCFFF71F
:103CA00037FFF9F759FD00200D49887148710871F7
:103CB0000120887048701420087007226846F4F7C5
:103CC000D6FA0199009800F091FF0221012000F03E
:103CD0006DFE1CBD01010020340800200090D003BF
:103CE000120100207047000010B50446552C03D186
:103CF00005494869804702E0034908688047002079
:103D00000249087010BD0000142B0020C4070020D9
:103D100010B54648007803000AF0B0FA0A06111BF5
:103D200026303B465051738141484068002802D0FC
:103D30003F494868804701203C49087000BF3C4823
:103D40008068002804D03A4988688047374908705D
:103D500069E03748C068002802D03549C868804704
:103D600003203249087000BF31480069002804D0A0
:103D70002F49086980472D49087054E02C48406954
:103D8000002802D02A494869804700202749087046
:103D900049E027488069002802D025498869804782
:103DA00006202249087000BF2148C069002804D0BD
:103DB0001F49C86980471D49087034E000BF1B488F
:103DC000007807280AD11A48006A002802D018494A
:103DD000086A804709201549087011E013480078E7
:103DE00008280AD11248406A002802D01049486ABF
:103DF000804709200D49087002E000200B49087037
:103E000000BF0A480078002808D00948806A0028C6
:103E100004D00749886A80470449087003E00020FD
:103E20000249087000BF00BF10BD0000C407002099
:103E3000142B00207047000010B50022FF219131A3
:103E4000104608F087FC0022FF219131012008F084
:103E500081FC00200AF0F6FD07F026FC07F07AFC52
:103E600007F090FC00F096FCF6F75CFF0220FCF7F0
:103E70007DFC002006490870FFF750F9FFF776F83F
:103E8000FFF79CF8F6F7AEFD00F084FD10BD0000D2
:103E90009C01002010B5012406F0E8FF012801D1A3
:103EA000052407E0F8F7A2FC0349884201D2012467
:103EB00000E00224204610BD204E000010B506246C
:103EC00006F0D4FF002800D1002406F0D5FF012819
:103ED00003D006F0D1FF072800D90924204610BDE1
:103EE00010B5F6F71FFF00221146012008F0A8FCCC
:103EF00000213A48F7F7E6F9002400BF00F000FF80
:103F000032217D200001FCF79FF800203449087021
:103F10000AE00022324801781046FEF727FE3048BA
:103F20000078401C2E4908702D4800782428F0DBCA
:103F300000202C49087009E000212A48007808F088
:103F400091F828480078401C2649087025480078D8
:103F50000D28F1DBFFF732F8F6F71AFC06F0D8FE71
:103F600021480078401C2049087008460078052840
:103F700012D300200870FFF70FF81C4800780A28B9
:103F800005D3002019490870FFF7E0F904E017484D
:103F90000078401C1549087006F06EFF0128ADD965
:103FA00006F06AFF0728A9D200200E49087008E031
:103FB0000C48007808F070F80A480078401C09495D
:103FC0000870084800780D28F2DBF6F71BFE552133
:103FD0000248F7F777F9204610BD000034080020AA
:103FE0001B010020190100201A0100201C010020E3
:103FF00010B5032408E000F083FE012000F08AFDE4
:10400000002801D0042400E0F5E700BF204610BDE1
:1040100010B500202D49086006F09EFA0120FCF73B
:10402000A5FBF7F74DFC55212948F7F74BF90AF0A6
:104030004DFCF6F767FBF9F785FEF6F7E3FD06F0B2
:1040400077FEF9F7B7FEFAF79FF8F8F7F9FEFFF7F2
:10405000E5FBFDF70FFFFFF7DDFCFFF74DFDFEF77A
:1040600035FF00F06BF8E12040020AF071F8F6F736
:104070002FFFFBF789FBFAF79FF8164AFF219131D2
:10408000002008F067FB134AFF219131012008F05E
:1040900061FB00221146104608F0A0FA002201211F
:1040A000104608F09BFA00220221104608F096FA0A
:1040B00000221146012008F091FA08F0CBF908F02F
:1040C00081FA0221012000F071FC10BD5000002097
:1040D000340800200090D00370B506460D46144603
:1040E0000E4806600E4805600E49206808600E49BB
:1040F000606808600D49A06808600D492069086083
:104100000C49E06808600C4960690860054800686F
:10411000002802D003480068804770BDC40000201A
:10412000CC000020AC000020B0000020B400002033
:10413000B8000020BC000020C000002000B587B0FF
:104140000C4801900C4802900C4803900020049009
:1041500005900B48069000200A49086048600A490B
:104160000860486001AA0121C9020848FFF7B4FFAE
:1041700007B000BD91410100D94401006144010034
:10418000E9430100E4140020DC0C0020EC190020BD
:1041900001207047F3B5C3B00446449E0020009050
:1041A00057E002E0641C761E00BF022E05D3207883
:1041B000EB28F7D160789028F4D1072E00D24AE09E
:1041C000A778FD1CB54200D945E0A81E205C00027E
:1041D000691E615C08434290042D38D9291FA01C38
:1041E0000AF08EFB4299884226D11D4800680028BB
:1041F00004D0B91EE01C1A4A12689047194800689A
:10420000002824D0E1786846017120798111684640
:10421000417120798106890E68468171381FC1B2CB
:104220006846C171C279611D02A8F4F720F801A89F
:104230000C49096888470AE00020009002E00098D5
:10424000401C00900098A842F9D300200090641907
:10425000761B072EA5D200BF4498801B45B0F0BD49
:10426000B8000020C0000020F7B5C0B015460026F9
:104270000027E81DFF210131884202DD002043B004
:10428000F0BDEB216846017090214170281DC1B23C
:10429000684681700021C1704098C1B268460171C2
:1042A0000524002605E04198805D69460855641C98
:1042B000761CAE42F7DBA11E00A802300AF020FBFC
:1042C00087B2381269460855641C0F55641C0648AD
:1042D0000068002805D021466846034A12689047C6
:1042E000CDE70020CBE70000B000002070B500242F
:1042F000002500261B4840681A490968884200D1F9
:1043000070BD1848406817490968884205D91548A2
:10431000406814490968451A07E0124800681149C5
:104320004968401A012189020D1AFF2D01D9FF2683
:1043300000E02E4600240DE00A4801680830405C89
:104340000949085507480088401C8005800D05492B
:104350000860641CB442EFD3B1B2034809F054FFC3
:1043600000BFCDE7E4140020EC18002070B5002554
:104370001A480068002830D0194A1288FF230133F8
:10438000991A184A1268164B1B88D018134A1268DB
:1043900090470546002D20D011480088401910494B
:1043A0000880084601880F480068FFF7F3FE0446BE
:1043B000002C0DDD0A480088844209DA084800888C
:1043C000021B08480068011906480068F3F74FFF10
:1043D00003480088001B0249088070BDB40000201B
:1043E000C8000020C400002010B50446A0781028A2
:1043F0000CD12079194908700846007801282BD182
:10440000002211462020FFF72FFF25E0A078122878
:1044100003D12079114908721EE0A07801281BD130
:104420002079332803D101200C49487005E0207918
:10443000352802D100200949487060790749887001
:10444000607A0006217A09040843E17909020843E9
:10445000A17908430149486010BD0000D00C00203C
:1044600070B503460022002400251A484068194E02
:104470003668B04201D1002070BD16484068154E24
:104480003668B04205D913484068124E3668841B1E
:1044900007E0104800680F4E7668801B0126F60280
:1044A000341AA14201D9254600E00D4600220CE055
:1044B000084806680830805D985406480088401C0B
:1044C0004005400D034E3060521CAA42F0D32846EE
:1044D000D2E70000DC0C002070B503460022002467
:1044E00015484068144D2D68A84208D3124840680A
:1044F000114D2D68401B0125AD022C1A04E00E4819
:1045000000680D4D6D68441BA14201D9012070BDAA
:1045100000220CE09D5C0848466808308555083844
:104520008088401C8005800D034D6860521C8A42C3
:10453000F0D30020EBE70000E414002010B502489F
:10454000FFF70EFB10BD000070F401000021014ACE
:104550001175704740600040014600BFF0200840E0
:1045600000110A23584302460807000F8018C0B202
:1045700070470146002204E0501CC2B208460A38C7
:10458000C1B20A29F8DA1007000E0843704700008C
:1045900010B5044601218020F6F71EFF607A01283D
:1045A00005D14248C078102108434049C870607A5C
:1045B000A22805D13E48007F802108433C49087766
:1045C000607A3B49087700203A4948770846407F9F
:1045D0002178084337494877E07B002805D0084612
:1045E000407F20210843334948773248407FC00844
:1045F000C000A17A08432F4948770846807FF721F9
:1046000008402C498877E078FFF7B3FF2949887480
:10461000A078FFF7AEFF2749C8746078FFF7A9FFBD
:10462000244908752078002805D10846007D2179A5
:10463000084320490875E079FFF79BFF1D498875FD
:104640006079FFF796FF1B494875A079FFF791FF46
:104650001849C875207AFFF78CFF16490876084676
:10466000807F4006400E8877E07A002806D0084612
:10467000807F402108430F49887703E00D48807F01
:104680000C498877A07BFFF774FF0A498876607B26
:10469000FFF76FFF0749C876207B08770846807FC1
:1046A000102188430349887710BD00002004024090
:1046B00060040440404F044010B504461B48807F0E
:1046C00001210843194988772078FFF752FF1749DD
:1046D00008756078FFF74DFF1449C874A078FFF79C
:1046E00048FF1249887420780C2806DD0846407F70
:1046F000082108430D49487709E00C48407F0B49E1
:1047000048770846007DE17808430849087507485E
:10471000807F400840000549887700BF0348807FBC
:10472000022108400028F9D110BD0000404F04408C
:1047300010B5002014490876162009F0C5FD0021A7
:10474000124801761248407F80210843104948777B
:104750000846807F012108430D49887700BF0C4837
:10476000807F022108400028F9D00948807F400856
:1047700040000749887700BF0548807F0221084034
:104780000028F9D110BD00004060004040610040A9
:10479000404F044010B50020074908700021202038
:1047A000F6F71AFE01210548017500200449087535
:1047B000152009F071FD10BD00500440406100401B
:1047C0004060004070B504460D46002C14D0002D0A
:1047D00012D0042D10D800F013F800280CD10026B8
:1047E00008E00649885D22460121F4F7BFFDA41CBC
:1047F000701CC6B2AE42F4DB70BD00008401002024
:1048000000200549897DC907C90F002901D0012071
:1048100000E00020704700000050044030B585B033
:1048200005460C46002003900490009001900290F1
:10483000072C0BDC0120A04081B268468181012158
:10484000C17303A90220FBF7ADF83EE0082C01D0AC
:10485000092C0BD10120A04081B268468181012141
:10486000C17303A90120FBF79DF82EE00A2C03D0A9
:104870000B2C01D00D2C0BD10120A04081B2684639
:1048800081810121C17303A90020FBF78BF81CE093
:104890000C2C01D00F2C0BD10120A04081B2684616
:1048A00081810121C17303A90E20FBF77BF80CE085
:1048B0000E2C0AD10120A04081B2684681810121DD
:1048C000C17303A90C20FBF76DF800216846017045
:1048D000C17041700121817000210171C1720D21EF
:1048E0008172FF21017200214172F4F79FFD03499B
:1048F0001520FDF7A1F905B030BD00004D450100C0
:1049000010B5002010490875152009F0C5FC0021DC
:104910000E4801751520002809DB00BF00BFC20644
:10492000D20E012191400A4A116000BF00BF00BFB2
:10493000084880798011032805D006480078802136
:1049400008430449087010BD4060004040610040C9
:1049500000E100E00050044010B5F4F761FE10BD26
:1049600010B501231A4600211846F6F7F1FC012282
:1049700011461046F6F762FDF6F74EFD034809F0C2
:1049800097FF02480249086010BD00000090D00364
:104990004807002000BF0448006904210843024979
:1049A000086130BF00BF704700ED00E0F3B585B08F
:1049B0000546002003900490EEB22804070E0F2F46
:1049C00054DA082E52DA002009E00C214143284A2B
:1049D000515AA94201D1044603E0411CC8B217282C
:1049E000F3D300BF0120B04086B20C2060432049C1
:1049F0004018C3780C20604340188278F8B23146E2
:104A00000190FBF773F868468681012181730021CC
:104A1000C17302214174F8B203A9FAF7C3FF0C2154
:104A20006143134A8918C888FBF7C6FF0C2060430E
:104A30000F494018C1886846018169460698887206
:104A400002A8FBF7D3FE0C226243094BD2189168EF
:104A50000C226243D21804201056FDF7EDF80C2109
:104A60006143034A8918C888FBF72AFF07B0F0BDE5
:104A700004F60100FEB505460C460020C043029036
:104A8000EFB22804060E0F2E42DA082F40DA01207A
:104A9000B8406946088080202040002816D10120B7
:104AA0008870A007800F022801D1487109E0A00793
:104AB000800F012802D16946487102E00020694652
:104AC0004871F0B26946FAF76DFF1FE000206946B1
:104AD00088700E202040002800D000BF1020204009
:104AE000002802D16946087102E001206946087178
:104AF000E007C00F002802D16946887102E001205A
:104B000069468871F0B26946FAF74CFF00200290BE
:104B10000298FEBD30B50146CAB20C04230E002037
:104B20000F2B0FDA082A0DDA01249440A2B2064CAA
:104B300003252D026419E45C1440002C01D00120EF
:104B400000E0002030BD000000000440F8B504463D
:104B50000F460020C0430090E6B22004050E0F2D42
:104B600011DA082E0FDA0120B04086B2002F04D1EE
:104B7000E8B23146FBF712F803E0E8B23146FBF742
:104B80001DF8002000900098F8BD00001649897FAC
:104B900001221143144A917700BF1349897F0222F1
:104BA00011400029F9D01049897C81700E49C97CD7
:104BB00041700D49097D01700B498A7D8271497DE3
:104BC00001710949CA7D42710A7EC271897F490813
:104BD0004900054A917700BF0349897F02221140AD
:104BE0000029F9D170470000404F044003B585B05B
:104BF00000200190029003900490002168464173C8
:104C0000817E01A8C1706846417E01A88170684616
:104C1000017E4171002101A80171082168460171DE
:104C2000817D01A8C1716846C17D4172417D01A8A5
:104C300081716846017D01A8017200216846817377
:104C4000C17301A881730C2141734121684601742D
:104C50000021C17401A8FFF79BFC1A200449888237
:104C600004491620FCF7E8FF00F006F807B000BD85
:104C7000204F0440FDE9010010B5FFF759FD10BDBC
:104C800070B504460D46601E0D49884200D90124C6
:104C9000002C00D1012440200A4908700846007801
:104CA0006043094948610321081F09F025FB0020E2
:104CB00005498861072008610448056070BD00004F
:104CC000FFFFFF007401002000E000E07001002001
:104CD0000020C043002809DBC206D20E012191400A
:104CE000054A1160BFF34F8FBFF36F8F00BF0020E5
:104CF000024908618861704780E100E000E000E05F
:104D000010B509F09FFA10BD1A20084908722B202F
:104D100048723C2088724D20C8727F20044909687F
:104D20000860AC200349487070470000000402404E
:104D3000780100200010024000B5184800780128D2
:104D400012D117480078642809DB02201549487100
:104D500008710020124908701049087004E01048DA
:104D60000078401C0E4908700F480078012814D1C3
:104D70000E480078012804D100200C4908700C4925
:104D800008700B480078322802DBF7F74FFE04E08A
:104D900007480078401C0649087000BD190700202C
:104DA0001807002008070020120700201407002021
:104DB00013070020F8B504460D4600270020009098
:104DC00003200003204000130090102C04D0122C6C
:104DD00002D01148844217D122202840222806D12F
:104DE00027073F0F39460098F5F778FC0646122052
:104DF000284012280ED12007000F471C3946009882
:104E0000F5F76CFC064605E02107090F0098F5F759
:104E100065FC06463046F8BD10100000FFB58BB0AB
:104E20001C460020079006900590384804901021F9
:104E30000B980840002801D0022707E040210B987A
:104E40000840002801D0012700E00027002C04D0F2
:104E5000149804700120089001E0102008900025AB
:104E600048E0002C08D025466000294A115A0C98C9
:104E7000F3F766F9079006E06800254A115A0C9886
:104E8000F3F75EF907903E4630E0711C0798F3F7A0
:104E900057F9400806900D98F3F7A8FA03900D9A79
:104EA0000699881AF3F7A2FA18490190F3F723FA42
:104EB00002900399F3F75CFA05900598F3F79DFAD1
:104EC00049004908039102900498F3F796FA4900C3
:104ED000490801910090039B029AF3F7A3FA03D2C9
:104EE0000A95099605980490701CC6B27F2ECCDDF9
:104EF000681CC5B208988542B3DB14990A980870FB
:104F000014990998487004980FB0F0BD0000C84289
:104F100018F701000246412A2ED010DC212A2AD09F
:104F200006DC102A45D0122A4BD0202A59D11CE089
:104F3000222A26D0232A2AD0402A52D116E08123C1
:104F40005B01D01A9A4228D008DC422A1AD0432AA0
:104F50001ED025481018002843D13AE0012822D05D
:104F600020281BD021283CD11EE000BF1F48038908
:104F70000B43038136E000BF1C4843890B43438148
:104F800030E000BF194883890B4383812AE000BFCA
:104F90001648C3890B43C38124E000BF14488388AB
:104FA0000B4383801EE000BF1148C3880B43C380BE
:104FB00018E00E4843890B43438103890B43038167
:104FC00010E00A48C3890B43C38183890B43838163
:104FD00008E00748C3880B43C38083880B43838062
:104FE00000E000BF00BF7047F0EFFFFF001104407A
:104FF00000140440F0B505460E46412D30D010DCBB
:10500000212D2CD006DC102D51D0122D56D0202D64
:1050100062D11CE0222D2AD0232D30D0402D5BD12F
:1050200016E081214901681A8D4230D008DC422DFA
:105030001ED0432D24D02A48281800284CD144E003
:1050400001282CD0202823D0212845D128E000BFDA
:10505000244F3888314600F049F804463DE000BF4F
:10506000204F7888314600F041F8044635E000BF13
:105070001C4FB888314600F039F804462DE000BFD7
:10508000184FF888314600F031F8044625E000BF9B
:10509000154F3888314600F029F804461DE000BF5E
:1050A000114F7888314600F021F8044615E00D4F85
:1050B0007888314600F01AF804460EE0094FF88867
:1050C000314600F013F8044607E0074F7888314670
:1050D00000F00CF8044600E000BF00BF2046F0BD21
:1050E000F0EFFFFF001104400014044002460020CE
:1050F00013460B40002B01D0012000E00020704738
:10510000FFB581B00E461746012F07D1F748407D05
:1051100000090001C01DF549487505E0F348407DD0
:1051200000090001F1494875049801287ED10A213F
:105130000198F3F705F80546ED48445DE007C00F18
:10514000002807D0E948007C00090001C01DE7499C
:10515000087405E0E548007C00090001E349087493
:1051600002202040002807D0E048C07BF02188437F
:105170007030DE49C87305E0DC48C07BF02188430D
:10518000DA49C87304202040002807D0D748807C23
:1051900000090001C01DD549887405E0D348807C12
:1051A00000090001D149887408202040002807D058
:1051B000CE48407CF02188437030CC49487405E0EB
:1051C000CA48407CF0218843C849487410202040D8
:1051D000002807D0C548407C00090001C01DC34914
:1051E000487405E0C148407C00090001BF4948748B
:1051F00020202040002807D0BC48007CF0218843B4
:105200007030BA49087405E0B848007CF021884342
:10521000B649087440202040002808D0B348807C5C
:10522000F02188437030B149887406E08BE0AF48C4
:10523000807CF0218843AD4988740A210198F2F7F7
:105240007FFF0D46AA48445DE007C00F002807D045
:10525000A648807BF02188437030A449887305E01C
:10526000A248807BF0218843A04988730220204017
:10527000002807D09D48807B00090001C01D9B4984
:10528000887305E09948807B00090001974988737D
:1052900004202040002807D09448007DF021884356
:1052A00070309249087505E09048007DF0218843F0
:1052B0008E49087508202040002807D08B48007DC3
:1052C00000090001C01D8949087505E08748007D77
:1052D000000900018549087510202040002807D0EA
:1052E0008248C07CF021884370308049C87405E052
:1052F0007E48C07CF02188437C49C874202020402F
:10530000002807D07948C07B00090001C01D7749FB
:10531000C87305E07548C07B000900017349C87374
:1053200040202040002807D07048C07C00090001C0
:10533000C01D6E49C87454E06C48C07C000900016F
:105340006A49C8744DE06948007C0009000167495A
:1053500008740846C07BF02188436449C873084636
:10536000807C0009000188740846407CF021884355
:105370005E4948740846407C0009000148740846AC
:10538000007CF0218843594908740846807CF0214C
:105390008843564988740846807BF02188435349E6
:1053A00088730846807B0009000188730846007DE9
:1053B000F02188434D4908750846007D0009000129
:1053C00008750846C07CF02188434849C8740846DF
:1053D000C07B00090001C8730846C07C00090001B9
:1053E000C8740A9801287DD10A213046F2F7A8FE38
:1053F00005463F48445DE007C00F002807D03B4802
:10540000407B00090001C01D3849487305E037485A
:10541000407B0009000135494873022020400028E4
:1054200007D03248007BF021884370302F49087341
:1054300005E02E48007BF02188432C4908730420A6
:105440002040002807D02948807DF0218843703013
:105450002649887505E02548807DF0218843234949
:10546000887508202040002807D02048807D00094A
:105470000001C01D1D49887505E01C48807D00099C
:1054800000011A49887510202040002807D01748CD
:10549000407DF021884370301449487505E0134879
:1054A000407DF02188431149487520202040002884
:1054B00007D00E48407BF021884370300B49487379
:1054C00005E00A48407BF0218843084948734020A2
:1054D000204000280ED00548C07D00090001C01DF5
:1054E000024900E092E0C8750AE00000EC210020CB
:1054F00068F101006D48C07D000900016B49C87565
:105500000A213046F2F71CFE0D466948445DE0076B
:10551000C00F002807D06548C07AF021884370305A
:105520006249C87205E06148C07AF02188435F494A
:10553000C87202202040002807D05C48C07A0009C9
:105540000001C01D5949C87205E05848C07A0009D9
:1055500000015649C87204202040002807D0534853
:10556000407E00090001C01D5049487605E04F48C3
:10557000407E000900014D4948760820204000285F
:1055800007D04A48007EF0218843703047490876AA
:1055900005E04648007EF021884344490876102003
:1055A0002040002807D04148007E00090001C01DAE
:1055B0003E49087605E03D48007E000900013B4970
:1055C000087620202040002807D03848007B0009BA
:1055D0000001C01D3549087305E03448007B00090F
:1055E00000013249087340202040002807D02F488E
:1055F000C07DF021884370302C49C87554E02B4899
:10560000C07DF02188432949C8754DE02748407B7B
:1056100000090001254948730846007BF0218843B2
:10562000224908730846807DF02188431F49887508
:105630000846807D0009000188750846407DF021FC
:1056400088431A4948750846407BF021884317492A
:1056500048730846C07D00090001C8750846C07A35
:10566000F02188431149C8720846C07A0009000138
:10567000C8720846407E0009000148760846007E50
:10568000F0218843094908760846007E0009000198
:1056900008760846007B0009000108730846C07DB3
:1056A000F02188430149C87505B0F0BDEC21002008
:1056B00068F10100FFB581B00E4617460198012838
:1056C0007ED10498002828D1FB480078012824D0F6
:1056D000F7F792F8F94988421FD3FAF7F7FE002846
:1056E0000DD0F748807DF02188437030F4498875EB
:1056F0000846C07C00090001C01DC8741AE0F048CB
:10570000807DF02188431030ED4988750846C07CC3
:1057100000090001401CC8740CE0E948807DF021BC
:1057200088437030E64988750846C07C000900014E
:10573000C01DC874E248C07CF02188437030E04945
:10574000C8740846007EF02188437030DC49087632
:105750000846807D00090001401C88750846407D90
:10576000F02188431030D64948750846407D00092D
:105770000001401C48750846007DF0218843103028
:10578000CF4908750846007D00090001401C0875D6
:10579000330008F073FD062E261E140C042FC84893
:1057A000007D00090001C01DC549087500BFC4483F
:1057B000007DF02188437030C149087500BF00E0CA
:1057C000AFE1BF48407D00090001C01DBC494875DC
:1057D00000BFBB48407DF02188437030B849487510
:1057E00000BFB748807D00090001C01DB44988751D
:1057F00000BF00E000BF00BF049800285ED1AE48A3
:10580000007801285AD0F6F7F7FFAC49884255D303
:10581000AB48C07FF0218843A949C8770846807FFC
:105820000009000188770846407FF0218843A44999
:1058300048770846007FF0218843A1490877084649
:10584000C07DF02188439E49C8750846C07F000985
:105850000001C8770846807FF021884398498877FF
:105860000846407F00090001C01D48770846807E39
:10587000F0218843924988760846807E000900011D
:1058800088760846407E0009000148760846007E7A
:105890000009000108760846007F0009000108772A
:1058A0000846C07EF02188438549C8760846407E78
:1058B000F0218843703082494876B8E16421384647
:1058C000F2F73EFC0546012D07D17D48C07FF0214F
:1058D000884370307A49C87705E07948C07FF02165
:1058E00088437749C8770A213846F2F729FC0A210C
:1058F0000090F2F725FC0D46642F02D37148445DF9
:1059000001E07148445DE007C00F002807D06C48F3
:10591000807F00090001C01D6949887705E068485B
:10592000807F000900016649887702202040002816
:1059300007D06348407FF021884370306049487742
:1059400005E05F48407FF02188435D4948770420A7
:105950002040002807D05A48007FF021884370304B
:105960005749087705E05648007FF021884354499D
:10597000087708202040002807D05148C07DF0213A
:10598000884370304E49C87505E04D48C07DF02110
:1059900088434B49C87510202040002807D048484C
:1059A000C07F00090001C01D4549C87705E0444893
:1059B000C07F000900014249C8772020204000280C
:1059C00007D03F48807FF021884370303C4988777A
:1059D00005E03B48807FF0218843394988774020A3
:1059E0002040002807D03648407F00090001C01D34
:1059F0003349487705E03248407F000900013049CB
:105A000048770A213846F2F79BFB0D462D48445D46
:105A1000E007C00F002807D02948807EF021884386
:105A200070302749887605E02548807EF02188433C
:105A30002349887602202040002807D02048807E15
:105A400000090001C01D1E49887605E01C48807EC3
:105A5000000900011A49887604202040002807D058
:105A60001748407E00090001C01D1549487605E031
:105A70001348407E00090001114948760820204063
:105A8000002807D00E48007E00090001C01D0C4907
:105A9000087605E00A48007E0009000108490876FA
:105AA00010202040002811D00548007F0009000187
:105AB000C01D034908770FE001010020B80B00006A
:105AC000C022002068F101007BF101005948007FED
:105AD000000900015749087720202040002807D0FE
:105AE0005448C07EF021884370305249C87605E0A2
:105AF0005048C07EF02188434E49C876402020405F
:105B0000002807D04B48407EF02188437030494937
:105B100048768CE04748407EF021884345494876E6
:105B200085E04448807D00090001424988750846A7
:105B3000407DF02188433F4948750846407D000973
:105B4000000148750846007DF021884339490875F1
:105B50000846007D0009000108750846C07C000960
:105B60000001C8740846807DF0218843314988755A
:105B70000846C07CF02188432E49C8740846007E40
:105B8000F02188432B4908760846C07FF0218843DE
:105B90002849C8770846807F0009000188770846B1
:105BA000407FF0218843234948770846007FF02151
:105BB0008843204908770846C07DF02188431D4965
:105BC000C8750846C07F00090001C8770846807F75
:105BD000F0218843174988770846407F0009000173
:105BE00048770846807EF021884312498876084627
:105BF000807E0009000188760846407E0009000189
:105C000048760846007E0009000108760846007FB5
:105C10000009000108770846C07EF0218843054945
:105C2000C8760846407EF02188430249487605B090
:105C3000F0BD0000C022002010B501460022002067
:105C40000A0EFE4B985CC307DB0F002B07D0FC4B02
:105C5000DB7FF024A3437033F94CE37705E0F84B86
:105C6000DB7FF024A343F64CE37702230340002BB1
:105C700007D0F34BDB7F1B091B01DB1DF04CE377E7
:105C800005E0EF4BDB7F1B091B01ED4CE3770423A1
:105C90000340002B07D0EA4B9B7F1B091B01DB1D38
:105CA000E74CA37705E0E64B9B7F1B091B01E44C07
:105CB000A37708230340002B09D0E14B20335B7806
:105CC0001B091B01DB1DDE4C2034637007E0DC4B3D
:105CD00020335B781B091B01D94C203463701023DF
:105CE0000340002B09D0D64B20331B78F024A3436C
:105CF0007033D34C2034237007E0D14B20331B7812
:105D0000F024A343CE4C2034237020230340002BE7
:105D100009D0CB4B20331B781B091B01DB1DC84C62
:105D20002034237007E0C64B20331B781B091B016E
:105D3000C34C2034237040230340002B07D0C04BBA
:105D40009B7FF024A3437033BD4CA37705E0BC4B8D
:105D50009B7FF024A343BA4CA377FF231B040B4083
:105D60001A0CB64B985CC307DB0F002B07D0B44B63
:105D70001B7F1B091B01DB1DB14C237705E0B04BDA
:105D80001B7F1B091B01AE4C237702230340002B12
:105D900007D0AB4BDB7EF024A3437033A84CE376F3
:105DA00005E0A74BDB7EF024A343A54CE376042358
:105DB0000340002B07D0A24B9B7EF024A3437033FB
:105DC0009F4CA37605E09E4B9B7EF024A3439C4C06
:105DD000A37608230340002B07D0994B5B7FF02468
:105DE000A3437033964C637705E0954B5B7FF024BB
:105DF000A343934C637710230340002B07D0904BB1
:105E00005B7F1B091B01DB1D8D4C637705E08C4B11
:105E10005B7F1B091B018A4C637720230340002B07
:105E200007D0874B1B7FF024A3437033844C237728
:105E300005E0834B1B7FF024A343814C2377402351
:105E40000340002B07D07E4BDB7E1B091B01DB1DB3
:105E50007B4CE37605E07A4BDB7E1B091B01784C1B
:105E6000E376FF231B020B401A0A744B985CC307AE
:105E7000DB0F002B07D0724B1B7EF024A343703343
:105E80006F4C237605E06E4B1B7EF024A3436C4CD5
:105E9000237602230340002B07D0694B1B7E1B098E
:105EA0001B01DB1D664C237605E0654B1B7E1B0941
:105EB0001B01634C237604230340002B07D0604B67
:105EC000DB7D1B091B01DB1D5D4CE37505E05C4BB5
:105ED000DB7D1B091B015A4CE37508230340002B93
:105EE00007D0574B9B7E1B091B01DB1D544CA3762F
:105EF00005E0534B9B7E1B091B01514CA3761023DD
:105F00000340002B07D04E4B5B7EF024A34370333D
:105F10004B4C637605E04A4B5B7EF024A343484C30
:105F2000637620230340002B07D0454B5B7E1B0983
:105F30001B01DB1D424C637605E0414B5B7E1B0978
:105F40001B013F4C637640230340002B07D03C4BA2
:105F5000DB7DF024A3437033394CE37505E0384B07
:105F6000DB7DF024A343364CE375CAB2334B985C17
:105F7000C307DB0F002B07D0314B1B7DF024A3435D
:105F800070332F4C237505E02D4B1B7DF024A3436C
:105F90002B4C237502230340002B07D0284B1B7D7D
:105FA0001B091B01DB1D264C237505E0244B1B7DC3
:105FB0001B091B01224C237504230340002B07D02F
:105FC0001F4BDB7C1B091B01DB1D1D4CE37405E033
:105FD0001B4BDB7C1B091B01194CE374082303409A
:105FE000002B07D0164B9B7CF024A3437033144C3A
:105FF000A37405E0124B9B7CF024A343104CA374C4
:1060000010230340002B07D00D4B5B7DF024A343EE
:1060100070330B4C637505E0094B5B7DF024A343A3
:10602000074C637520230340002B0BD0044B5B7D92
:106030001B091B01DB1D024C637509E068F10100BF
:10604000A02200200C4B5B7D1B091B010A4C6375D1
:1060500040230340002B07D0074BDB7CF024A343F5
:106060007033054CE37405E0034BDB7CF024A34361
:10607000014CE37410BD0000A022002000B50128EF
:106080007ED1FE4AD278F0239A437032FB4BDA700D
:106090001A46127912091201D21D1A711A46127982
:1060A000F0239A437032F54B1A711A46527912094D
:1060B0001201D21D5A711A465279F0239A43703256
:1060C000EE4B5A711A46D27912091201D21DDA71B9
:1060D0001A46D279F0239A437032E84BDA711A46A5
:1060E000527A12091201D21D5A721A46527AF023BC
:1060F0009A437032E14B5A721A46927AF0239A43CD
:106100007032DE4B9A721A469278F0239A437032BC
:10611000DA4B9A701A46D27A12091201D21DDA723B
:106120001A46527812091201D21D5A701A46D27AB2
:10613000F0239A437032D14BDA721A46203AD27F5A
:10614000F0239A437032CD4B203BDA77CB4A127B57
:1061500012091201D21D20331A731A46203A927F77
:1061600012091201D21D203B9A77C44A127BF023F8
:106170009A437032C14B1A731A46203A127F00E0DC
:10618000F2E1F0239A437032BC4B203B1A77BB4AB2
:10619000527B12091201D21D20335A731A46203A3B
:1061A000D27E12091201D21D203BDA76B44AD2788F
:1061B000F0239A437032B24BDA701A46127B1209FE
:1061C0001201D21D1A731A46127912091201D21D38
:1061D0001A711A46927AF0239A437032A84B9A7237
:1061E0001A461279F0239A437032A54B1A711A4657
:1061F000527912091201D21D5A711A469279120966
:106200001201D21D9A711A46127A12091201D21D78
:106210001A721A46127AF0239A437032984B1A7205
:106220001A46527A12091201D21D5A72934A927971
:1062300012091201521C914B9A711A469279F0235D
:106240009A4310328D4B9A711A46127A1209120132
:10625000521C1A721A46127AF0239A431032874B54
:106260001A721A46927A12091201521C9A721A462E
:10627000D27812091201521CDA701A469278120969
:106280001201521C9A701A465278F0239A43103227
:106290007A4B5A701A461278F0239A431032774B91
:1062A0001A701A46127812091201521C1A701A46F4
:1062B000203AD27F12091201521C203BDA771A468B
:1062C000927FF0239A4310326C4B203B9A771A4608
:1062D000527FF0239A431032684B203B5A771A467C
:1062E000527F12091201521C5A771A46127F120964
:1062F0001201521C1A771A46D27EF0239A431032AA
:106300005E4B203BDA761A46927EF0239A43103297
:106310005A4B203B9A765A4A127BF0239A4310320A
:10632000574B1A731A46D27AF0239A431032544BC1
:10633000DA721A46D27A12091201521CDA721A461D
:10634000927A12091201521C9A721A46527AF0235A
:106350009A4310324A4B5A721A465279F0239A43A2
:106360001032474B5A711A46D279F0239A431032B1
:10637000434BDA710B0007F081FF19F3E9DFD5CB4E
:10638000C1B7ADA3998F87786E645A50463E362EBA
:10639000261E160EF5003A4AD279F0239A4370323F
:1063A000374BDA7100BF364A5279F0239A43703284
:1063B000334B5A7100BF324A527AF0239A437032FB
:1063C0002F4B5A7200BF2E4A927A12091201D21D27
:1063D0002B4B9A7200BF2A4AD27A12091201D21D9F
:1063E000274BDA7200BF264AD27AF0239A437032E2
:1063F000234BDA7200BF224A127BF0239A43703299
:106400001F4B1A7300BF1D4A203A927EF0239A4315
:1064100070321A4B203B9A7600BF184A203AD27E3F
:10642000F0239A437032154B203BDA7600BF134AB3
:10643000203A127F12091201D21D104B203B1A770D
:1064400000BF0E4A203A527F12091201D21D0B4B97
:10645000203B5A7700BF094A203A527FF0239A43E3
:106460007032064B203B5A7700BF044A203A927F95
:10647000F0239A437032014B203B03E00C220020B2
:10648000E02200209A7700BFDC4AD27F1209120175
:10649000D21DDA4BDA7700BFD84A203212781209BF
:1064A0001201D21DD54B20331A7000BFD34A2032BF
:1064B0001278F0239A437032D04B20331A7000BF09
:1064C000CE4A20325278F0239A437032CB4B20339D
:1064D0005A7000BFC94A2032927812091201D21DA7
:1064E000C64B20339A7000BFC44A2032D2781209BA
:1064F0001201D21DC14B2033DA7000BFBF4A2032D7
:10650000927A12091201D21DBC4B20339A7200BF3D
:10651000BA4A2032127AF0239A437032B74B2033B2
:106520001A7200BFB54A2032127A12091201D21D26
:10653000B24B20331A7200BFB04A20329279F02356
:106540009A437032AD4B20339A7100BFAB4A203270
:10655000927912091201D21DA84B20339A7100BF03
:1065600001E0FFE700BF47E1A44A2032D278F023E0
:106570009A43A24B2033DA701A461279120912019B
:106580001A711A461279F0239A439C4B20331A71E0
:106590001A465279120912015A711A465279F02399
:1065A0009A43964B20335A711A46D2791209120136
:1065B000DA711A46D279F0239A43904B2033DA717C
:1065C0001A46527A120912015A721A46527AF02366
:1065D0009A438A4B20335A721A46927AF0239A438E
:1065E000864B20339A721A469278F0239A43834B53
:1065F00020339A701A46D27A12091201DA721A46B8
:106600005278120912015A701A46D27AF0239A432C
:106610007A4B2033DA72794AD27FF0239A43774B50
:10662000DA771A462032127B1209120120331A73CC
:10663000724A927F12091201203B9A771A46203241
:10664000127BF0239A436D4B20331A736B4A127FEF
:10665000F0239A43694B1A771A462032527B12096B
:10666000120120335A73654AD27E12091201203B6F
:10667000DA76634AD278F0239A43614BDA701A468D
:10668000127B120912011A731A46127912091201A9
:106690001A711A46927AF0239A43594B9A721A4603
:1066A0001279F0239A43564B1A711A4652791209FD
:1066B00012015A711A469279120912019A711A46F8
:1066C000127A120912011A721A46127AF0239A43A8
:1066D0004B4B1A721A46527A120912015A72474AE1
:1066E0002032927912091201444B20339A711A46D2
:1066F0009279F0239A43414B20339A711A46127AC9
:10670000120912011A721A46127AF0239A433B4B6D
:1067100020331A721A46927A120912019A721A4694
:10672000D27812091201DA701A469278120912010F
:106730009A701A465278F0239A43304B20335A709D
:106740001A461278F0239A432C4B20331A701A46BB
:106750001278120912011A70284AD27F1209120106
:10676000203BDA771A46927FF0239A43234B9A779D
:106770001A46527FF0239A43204B5A771A46527F8B
:10678000120912015A771A46127F120912011A775A
:106790001A46D27EF0239A43184BDA761A46927E36
:1067A000F0239A43154B9A76154A127BF0239A43AD
:1067B000134B1A731A46D27AF0239A43104BDA72AB
:1067C0001A46D27A12091201DA721A46927A12091C
:1067D00012019A721A46527AF0239A43084B5A725F
:1067E0001A465279F0239A43054B5A711A46D279C8
:1067F000F0239A43024BDA7100BD0000EC21002027
:10680000E022002070B505460C46012D7ED1B1482E
:10681000407D00090001C01DAE4948750846007D55
:10682000F02188431030AB4908750846007D000907
:106830000001401C08750846C07CF02188431030D8
:10684000A449C8740846807CF02188431030A149CF
:1068500088740846807C00090001401C8874F9F7A0
:1068600089FE02286ED19C48007801286AD0F5F78D
:10687000C3FF9A49884265D3F9F728FE00282FD034
:106880009448007DF021884370309249087508468D
:10689000007D00090001C01D08750846C07CF0217C
:1068A000884370308B49C8740846807CF021884347
:1068B0007030884988740846807C00090001C01D3A
:1068C00088740846407DF0218843703081494875BE
:1068D0000846407CF021884370307E494874F8E0D7
:1068E0007C48007DF021884310307A4908750846BD
:1068F000007D00090001401C08750846C07CF0219D
:10690000884310307349C874084600E0B4E0807CC6
:10691000F021884310306F4988740846807C000954
:106920000001401C88740846407DF02188431030E7
:10693000684948750846407CF02188431030654915
:106940004874C6E0F9F738FD002826D1F5F754FF62
:106950006249884221D3F9F7B9FD00280ED05D487D
:10696000407DF021884370305A4948750846407C84
:10697000F02188437030574948741CE05548407DE9
:10698000F02188431030534948750846407CF02177
:10699000884310304F4948740DE04E48407DF02147
:1069A000884370304B4948750846407CF021884345
:1069B000703048494874F9F7FFFC01282AD146484D
:1069C0000078012826D0F5F717FF4449884221D3E3
:1069D0004048407DF021884370303E494875084664
:1069E000407CF021884370303A494874F9F76EFDD5
:1069F000002807D03748007DF021884370303549A2
:106A0000087566E03348007DF02188431030314935
:106A100008755EE0230007F031FC062C241C140CE2
:106A2000042D2C48807C00090001C01D2949887470
:106A300000BF2848807CF021884370302549887445
:106A400000BF2448C07CF021884370302149C874BD
:106A500000BF2048007D00090001C01D1D490875C8
:106A600000BF1C48007DF02188437030194908752B
:106A700000BF00E000BF2CE01648407DF0218843B5
:106A8000144948750846007DF0218843114908756E
:106A90000846007D0009000108750846C07CF02109
:106AA00088430C49C8740846807CF0218843094912
:106AB00088740846807C0009000188740846407D7F
:106AC0000009000148750846407CF02188430149CF
:106AD000487470BD0C22002001010020B80B00009A
:106AE00030B50246002901D1002000E00720130044
:106AF00007F0C4FB0F09141F2B3743505D67727CEE
:106B000088929FA9B500574B5B7EF024A3430401F4
:106B1000F0252C402343534C6376A1E0524B9B79E4
:106B2000F024A3430401F0252C4023434E4CA371D1
:106B300096E04D4B2033DB791B091B010407240F22
:106B40002343494C2034E3718AE0464B2033DB7CFD
:106B50001B091B010407240F2343424C2034E37418
:106B60007EE0404B40331B781B091B010407240FB8
:106B700023433C4C4034237072E03A4B2033DB7F9C
:106B8000F024A3430401F0252C402343354C20344A
:106B9000E37765E0334B20335B7BF024A3430401B0
:106BA000F0252C4023432F4C2034637358E02E4BA8
:106BB0009B791B091B010407240F23432A4CA37153
:106BC0004EE0294B9B7CF024A3430401F0252C408C
:106BD0002343254CA37443E0234BDB7E1B091B019D
:106BE0000407240F2343204CE37639E01D4B203368
:106BF000DB7F1B091B010407240F2343194C20349E
:106C0000E3772DE0174B9B7E1B091B010407240F24
:106C10002343144CA37623E0134B20339B79F024B9
:106C2000A3430401F0252C4023430F4C2034A371CF
:106C300016E00D4BDB7D1B091B010407240F2343CA
:106C4000094CE3750CE0074B20335B7C1B091B01EF
:106C50000407240F2343034C2034637400E000BF77
:106C600000BF30BDEC210020C0220020F7B582B06B
:106C70000746154600260024FE480078012804D067
:106C8000F5F7BAFDFC49884279D2FC48407CF021F6
:106C900088437030F94948740846807C0009000137
:106CA000C01D88740846007D00090001C01D0875DC
:106CB0000846007DF02188437030F0490875084689
:106CC000807CF02188437030EC4988740846C07C91
:106CD00000090001C01DC8740846C07CF02188432B
:106CE0007030E649C8740846407C00090001C01DA8
:106CF00048740846407D00090001C01D48750846DB
:106D0000407DF02188437030DC4948750846007C9E
:106D1000F02188437030D94908740846007C000986
:106D20000001C01D08740846C07BF0218843703004
:106D3000D249C87300220A211046FBF717FF002230
:106D400013211046FBF712FF002211211046FBF71A
:106D50000DFF002212211046FBF708FF00220E2132
:106D60001046FBF703FF00220F211046FBF7FEFE43
:106D7000002210211046FBF7F9FEFDE3FFE7039820
:106D8000801E0F2878D243007B449B885B009F4481
:106D90000E007400D9003F01AC01100274027300B0
:106DA000730073007300DA023D037300A303B3485A
:106DB000407CF0218843B14948740846807C000932
:106DC000000188740846007D00090001C01D087597
:106DD0000846007DF02188437030A84908750846B0
:106DE000807CF0218843A54988740846C07C00094E
:106DF0000001C01DC8740846C07CF02188439F492B
:106E0000C8740846407C0009000148740846407D6B
:106E10000009000148750846407DF02188439749E4
:106E200048750846007CF021884394490874084658
:106E3000007C0009000108740846C07BF0218843EB
:106E40008E49C87364220A210020FBF78FFE64225A
:106E500013210020FBF78AFE00220E211046FBF7CB
:106E600085FE00220F211046FBF780FE0022102134
:106E70001046FBF77BFEF6E393E38048407CF0216D
:106E800088437E4948740846807C00090001887464
:106E90000846007D00090001C01D08750846007DF8
:106EA000F02188437030754908750846807CF021D0
:106EB0008843724988740846C07C00090001C87480
:106EC0000846C07CF02188436C49C8740846407C61
:106ED0000009000148740846407D00090001C01DFA
:106EE00048750846407DF021884364494875084646
:106EF000007CF0218843614908740846007C000941
:106F0000000108740846C07BF02188435B49C873C0
:106F100064220A210020FBF729FE642213210020AD
:106F2000FBF724FE00220E211046FBF71FFE002275
:106F30000F211046FBF71AFE002210211046FBF726
:106F400015FE90E34D48407CF02188434B4948743E
:106F50000846807C00090001C01D88740846007D39
:106F600000090001C01D08750846007DF021884316
:106F70007030424908750846807CF02188437030A3
:106F80003E4988740846C07C00090001C874084660
:106F9000C07CF02188433949C8740846407C000908
:106FA000000148740846407D000900014875084604
:106FB000407DF0218843314948750846007CF02126
:106FC00088432E4908740846007C000900010874B3
:106FD0000846C07BF02188432849C87364220A21EF
:106FE0000020FBF7C3FD642213210020FBF7BEFD48
:106FF00000220E211046FBF7B9FD00220F2110469A
:10700000FBF7B4FD002210211046FBF7AFFD2AE389
:107010001A48407CF0218843184948740846807C0F
:1070200000090001C01D88740846007D00090001A8
:10703000C01D08750846007DF021884370300F4957
:1070400008750846807CF02188430C4988740846FE
:10705000C07C00090001C8740846C07CF021884348
:107060000649C8740846407C00090001C01D4874E8
:10707000084605E001010020B80B00002C2200208A
:10708000407D0009000148750846407DF021884395
:10709000FE4948750846007CF0218843FB49087486
:1070A0000846007C0009000108740846C07BF021F6
:1070B0008843F649C87364220A210020FBF756FD75
:1070C000642213210020FBF751FD00220E211046FF
:1070D000FBF74CFD00220F211046FBF747FD002275
:1070E00010211046FBF742FDBDE2E848407CF0214C
:1070F0008843E64948740846807C0009000188748A
:107100000846007D0009000108750846007DF02151
:1071100088437030DD4908750846807CF02188433B
:10712000DA4988740846C07C00090001C874084622
:10713000C07CF02188437030D449C8740846407C34
:107140000009000148740846407D000900014875A7
:107150000846407DF0218843CC4948750846007CAC
:10716000F0218843C94908740846007C00090001E1
:1071700008740846C07BF0218843C449C873642260
:107180000A210020FBF7F2FC642213210020FBF708
:10719000EDFC00220E211046FBF7E8FC00220F2137
:1071A0001046FBF7E3FC002210211046FBF7DEFC43
:1071B00059E2B648407CF0218843B44948740846F7
:1071C000807C0009000188740846007D00090001E8
:1071D00008750846007DF02188437030AB4908757A
:1071E0000846807CF0218843A84988740846C07C02
:1071F00000090001C8740846C07CF0218843A349F7
:10720000C8740846407C0009000148740846407D67
:107210000009000148750846407DF0218843703020
:107220009A4948750846007CF021884397490874BC
:107230000846007C0009000108740846C07BF02164
:1072400088439249C87364220A210020FBF78EFC10
:10725000642213210020FBF789FC00220E21104636
:10726000FBF784FC00220F211046FBF77FFC002275
:1072700010211046FBF77AFCF5E18448407CF021B0
:1072800088437030814948740846807C00090001B9
:10729000C01D88740846007D00090001C01D0875E6
:1072A0000846007DF021884370307849087508460B
:1072B000807CF0218843754988740846C07C0009A9
:1072C0000001C8740846C07CF02188436F49C87427
:1072D0000846407C0009000148740846407D0009CA
:1072E000000148750846407DF0218843674948758C
:1072F0000846007CF0218843644908740846007CF5
:107300000009000108740846C07BF02188435F49EA
:10731000C87364220A210020FBF728FC6422132191
:107320000020FBF723FC00220E211046FBF71EFC79
:1073300000220F211046FBF719FC002210211046F5
:10734000FBF714FC8FE15148407CF02188434F4902
:1073500048740846807C0009000188740846007D56
:107360000009000108750846007DF021884347495F
:1073700008750846807CF021884344498874084693
:10738000C07C00090001C8740846C07CF021884315
:107390003E49C8740846407C00090001487408460C
:1073A000407D0009000148750846407DF021884372
:1073B000364948750846007CF021884333490874F3
:1073C0000846007C0009000108740846C07BF021D3
:1073D000884370302D49C87300220A211046FBF7FC
:1073E000C5FB002213211046FBF7C0FB64220E21CF
:1073F0000020FBF7BBFB00220F211046FBF7B6FB7A
:10740000002210211046FBF7B1FB2CE11F48407C05
:10741000F02188431D4948740846807C000900011A
:1074200088740846007D0009000108750846007D43
:10743000F0218843154908750846807CF02188436F
:10744000124988740846C07C00090001C8740846C7
:10745000C07CF02188430D49C8740846407C00096F
:10746000000148740846407D00090001487508463F
:10747000407DF0218843054948750846007CF0218D
:107480008843024908740846007C01E02C22002051
:1074900000090001C01D08740846C07BF021884324
:1074A000F949C87300220A211046FBF75FFB00224E
:1074B00013211046FBF75AFB00220E211046FBF762
:1074C00055FB64220F210020FBF750FB0022102106
:1074D0001046FBF74BFBC6E0EB48407CF0218843AD
:1074E000E94948740846807C000900018874084610
:1074F000007D0009000108750846007DF0218843E1
:10750000E14908750846807CF0218843DE4988748B
:107510000846C07C00090001C8740846C07CF02100
:107520008843D949C8740846407C00090001487462
:107530000846407D0009000148750846407DF0215D
:107540008843D14948750846007CF0218843703053
:10755000CD4908740846007C0009000108740846FB
:10756000C07BF0218843C849C87300220A21104615
:10757000FBF7FCFA002200E076E013211046FBF74F
:10758000F5FA00220E211046FBF7F0FA00220F2137
:107590001046FBF7EBFA642210210020FBF7E6FA15
:1075A00061E0B948407CF0218843B74948740846F7
:1075B000807C0009000188740846007D00090001F4
:1075C00008750846007DF0218843AF4908750846D4
:1075D000807CF0218843AC4988740846C07C00094F
:1075E0000001C8740846C07CF0218843A649C874CD
:1075F0000846407C0009000148740846407D0009A7
:10760000000148750846407DF02188439E49487531
:107610000846007CF02188439B4908740846007C9A
:107620000009000108740846C07BF0218843964990
:10763000C87300220A211046FBF798FA0022132192
:107640001046FBF793FA00220E211046FBF78EFA44
:1076500000220F211046FBF789FA00221021104664
:10766000FBF784FA00BF00BF002F76D064221121FF
:107670000020FBF77BFA642212210020FBF776FA48
:1076800082480078012804D0F5F7B6F8804988428E
:1076900016D28048807BF021884370307D49887302
:1076A000084640300078F0218843703079494031F5
:1076B00008700846007800090001C01D08702DE020
:1076C0007D20C000854214D27248807BF02188431F
:1076D00070498873084640300078F0218843703044
:1076E0006C494031087008460078000900010870B4
:1076F00014E06848807BF0218843703065498873C6
:10770000084640300078F0218843624940310870D3
:107710000846007800090001C01D08707D20C000E7
:10772000854205D201462846F0F70AFD064604E0E8
:1077300059492846F0F704FD06465848845DE0079D
:10774000C00F00280AD053484030C078000900011B
:10775000C01D50494031C87008E0A6E24D48403095
:10776000C078000900014B494031C8700220204018
:10777000002807D04748C07900090001C01D4549CD
:10778000C87105E04348C079000900014149C8714A
:1077900004202040002807D03E48807900090001DD
:1077A000C01D3C49887105E03A4880790009000114
:1077B0003849887108202040002807D03548407992
:1077C000F021884370303349487105E031484079F1
:1077D000F02188432F49487110202040002807D00D
:1077E0002C48407900090001C01D2A49487105E074
:1077F000284840790009000126494871202020408E
:10780000002807D023480079F021884370302149AF
:10781000087105E01F480079F02188431D4908716F
:1078200040202040002807D01A488079F021884362
:1078300070301849887105E016488079F021884336
:10784000144988717D20C000854207D264212846F2
:10785000F0F776FC06461148845D27E0642128464F
:10786000F0F76EFC7D21C9000090F0F769FC0191F2
:1078700064210198F0F764FC06460948854213D359
:107880000848845D12E000002C2200200101002045
:10789000B80B0000A0220020A08601007BF10100AF
:1078A0001027000068F10100F948845DE007C00F6F
:1078B000002807D0F7488078F02188437030F549D8
:1078C000887005E0F3488078F0218843F14988709A
:1078D00002202040002809D0EE484038807A000974
:1078E0000001C01DEB494039887207E0E948403883
:1078F000807A00090001E74940398872042020405D
:10790000002809D0E3484038407A00090001C01D32
:10791000E0494039487207E0DE484038407A0009C3
:107920000001DC494039487208202040002809D075
:10793000D8484038007AF02188437030D549403922
:10794000087207E0D3484038007AF0218843D149D3
:107950004039087210202040002809D0CD48403816
:10796000007A00090001C01DCA494039087207E0C9
:10797000C8484038007A00090001C64940390872F9
:1079800020202040002809D0C2484038C079F0218A
:1079900088437030BF494039C87107E0BD4840385E
:1079A000C079F0218843BB494039C871402020404C
:1079B000002809D0B7484038407AF0218843703019
:1079C000B4494039487207E0B2484038407AF02163
:1079D0008843B049403948727D20C000854210D2AA
:1079E0000A212846F0F7ACFB0A210190F0F7A8FB2A
:1079F0000E460A2D02D3A848845D11E0A448845D98
:107A00000EE064212846F0F79BFB0A210090F0F776
:107A100097FB0A210190F0F793FB0E469E498C5D7F
:107A2000E007C00F002807D09A48807800090001BD
:107A3000C01D9849887005E09648807800090001CB
:107A40009449887002202040002809D0914840388D
:107A5000807B00090001C01D8E494039887307E012
:107A60008C484038807B000900018A49403988737E
:107A700004202040002809D086484038407B000977
:107A80000001C01D83494039487307E081484038F0
:107A9000407B000900017F4940394873082020409D
:107AA000002809D07B484038007BF02188437030A3
:107AB00078494039087307E076484038007BF02168
:107AC000884374494039087310202040002809D0A9
:107AD00070484038C07A00090001C01D6D49403926
:107AE000C87207E06B484038C07A00090001694954
:107AF0004039C87220202040002809D0654840380D
:107B0000807AF0218843703062494039887207E0FA
:107B100060484038807AF02188435E494039887255
:107B200040202040002809D05A484038407BF021AE
:107B30008843703057494039487307E0554840380A
:107B4000407BF02188435349403948737D20C00071
:107B5000854207D20A212846F0F7F2FA0E464E482F
:107B6000845D0AE064212846F0F7EAFA0A210190D0
:107B7000F0F7E6FA0E4648498C5DE007C00F002892
:107B800007D044484078F02188437030414948701C
:107B900005E040484078F02188433E494870022083
:107BA0002040002807D03B48407800090001C01D54
:107BB0003849487005E037484078000900013549E8
:107BC000487004202040002809D032484038007C0A
:107BD000F021884370302F494039087407E02D4860
:107BE0004038007CF02188432A4940390874082035
:107BF0002040002809D027484038007C00090001B7
:107C0000C01D24494039087407E022484038007CF0
:107C1000000900011F494039087410202040002845
:107C200009D01C484038C07BF02188437030194986
:107C30004039C87307E017484038C07BF0218843BB
:107C400014494039C87320202040002809D0114829
:107C50004038C07B00090001C01D0E494039C8737F
:107C600007E00C484038C07B000900010949403951
:107C7000C87340202040002810D006484038407C7F
:107C800000090001C01D034940394874E8E00000C4
:107C90007BF10100E022002068F101007148407C86
:107CA000000900016F494874DAE000220A211046F9
:107CB000FAF75CFF002213211046FAF757FF002263
:107CC00011211046FAF752FF002212211046FAF74E
:107CD0004DFF00220E211046FAF748FF00220F2127
:107CE0001046FAF743FF002210211046FAF73EFF34
:107CF0005C484030C078000900015A494031C870E2
:107D00005848C079000900014039C8710846807997
:107D100000090001887108464079F02188435149E3
:107D20004871084640790009000148710846007909
:107D3000F02188434B49087108468079F021884337
:107D400048498871084640308078F0218843454989
:107D5000403188704348807A0009000140398872B8
:107D60000846407A0009000148720846007AF0216E
:107D700088433C4908720846007A000900010872ED
:107D80000846C079F02188433649C8710846407AD0
:107D9000F021884333494872084640308078000912
:107DA0000001403188702F48807B00090001403974
:107DB00088730846407B0009000148730846007B31
:107DC000F0218843274908730846C07A000900015A
:107DD000C8720846807AF021884322498872084692
:107DE000407BF02188431F49487308464030407863
:107DF000F02188431B49403148700846407800090B
:107E0000000148701748007CF02188431549087428
:107E10000846007C0009000108740846C07BF02178
:107E200088431049C8730846C07B00090001C87325
:107E30000846407C0009000148740846807BF02118
:107E4000884308498873084640300078F021884309
:107E500004494031087008460078000900010870A4
:107E600005B0F0BDA0220020F7B582B007460E464F
:107E70000121FF200830FCF769FE0121FC48FCF7D6
:107E800065FEFC48007801287ED0F4F7B5FCFA497D
:107E9000884279D3F8F79CFA032843D1F8F792FA8D
:107EA000002803D0F8F78EFA01283BD1002F1CD10F
:107EB000F8F70CFB00280CD0F048407CF0218843F8
:107EC000EE4948740846807C00090001C01D887492
:107ED000EEE0EA48407CF0218843E84948740846CF
:107EE000807C000900018874E2E0F8F7EFFA0028CE
:107EF0000CD0E248407CF02188437030DF49487460
:107F00000846807C000900018874D1E0DB48407C91
:107F1000F0218843D94948740846807C0009000153
:107F20008874C5E0F8F74EFA002803D0F8F74AFA4B
:107F3000012865D1002F0CD1D048407CF021884326
:107F4000CE4948740846807C00090001C01D887431
:107F50000BE0CA48407CF02188437030C749487420
:107F60000846807C000900018874F8F72BFA002885
:107F700021D1C2482030C078F02188437030BF49F9
:107F80002031C870BD4800E064E0807D0009000138
:107F9000203988750846807DF0218843B749887567
:107FA000642223210020FAF7E1FD0022222110465D
:107FB000FAF7DCFD7CE0F8F705FA012878D1AF4844
:107FC0002030C078F0218843AC492031C870AB48DC
:107FD000807D00090001C01D203988750846807D1C
:107FE000F02188437030A54988750022232110466E
:107FF000FAF7BCFD642222210020FAF7B7FD57E012
:108000009E48407CF02188439C4948740846807C07
:1080100000090001887408462030C078F0218843A8
:1080200096492031C8709548807D000900012039AB
:1080300088750846807DF021884390498875002224
:1080400023211046FAF792FD002222211046FAF76A
:108050008DFD2DE08948407CF021884370308749B0
:1080600048740846807C00090001C01D88740846D9
:108070002030C078F0218843703080492031C870AA
:108080007E48807D00090001C01D203988750846A2
:10809000807DF021884370307849887564222321DF
:1080A0000020FAF763FD642222210020FAF75EFD2A
:1080B000F8F788F9002808D06E480078012804D025
:1080C000F4F79AFB6C49884276D26D48864209D90A
:1080D0006A4820304079F021884370306749203168
:1080E000487107E0654820304079F02188436349B2
:1080F0002031487163493046F0F722F80A21019097
:10810000F0F71EF80D465E48401C864202D35E48DA
:10811000445D01E05D48445DE007C00F002809D0E0
:1081200056482030C07800090001C01D5349203155
:10813000C87007E051482030C078000900014F495D
:108140002031C87002202040002809D04B48203040
:108150008078F0218843703048492031887007E0EA
:10816000464820308078F021884344492031887087
:1081700004202040002809D0404820304078F021D9
:10818000884370303D492031487007E03B4820303B
:108190004078F02188433949203148700820204038
:1081A00000280AD035482030407900090001C01D60
:1081B00032492031487108E0A1E23048203040794E
:1081C000000900012D49203148711020204000286D
:1081D00009D02A4820300079F0218843703027499F
:1081E0002031087107E0254820300079F0218843CC
:1081F00022492031087120202040002809D01F4842
:108200002030007900090001C01D1C49203108718F
:1082100007E01A4820300079000900011749203191
:10822000087140202040002809D014482030807870
:1082300000090001C01D11492031887007E00F4876
:1082400020308078000900010C49203188707D21A0
:10825000C9003046EFF774FF0A210190EFF770FF75
:108260000D460848864213D30748445D12E00000DB
:108270000505000001010020B80B0000A02200202D
:108280009F8601001027000068F101007BF10100CA
:10829000F948445DE007C00F002807D0F748C07FC9
:1082A000F02188437030F549C87705E0F348C07F76
:1082B000F0218843F149C87702202040002807D0E8
:1082C000EE48C07F00090001C01DEC49C87705E0F9
:1082D000EA48C07F00090001E849C877042020402F
:1082E000002807D0E548807F00090001C01DE34950
:1082F000887705E0E148807F00090001DF49887741
:1083000008202040002809D0DC48203040780009AF
:108310000001C01DD9492031487007E0D7482030FE
:10832000407800090001D5492031487010202040D4
:10833000002809D0D14820300078F02188437030DF
:10834000CE492031087007E0CC4820300078F02179
:108350008843CA492031087020202040002809D0D5
:10836000C6482030007800090001C01DC3492031F3
:10837000087007E0C1482030007800090001BF49BB
:108380002031087040202040002807D0BB48807F63
:10839000F02188437030B949887705E0B748807F7D
:1083A000F0218843B549887764213046EFF7C8FE4D
:1083B0000A210190EFF7C4FE0D467D20C0008642E1
:1083C00002D3AF48445D01E0AB48445DE007C00F15
:1083D000002807D0A948007F00090001C01DA74957
:1083E000087705E0A548007F00090001A349087748
:1083F00002202040002807D0A048C07EF0218843FA
:1084000070309E49C87605E09C48C07EF0218843C4
:108410009A49C87604202040002807D09748807EDB
:10842000F021884370309549887605E09348807E36
:10843000F02188439149887608202040002807D001
:108440008E48407FF021884370308C49487705E0A2
:108450008A48407FF021884388494877102020408F
:10846000002807D08548407F00090001C01D8349CE
:10847000487705E08148407F000900017F4948773F
:1084800020202040002807D07C48007FF02188432E
:1084900070307A49087705E07848007FF0218843FA
:1084A0007649087740202040002807D07348C07ED6
:1084B00000090001C01D7149C87605E06F48C07E03
:1084C000000900016D49C8760A213046EFF738FEF1
:1084D0000A210190EFF734FE0D46642E02D368485E
:1084E000445D01E06448445DE007C00F002807D008
:1084F0006248007EF021884370306049087605E0CC
:108500005E48007EF02188435C49087602202040C6
:10851000002807D05948007E00090001C01D5749B6
:10852000087605E05548007E0009000153490876A9
:1085300004202040002807D05048C07D00090001D9
:10854000C01D4E49C87505E04C48C07D00090001BA
:108550004A49C87508202040002807D04748807E37
:1085600000090001C01D4549887605E04348807E2A
:10857000000900014149887610202040002807D0DA
:108580003E48407EF021884370303C49487605E003
:108590003A48407EF02188433849487620202040E0
:1085A000002807D03548407E00090001C01D33492E
:1085B000487605E03148407E000900012F494876A1
:1085C00040202040002807D02C48C07DF02188435F
:1085D00070302A49C87505E02848C07DF0218843DD
:1085E0002649C8750A213046EFF7AAFD0D462448F2
:1085F000445DE007C00F002807D02048007DF0212F
:10860000884370301D49087505E01C48007DF02145
:1086100088431A49087502202040002807D01748CF
:10862000007D00090001C01D1449087505E01348CC
:10863000007D000900011149087504202040002830
:1086400007D00E48C07C00090001C01D0B49C8744A
:1086500005E00A48C07C000900010849C8740820E8
:10866000204000280ED00548807CF02188437030DF
:10867000024988740CE000007BF10100A022002078
:1086800068F10100FA48807CF0218843F849887439
:1086900010202040002807D0F548407DF021884375
:1086A0007030F349487505E0F148407DF02188437A
:1086B000EF49487520202040002807D0EC48407D35
:1086C00000090001C01DEA49487505E0E848407D01
:1086D00000090001E649487540202040002807D0E5
:1086E000E348C07CF02188437030E149C8746DE2F2
:1086F000DF48C07CF0218843DD49C874F7E7F7F70D
:1087000061FE01287CD1DA4820304079F02188438D
:10871000D749203148710846C07800090001C87067
:1087200008468078F0218843D14920318870084676
:108730004078F0218843CE4920314870084640797E
:1087400000090001487108460079F0218843C849B2
:1087500020310871084600790009000108710846B7
:1087600080780009000188707D21C9000498EFF726
:10877000E7FC0546BF48445DE007C00F002807D06E
:10878000BB48C07FF02188437030B949C87705E005
:10879000B748C07FF0218843B549C8770220204000
:1087A000002807D0B248C07F00090001C01DB049B1
:1087B000C87705E0AE48C07F00090001AC49C87722
:1087C00004202040002807D0A948807F000900012C
:1087D000C01DA749887705E0A548807F00090001F2
:1087E000A34988770820204000280AD0A0482030DC
:1087F000407800090001C01D9D492031487008E003
:10880000ECE19B4820304078000900019849203174
:10881000487010202040002809D09548203000786A
:10882000F0218843703092492031087007E0904869
:1088300020300078F02188438D49203108702020B5
:108840002040002809D08A48203000780009000123
:10885000C01D87492031087007E085482030007826
:108860000009000182492031087040202040002882
:1088700007D07F48807FF021884370307C4988771B
:1088800005E07B48807FF02188437949887764211F
:108890000498EFF755FC0A210190EFF751FC0D46C3
:1088A0007D21C9000498884202D37348445D01E0E9
:1088B0007048445DE007C00F002807D06C48007F77
:1088C00000090001C01D6A49087705E06848007F7B
:1088D000000900016649087702202040002807D0DF
:1088E0006348C07EF021884370306149C87605E056
:1088F0005F48C07EF02188435D49C876042020404F
:10890000002807D05A48807EF021884370305849AB
:10891000887605E05648807EF02188435449887661
:1089200008202040002807D05148407FF02188438C
:1089300070304F49487705E04D48407FF02188432B
:108940004B49487710202040002807D04848407FF6
:1089500000090001C01D4649487705E04448407FB2
:10896000000900014249487720202040002807D014
:108970003F48007FF021884370303D49087705E08B
:108980003B48007FF0218843394908774020204048
:10899000002807D03648C07E00090001C01D3449B8
:1089A000C87605E03248C07E000900013049C8762B
:1089B0000A210498EFF7C4FB0A210190EFF7C0FBEE
:1089C0000D462D48445DE007C00F002807D0284819
:1089D000007EF021884370302549087605E0244860
:1089E000007EF0218843224908760220204000289A
:1089F00007D01F48007E00090001C01D1C490876F1
:108A000005E01B48007E0009000119490876042092
:108A10002040002807D01648C07D00090001C01D75
:108A20001349C87505E01248C07D000900011049CE
:108A3000C87508202040002807D00D48807E000916
:108A40000001C01D0A49887605E00948807E0009BA
:108A50000001074988761020204000280ED00448E5
:108A6000407EF02188437030014948760CE00000D8
:108A7000A02200207BF1010068F10100FE48407E49
:108A8000F0218843FC49487620202040002807D068
:108A9000F948407E00090001C01DF749487605E00D
:108AA000F548407E00090001F34948764020204007
:108AB000002807D0F048C07DF02188437030EE498F
:108AC000C87505E0EC48C07DF0218843EA49C875C7
:108AD0000A210498EFF734FB0D46E848445DE007AF
:108AE000C00F002807D0E448007DF0218843703093
:108AF000E149087505E0E048007DF0218843DE4942
:108B0000087502202040002807D0DB48007D0009BE
:108B10000001C01DD849087505E0D748007D00094F
:108B20000001D549087504202040002807D0D2480C
:108B3000C07C00090001C01DCF49C87405E0CE48C3
:108B4000C07C00090001CC49C874082020400028DE
:108B500007D0C948807CF02188437030C6498874AA
:108B600005E0C548807CF0218843C3498874102003
:108B70002040002807D0C048407DF0218843703055
:108B8000BD49487505E0BC48407DF0218843BA499D
:108B9000487520202040002807D0B748407D0009B4
:108BA0000001C01DB449487505E0B348407D000987
:108BB0000001B149487540202040002807D0AE4848
:108BC000C07CF02188437030AB49C87440E2AA48A9
:108BD000C07CF0218843A849C87439E2F7F7F2FB5A
:108BE00002287DD1A44820304079F0218843A24951
:108BF000203148710021A248F2F764FA552830D19B
:108C0000A048FDF719F89C482030C0780009000101
:108C100099492031C87008468078F02188439649E8
:108C20002031887008464078F021884392492031ED
:108C300048700846407900090001487108460079EB
:108C4000F02188438C4920310871084600790009D9
:108C5000000108710846807800090001C01D887075
:108C6000F6E189480078401C874908708248203026
:108C7000C07800090001C01D7F492031C870084636
:108C80008078F021884370307B4920318870084615
:108C90004078F0218843784920314870084640796F
:108CA00000090001487108460079F02188437030BE
:108CB0007149203108710846007900090001C01D82
:108CC00008710846807800090001C01D88706F484F
:108CD000007800280BD1FCF7AFFF00206A4900E0C4
:108CE00065E008706A4908606A490860B0E1664852
:108CF0000078642828DA684800786449097888424E
:108D000004DB62480078401E634908705F480278BF
:108D100062495F480068F6F7C3FA00280FD15E4841
:108D2000007880005D490858002808D05A4800782B
:108D3000800008585649086000205349087054487C
:108D40000068544908602DE04F480078642829DB0A
:108D500051480078401C50490870084600784B493B
:108D60000978884202DB00204B4908704A480078A5
:108D700080004A4908584649086000204249087066
:108D8000434800684349096888420BD1424800784B
:108D9000401C414908700846007880003F49085847
:108DA0003B4908603A480068FCF746FF50E1F7F796
:108DB00009FB03289AD1304820304079F0218843BC
:108DC0002D49203148710846C07800090001C01DB6
:108DD000C87008468078F021884327492031887080
:108DE00008464078F021884370302349203148708C
:108DF0000846407900090001C01D48710846007905
:108E0000F02188431C492031087108460079000987
:108E10000001C01D08710846807800090001C01DCE
:108E200088701548C07FF02188431349C8770846E9
:108E3000C07F00090001C8770846807F0009000153
:108E400088770846203040780009000120314870BA
:108E500008460078F0218843074920310870084609
:108E600000780009000108700348807FF0218843E2
:108E700001498877084613E0A022002068F101002C
:108E8000280800200B0B0B0B700000208200002034
:108E9000680000206C00002064000020B00B00205F
:108EA000007F00090001C01D08770846C07EF02140
:108EB000884370306749C8760846807EF021884331
:108EC0007030644988760846407FF02188437030CE
:108ED000604948770846407F00090001C01D487777
:108EE0000846007FF021884370305A4908770846C9
:108EF000C07E00090001C876F7F7A4FA002855D112
:108F00005448007EF0218843703052490876084664
:108F1000007E0009000108760846C07D00090001B6
:108F2000C8750846807E0009000188760846407EA4
:108F3000F02188437030474948760846407E000952
:108F40000001C01D48760846C07DF021884370307E
:108F50004049C8750846007DF021884370303D497E
:108F600008750846007D0009000108750846C07CA8
:108F700000090001C8740846807CF0218843354907
:108F800088740846407DF021884370303149487527
:108F90000846407D00090001C01D48750846C07C98
:108FA000F021884370302B49C87451E02948007E75
:108FB000F02188437030274908760846007E000972
:108FC0000001C01D08760846C07D00090001C01DD3
:108FD000C8750846807E0009000188760846407EF4
:108FE000F021884370301B4948760846407E0009CE
:108FF0000001C01D48760846C07DF0218843154910
:10900000C8750846007DF021884312490875084656
:10901000007D0009000108750846C07C00090001B8
:10902000C8740846807CF02188430A498874084641
:10903000407DF0218843074948750846407D000976
:10904000000148750846C07CF02188430149C87476
:1090500005B0F0BDA0220020FFB581B006461D4638
:10906000002000900027002E76D0FA488079F02169
:1090700088437030F749887108462038007FF02116
:1090800088437030F34920390877F3480078012885
:1090900073D0F3F7B1FBF14988426ED3F7F798F933
:1090A00004286CD1002D34D1EA482038807EF0218C
:1090B00088437030E74920398876E6480079F02106
:1090C00088437030E3490871F7F700FA002810D0A0
:1090D000E0482038807D00090001DE49203988758C
:1090E0000846807DF02188437030DA492039887540
:1090F000A5E0D8482038807D00090001D5492039F5
:1091000088750846807DF0218843D24920398875CA
:1091100095E0D0482038807EF0218843CD49203921
:109120008876CC480079F0218843CA490871F7F75E
:10913000CDF9002811D0C7482038807D00090001F2
:10914000C01DC449203988750846807DF0218843B8
:10915000C0492039887572E07CE3BE482038807DA4
:1091600000090001BB49203988750846807DF0213F
:109170008843B8492039887561E040E0FFE7002D59
:109180001FD1B4482038807D00090001B149203941
:1091900088750846807DF02188437030AD492039BC
:1091A00088750846807EF02188437030A9492039AF
:1091B0008876A8480079F02188437030A549087165
:1091C0003DE0A4482038807D00090001C01DA14970
:1091D000203988750846807DF02188439D492039D3
:1091E00088750846807EF02188439A492039887620
:1091F00098480079F0218843964908711FE0954806
:109200002038807D00090001C01D924920398875F1
:109210000846807DF021884370308E49203988755A
:109220000846807EF021884370308A49203988764C
:1092300088480079F02188437030864908710A987F
:1092400001287DD10A210298EEF77AFF0090844927
:1092500000980C5CE007C00F002807D07D48C0795B
:1092600000090001C01D7B49C87105E07948C0793B
:10927000000900017749C87102202040002807D06A
:109280007448807900090001C01D7249887105E0A9
:1092900070488079000900016E49887104202040DF
:1092A000002807D06B48407900090001C01D6949BA
:1092B000487105E067484079000900016549487137
:1092C00008202040002807D06248007AF021884317
:1092D00070306049087205E05E48007AF0218843EA
:1092E0005C49087210202040002807D05948007AB5
:1092F00000090001C01D5749087205E05548007A71
:10930000000900015349087220202040002807D09E
:109310005048C079F021884370304E49C87105E04B
:109320004C48C079F02188434A49C8714020204008
:10933000002809D047484079F0218843703000E088
:1093400097E04449487105E042484079F02188435C
:10935000404948710A210298EEF7F2FE0091404917
:1093600000980C5CE007C00F002807D03948C0788F
:1093700000090001C01D3749C87005E03548C078B4
:10938000000900013349C87002202040002807D09E
:1093900030488078F021884370302E49887005E08D
:1093A0002C488078F02188432A4988700420204086
:1093B000002807D027484078F0218843703025499D
:1093C000487005E023484078F021884321494870DF
:1093D00008202040002807D01E48407800090001DE
:1093E000C01D1C49487005E01A484078000900017A
:1093F0001849487010202040002807D015480079EF
:1094000000090001C01D1349087105E011480079E9
:10941000000900010F49087120202040002807D0D2
:109420000C48C078F021884370300A49C87005E0C4
:109430000848C078F02188430649C8704020204081
:1094400000280FD00348807800090001C01D0149A1
:1094500088705CE02C22002001010020B80B000085
:1094600068F10100F948807800090001F749887027
:109470004DE0F6484079F02188437030F349487157
:109480000846807800090001C01D88700846C07930
:1094900000090001C871084680790009000188713F
:1094A000084640790009000148710846007AF02119
:1094B0008843E64908720846007A000900010872EC
:1094C0000846C079F0218843E049C8710846C07851
:1094D00000090001C87008468078F0218843DB4904
:1094E000887008464078F0218843D849487008467B
:1094F0004078000900014870084600790009000121
:1095000008710846C078F0218843D049C8700B988C
:1095100001287DD10A210398EEF712FE0746CC48B8
:10952000C45DE007C00F002809D0C8482038407F3C
:1095300000090001C01DC5492039487707E0C3482C
:109540002038407F00090001C049203948770220B7
:109550002040002809D0BD482038007F00090001C4
:10956000C01DBA492039087707E0B8482038007F85
:1095700000090001B549203908770420204000285F
:1095800009D0B2482038C07E00090001C01DAF4993
:109590002039C87607E0AD482038C07E00090001B8
:1095A000AA492039C87608202040002809D0A748B9
:1095B0002038807FF02188437030A4492039887793
:1095C00007E0A2482038807FF02188439F49203956
:1095D000887710202040002809D09C482038807FC0
:1095E00000090001C01D99492039887707E0974894
:1095F0002038807F00090001944920398877202095
:10960000204000280BD091482038407FF02100E016
:10961000C5E0884370308D492039487707E08B4892
:109620002038407FF02188438849203948774020FE
:109630002040002809D085482038C07EF02188438A
:10964000703082492039C87607E080482038C07ED3
:10965000F02188437D492039C8760A210398EEF726
:109660006FFD0F467A48C45DE007C00F002809D09F
:1096700076482038407E00090001C01D734920391A
:10968000487607E071482038407E000900016F49A4
:109690002039487602202040002809D06B48203825
:1096A000007EF0218843703068492039087607E051
:1096B00066482038007EF0218843644920390876C6
:1096C00004202040002809D060482038C07DF021C7
:1096D000884370305D492039C87507E05B48203801
:1096E000C07DF021884359492039C87508202040A1
:1096F000002809D055482038C07D00090001C01D50
:1097000052492039C87507E050482038C07D00090B
:1097100000014E492039C87510202040002809D08A
:109720004A482038807E00090001C01D4749203981
:10973000887607E045482038807E000900014349CB
:109740002039887620202040002809D03F48203842
:10975000407EF021884370303C492039487607E04C
:109760003A482038407EF0218843384920394876ED
:1097700040202040002809D034482038007E0009CD
:109780000001C01D31492039087629E12F482038D1
:10979000007E000900012D492039087620E12B4880
:1097A0002038C07EF0218843703028492039C8769F
:1097B0000846007E00090001C01D08760846407F6B
:1097C0000009000148770846007F0009000108777A
:1097D0000846C07E00090001C8760846807FF02157
:1097E00088431A49203988770846807F000900019C
:1097F00088770846407FF02188431449203948770C
:109800000846407E0009000148760846007EF021A7
:1098100088430E49203908760846C07DF0218843E8
:109820000A492039C8750846C07D00090001C8757D
:109830000846807E0009000188760846407EF021B7
:109840008843024920394876CAE000002C220020D3
:1098500068F101006348C07EF02188436149C87601
:109860000846007E0009000108760846407F00098E
:10987000000148770846007F000900010877084684
:10988000C07E00090001C8760846807FF021884329
:10989000544988770846807F000900018877084688
:1098A000407FF02188434F4948770846407E0009B1
:1098B000000148760846007EF02188434949087631
:1098C0000846C07DF02188434649C8750846C07DDA
:1098D00000090001C8750846807E000900018876ED
:1098E0000846407EF02188433E49487608462030AD
:1098F0004079F02188433B492031487108468078FF
:109900000009000188700846C07900090001C8718B
:1099100008468079000900018871084640790009ED
:10992000000148710846007AF02188432D49203112
:1099300008720846007A0009000108720846C079DA
:10994000F021884327492031C8710846C0780009B2
:109950000001C87008468078F021884321492031F1
:10996000887008464078F02188431E4920314870AD
:10997000084640780009000148700846007900094F
:10998000000108710846C078F0218843154920314C
:10999000C8701448807D0009000120398875084688
:1099A000807DF02188430F4988750846807EF0212C
:1099B00088430C4988760846007FF021884309498E
:1099C0000877084620300079F02188430549203186
:1099D000087108468079F021884302492031887156
:1099E00005B0F0BD0C220020F7B582B00D46174639
:1099F0000026029801287CD1632D0ADD0121FF2079
:109A00000630FBF7A3F80121FF200730FBF79EF893
:109A100016E0092D0ADD0121FF200630FBF796F83C
:109A20000021FF200730FBF791F809E00021FF201B
:109A30000630FBF78BF80021FF200730FBF786F894
:109A4000FA48007801286ED0F2F7D6FEF84988422D
:109A500069D3F6F7BDFC032866D1002F30D1F6F7A5
:109A600035FD002816D0F348407BF0218843F149AA
:109A700048730846C07B00090001C01DC8736422FA
:109A800008210020F9F772F8002209211046F9F7A1
:109A90006DF890E0E748407BF0218843E549487342
:109AA0000846C07B00090001C87300220821104647
:109AB000F9F75CF8002209211046F9F757F87AE027
:109AC000F6F704FD002818D0DA48407BF0218843DF
:109AD0007030D84948730846C07B00090001C8733C
:109AE000002208211046F9F741F8642209210020DC
:109AF00000E0ACE1F9F73AF85DE0CE48407BF021B8
:109B00008843CC4948730846C07B00090001C873EC
:109B1000002208211046F9F729F8002209211046F1
:109B2000F9F724F847E02FE0002F16D1C148407B19
:109B3000F0218843BF4948730846C07B00090001F3
:109B4000C01DC873642208210020F9F70FF8002215
:109B500009211046F9F70AF82DE0B648407BF021BC
:109B600088437030B34948730846C07B0009000140
:109B7000C873002208211046F8F7F8FF6422092173
:109B80000020F8F7F3FF16E0AA48407BF021884355
